:100000000C94952A0C946FA10C9444A10C9419A102
:100010000C94EEA00C94C3A00C9498A00C946DA02A
:100020000C9442A00C94C62A0C94C62A0C94C62A9E
:100030000C94C62A0C94F1A10C94C62A0C94C62ADE
:100040000C94C62A0C94E1840C94C62A0C94C62AFB
:100050000C94C62A0C94C62A0C94F6730C949AA39A
:100060000C94C62A0D947E270D9422280C94C62A3F
:100070000C94C62A0C94C62A0C94C62A0C94C62A40
:100080000C94C62A0C94C62A0C94C62A0C94C62A30
:100090000C94C62A0C94C62A0C94C62A0C94C62A20
:1000A0000C94C62A0C94C62A0C94C62A0C94C62A10
:1000B0000C94C62A0C94C62A0C94C62A0C94C62A00
:1000C0000C94C62A0C94C62A0C94C62A0C94C62AF0
:1000D0000C94C62A0C94C62A0C94C62A0C94C62AE0
:1000E0000C94C62AA99CAC9C9B9C9F9CA59CE39CC1
:1000F000B09CB49CBA9CBE9CC29CC89CCC9CD09C1E
:10010000E39CD69CDA9CDE9CB6A2BBA2C0A2CAA28B
:10011000D4A24DA3DEA2E6A2EEA2F8A202A30CA3F3
:100120001BA325A34DA32FA339A343A3A3DF89DFDB
:100130008CDF8FDF92DF9EDF95DFACDF98DF9BDF08
:100140001001EA0006011A0122011401F200140153
:10015000E000F0001401DE0008010801EC00EC00F2
:10016000EC001C011C011C01E8000C010C010C013D
:10017000084AD73B3BCE016E84BCBFFDC12F3D6C0E
:1001800074319ABD56833DDA3D00C77F11BED9E474
:10019000BB4C3E916BAAAABE000000803F05A84C54
:1001A000CDB2D44EB93836A9020C50B99186880820
:1001B0003CA6AAAA2ABE000000803F000D94E927B1
:1001C0000D94DF270D9440100D94CD150D94BE0DA8
:1001D0000D94DC2A0D94B3270D94C82A0D94BB0D01
:1001E0000D94E3270D94DB270D94CF0B0D94521340
:1001F0000D947D140D9412110D94C70D0D94A9103A
:100200000D94CF230D94B80D0D94050F0D94C427B4
:100210000D94C12A0D9450050D94D62A0D94610CAD
:100220000D94AD270D947B110D94EC270D94D70FF1
:100230000D946E0F0D94CF270D94CF2A0D942D267B
:100240000D94DE220D94D7274E414E494E49545904
:10025000494E46CDCCCC3D0AD7233C17B7D1387791
:10026000CC2B329595E6241FB14F0A0000204100A7
:1002700000C84200401C4620BCBE4CCA1B0E5AAEF1
:10028000C59D7420746F6F206C6F6E6720657874E5
:10029000727573696F6E2070726576656E746564D1
:1002A0000A0020636F6C6420657874727573696FDF
:1002B0006E2070726576656E7465640A0047322F31
:1002C00047332062616420706172616D657465728C
:1002D000730A00536C6565702E2E2E0050726F628B
:1002E000696E67206661696C6564004D3131372045
:1002F000426564206C6576656C696E67206661692D
:100300006C65642E0A4730205A31300A4730204548
:10031000300A4D3330302050323520533838300ACF
:100320004D333030205035302053300A4D3330308B
:100330002050323520533838300A4D333030205079
:1003400035302053300A4D33303020503235205371
:100350003838300A4734205331004D31313720507E
:10036000726F6265207375636365737366756C0A7B
:100370000050524F4245204641494C20434C454194
:100380004E204E4F5A5A4C450A004D3130342053BE
:100390003137300A4D313137205265776970696ED7
:1003A00067206E6F7A7A6C650A4D3132310A4730B8
:1003B000205A31300A4732382058302059300A4DFF
:1003C00031303920523137300A4D313137205265C2
:1003D000776970696E67206E6F7A7A6C650A47314B
:1003E00032205030205331322054300A4D313034D5
:1003F00020533136300A4D3132300A4D31313720F9
:1004000050726F62696E672062656400205A3A20FC
:100410000020593A200042656420583A2000456E79
:10042000642066696C65206C6973740A00426567B4
:10043000696E2066696C65206C6973740A004D31C1
:100440003235005072696E742074696D653A20000F
:100450004C756C7A426F74204D696E69204C434430
:10046000204F66662E00544845524D414C5F505215
:100470004F54454354494F4E004155544F524550F7
:100480004F52545F53445F53544154555300454DAC
:10049000455247454E43595F5041525345520043E0
:1004A0004153455F4C494748545F4252494748547D
:1004B0004E45535300544F47474C455F4C494748BE
:1004C000545300534F4654574152455F504F574580
:1004D00052004255494C445F50455243454E5400EA
:1004E0004C4556454C494E475F44415441005A5F84
:1004F00050524F4245004155544F4C4556454C00D3
:100500005052494E545F4A4F420050524F47524555
:100510005353004155544F5245504F52545F544528
:100520004D5000564F4C554D45545249430045459A
:1005300050524F4D0053455249414C5F584F4E5F0A
:10054000584F4646004649524D574152455F4E412D
:100550004D453A4D61726C696E20204649524D57A7
:100560004152455F56455253494F4E3A312E312E36
:10057000392E33342045585452554445525F54590E
:1005800050453A4165726F73747275646572205399
:100590004F555243455F434F44455F55524C3A686F
:1005A000747470733A2F2F636F64652E616C65707D
:1005B000686F626A656374732E636F6D2F6469661A
:1005C000667573696F6E2F4D41524C494E205052E3
:1005D0004F544F434F4C5F56455253494F4E3A315B
:1005E0002E30204D414348494E455F545950453ABD
:1005F0004C756C7A426F74204D696E69204C43448F
:100600002045585452554445525F434F554E543A35
:100610003120555549443A30383366363866312DE5
:10062000303238652D343934632D393865312D66D3
:1006300032653064666165653961350A002F2F20A7
:10064000007A5F6D61783A20007A5F6D696E3A20BA
:1006500000795F6D61783A2000795F6D696E3A20AC
:1006600000785F6D61783A2000785F6D696E3A209E
:10067000005265706F7274696E6720656E64737482
:100680006F70207374617475730A0020466C6F7705
:100690003A200050726F6265205A204F666673657B
:1006A000743A2000496E76616C69642065787472D2
:1006B000756465720A0043290A0061626C656420F2
:1006C000286D696E2074656D702000436F6C642026
:1006D00065787472756465732061726520004B647F
:1006E000200023646566696E652044454641554C8B
:1006F000545F004B69200023646566696E65204481
:10070000454641554C545F004B702000236465669C
:10071000696E652044454641554C545F005049443C
:10072000204175746F74756E652066696E697368B3
:100730006564212050757420746865206C61737441
:10074000204B702C204B6920616E64204B64206329
:100750006F6E7374616E74732066726F6D20626564
:100760006C6F7720696E746F20436F6E6669677572
:10077000726174696F6E2E680A0050494420417599
:10078000746F74756E65206661696C656421207490
:10079000696D656F75740A00453120544845524DA6
:1007A000414C2052554E4157415900424544205436
:1007B0004845524D414C2052554E415741590054E5
:1007C0006865726D616C2052756E61776179004564
:1007D000312048656174696E67206661696C656483
:1007E000004265642068656174696E6720666169AE
:1007F0006C65640048656174696E67206661696C48
:10080000656400504944204175746F74756E6520AD
:100810006661696C6564212054656D7065726174F0
:1008200075726520746F6F20686967680A00204BD5
:10083000643A2000204B693A2000204B703A200097
:100840000A20436C617373696320504944200A0095
:100850002054753A2000204B753A2000206D6178B5
:100860003A2000206D696E3A200020643A20002072
:10087000626961733A2000504944204175746F7475
:10088000756E65206661696C656421204261642033
:100890006578747275646572206E756D6265720A32
:1008A00000504944204175746F74756E65207374EF
:1008B0006172740A0020643A0020693A0020703A9C
:1008C000004E6F2063617365206C696768740A006D
:1008D00020202020202846312E30203D2066756CB7
:1008E0006C20636F7272656374696F6E2C20463082
:1008F0002E30203D206E6F20636F727265637469C5
:100900006F6E290A002020466164653A202020206D
:1009100020202020202020202020202020460020D1
:1009200020536D6F6F7468696E6720286D6D293A6A
:10093000202020202020205300202044697374614F
:100940006E636520286D6D293A202020202020200C
:10095000205A004261636B6C61736820636F72722E
:10096000656374696F6E206973206163746976656D
:100970003A0A004261636B6C61736820636F727244
:10098000656374696F6E20697320696E6163746951
:1009900076653A0A004261636B6C617368206D652D
:1009A00061737572656D656E7420286D6D293A20CE
:1009B0002000496E736572742066696C616D656EA6
:1009C0007420616E64207072657373206275747434
:1009D0006F6E20286F72204D313038290A00507216
:1009E00065737320627574746F6E20286F72204D6A
:1009F0003130382920746F2068656174206E6F7AF9
:100A00007A6C650A00496E736572742066696C6160
:100A10006D656E7420616E64207072657373206200
:100A20007574746F6E20286F72204D313038290A2A
:100A3000003A200050726F6265205A204F6666733C
:100A40006574003F5A206F7574206F662072616E66
:100A5000676520282D3220746F2035290A003F4B0E
:100A60002076616C7565206F7574206F66207261E9
:100A70006E67652028302D3130292E0A00416476BA
:100A8000616E6365204B3D00416374697665204566
:100A9000787472756465723A2000496E76616C698B
:100AA000642065787472756465720A0025753A254C
:100AB00030327500253032753A2530327500257593
:100AC0006420253032753A25303275000006090061
:100AD000FE000000000001090008FE0000050808F3
:100AE00006000040F0C888889878100508080600BD
:100AF00000C0F88888888888F80505050600012068
:100B000030F830200508080600002070F82020206A
:100B100020E00509090600FF2070A8A8B8888870A1
:100B2000200509090600FFE080C0B0A82830282869
:100B30000509090600FFF8A88888888888A8F805AC
:100B40000A0A0600FE205050505088A8A88870035A
:100B5000030306000340A04000060900FE070192BF
:100B60000321207FFF07FF07FF00000006000001B0
:100B70000707060200808080808000800302020652
:100B80000105A0A00507070600005050F850F850D6
:100B9000500507070600002078A07028F020050700
:100BA00007060000C0C81020409818050707060077
:100BB000006090A040A89068020303060104C040B2
:100BC0008003070706010020408080804020030743
:100BD0000706010080402020204080050505060012
:100BE0000120A870A8200505050600012020F82096
:100BF000200203030602FFC0408005010106000336
:100C0000F8020202060200C0C00505050600010840
:100C100010204080050707060000708888888888B3
:100C20007003070706010040C040404040E0050750
:100C300007060000708808708080F8050707060026
:100C400000F81020100808F0050707060000103013
:100C50005090F81010050707060000F880F008080B
:100C60008870050707060000708080F0888870058E
:100C70000707060000F808102020202005070706B7
:100C8000000070888870888870050707060000706B
:100C9000888878080870020505060200C0C000C0F8
:100CA000C00206060602FFC0C000C040800407075D
:100CB00006000010204080402010050303060002BB
:100CC000F800F8040707060100804020102040804B
:100CD0000507070600007088081020002005070798
:100CE00006000070880868A8A870050707060000BD
:100CF000708888F8888888050707060000F08888CB
:100D0000F08888F0050707060000708880808088DA
:100D100070050707060000F08888888888F00507B6
:100D200007060000F88080F08080F80507070600BD
:100D300000F88080F080808005070706000070883A
:100D400080B8888870050707060000888888F888BA
:100D500088880107070602008080808080808005E7
:100D600007070600003810101010906005070706EE
:100D700000008890A0C0A0908805070706000080AA
:100D80008080808080F805070706000088D8A88842
:100D90008888880507070600008888C8A89888887A
:100DA000050707060000708888888888700507078F
:100DB000060000F08888F0808080050707060000A4
:100DC00070888888A89068050707060000F0888862
:100DD000F0A090880507070600007880807008085A
:100DE000F0050707060000F8202020202020050736
:100DF000070600008888888888887005070706002D
:100E000000888888888850200507070600008888A1
:100E1000888888A850050707060000888850205059
:100E2000888805070706000088888850202020054C
:100E30000707060000F80810204080F8030707069F
:100E40000100E08080808080E005050506000180CB
:100E500040201008030707060100E0202020202082
:100E6000E005030306000420508805010106000088
:100E7000F802020206020580400505050600007022
:100E8000087888780507070600008080B0C8888841
:100E9000F0050505060000708080887005070706CC
:100EA0000000080868988888780505050600007025
:100EB00088F880700507070600003048E040404091
:100EC000400506060600FF70888878087005070749
:100ED0000600008080B0C8888888010707060200E5
:100EE000800080808080800308080601FF200020A9
:100EF000202020A040040707060000808090A0C0AA
:100F0000A090030707060100C04040404040E005B4
:100F10000505060000D0A8A8A8A80505050600003C
:100F2000B0C8888888050505060000708888887024
:100F30000506060600FFF08888F080800506060694
:100F400000FF788888780808050505060000B0C805
:100F500080808005050506000070807008F0040799
:100F6000070600004040E04040403005050506000F
:100F700000888888986805050506000088888850DC
:100F8000200505050600008888A8A8500505050667
:100F9000000088502050880506060600FF888888D3
:100FA000780870050505060000F8102040F80307D2
:100FB000070601002040408040402001070706024C
:100FC00000808080808080800307070601008040C9
:100FD00040204040800502020600026890000000A8
:100FE000060000202020202020005A005900202048
:100FF0002020005800092000000000000000000030
:10100000000000003FFFF0000000000000000000B2
:101010000000003800700000000000000000000028
:10102000000030FC30000000000000000000000064
:101030000020FC1000000000000000000000000084
:1010400020781000000000000000000000000020D8
:1010500030100000000000000000000000002C0024
:10106000D03FC0000000000000002082002E31D0E0
:101070007FE0000000000000001041002F7BD07FC7
:10108000E0000000000000001041002F7BD07FE056
:10109000000000000000002082002E31D03FC00080
:1010A0000000000000004104002C00D03FC0000000
:1010B00000000000008208002030107FE0000000E7
:1010C000000000008208002078107FE0000000008F
:1010D00000000041040020FC107FE0000000000040
:1010E000000020820030FC301F8000000000000063
:1010F000000000003800700F000000000000000039
:10110000FFFFC03FFFF0060000000000000000FFEE
:10111000FFC0000000000000000000000000000010
:10112000003FFFF000000000000000000000000091
:1011300038007000000000000000000000000031D6
:10114000863000000000000000000000000023873F
:101150001000000000000000000000000027879041
:101160000000000000000000000000002F87D000F9
:1011700000000000000000000000002F03D03FC06E
:10118000000000000000002082002030107FE000FE
:101190000000000000001041002078107FE00000F7
:1011A00000000000001041002078107FE0000000E7
:1011B000000000002082002030103FC0000000002E
:1011C0000000004104002F03D03FC00000000000D9
:1011D00000008208002F87D07FE0000000000000A0
:1011E000008208002787907FE000000000000000D8
:1011F0004104002387107FE0000000000000002071
:1012000082003186301F80000000000000000000D6
:10121000003800700F0000000000000000FFFFC059
:101220003FFFF0060000000000000000FFFFC000CC
:10123000000020746F6F206C6F6E67206578747289
:101240007573696F6E2070726576656E7465640A79
:101250000020636F6C6420657874727573696F6EBB
:101260002070726576656E7465640A004E6F204367
:101270006865636B73756D2077697468206C696E3F
:1012800065206E756D6265722C204C617374204C04
:10129000696E653A200053544F505045442E20004B
:1012A0005072696E7465722073746F70706564201B
:1012B00064756520746F206572726F72732E20469C
:1012C000697820746865206572726F7220616E643F
:1012D00020757365204D39393920746F207265731C
:1012E000746172742E202854656D70657261747516
:1012F00072652069732072657365742E205365745E
:1013000020697420616674657220726573746172FD
:1013100074696E67290A004E6F20436865636B73BA
:10132000756D2077697468206C696E65206E756DC7
:101330006265722C204C617374204C696E653A2092
:1013400000636865636B73756D206D69736D61749F
:1013500063682C204C617374204C696E653A2000E0
:101360004C696E65204E756D626572206973206EE2
:101370006F74204C617374204C696E65204E756DDE
:101380006265722B312C204C617374204C696E6540
:101390003A20004D313130004D333100534420723A
:1013A000656164206572726F720A00446F6E652019
:1013B0007072696E74696E672066696C650A0020D8
:1013C000496E76616C6964206578747275646572C3
:1013D0002000000040C00000E0C0000000C000008D
:1013E000224300003E4300001F431000C9021001C9
:1013F0002C014001220170011801B0010E01F00121
:1014000004015002FA00B002F0003003E600D003FD
:10141000DC009004D2007005C800A006BE000008E1
:10142000B400B009AA00D00BA000600E96006011B5
:101430008C000015820020197800C01D6E00A022CB
:101440006400B0275A00902C500000314600E03470
:101450003C0010383200903A2800603C1E00A03D4D
:101460001400803E0A00203F00006265640A002CE0
:101470002073797374656D2073746F707065642167
:10148000204865617465725F49443A200042656492
:101490002068656174696E67206661696C656400C7
:1014A00048656174696E67206661696C65640045B2
:1014B000312048656174696E67206661696C656496
:1014C0000048656174696E67206661696C656400D7
:1014D0004B494C4C45442E20001000AD0330016AAE
:1014E0000150022B0170030A019004F500B005E5DC
:1014F00000D006D800F007CE001009C500300ABEA3
:1015000000500BB700700CB100900DAB00B00EA6F0
:1015100000D00FA200F0109D00101299003013951A
:10152000005014920070158E0090168B00B0178733
:1015300000D0188400F0198100101B7E00301C7B45
:1015400000501D7900701E7600901F7300B020704F
:1015500000D0216E00F0226B001024690030256657
:1015600000502663007027610090285E00B0295C5F
:1015700000D02A5900F02B5600102D5400302E5167
:1015800000502F4E0070304B0090314800B0324573
:1015900000D0334200F0343E0010363B0030373785
:1015A000005038330070392E00903A2900B03B23A8
:1015B00000D03C1B00F03D1100103F0100F03F0047
:1015C000004531204572723A204D415854454D50E6
:1015D000004572723A204D415854454D50204245C5
:1015E00044004D415854454D5020747269676765F9
:1015F000726564004531204572723A204D494E545F
:10160000454D50004572723A204D494E54454D505B
:1016100020424544004D494E54454D502074726956
:10162000676765726564004D383420582059205A28
:10163000204500202F002042403A0020403A00433D
:101640004F4D4D554E49434154494F4E0044525918
:1016500052554E004552524F525300494E464F008C
:101660004543484F0020573A0045787472756465C9
:101670007220436F6F6C696E672E2E2E0045787452
:1016800072756465722048656174696E672E2E2ECE
:101690000020573A0042656420636F6F6C696E6783
:1016A0002E2E2E004265642068656174696E672E77
:1016B0002E2E0060165B1654164D163F166F66668A
:1016C0000044454255473A004D3131332053004DD7
:1016D00031343520533C696E6465783E206F7574F3
:1016E000206F662072616E67652028302D31290ACF
:1016F00000205A3A0020593A0020436F756E74203A
:10170000583A0020453A00205A3A0020593A0058E9
:101710003A003A004361703A0020540020520041E0
:101720006363656C65726174696F6E3A2050002066
:101730005A00205900580020204D61783A2000209E
:101740005A00205900580020204D696E3A20004F61
:101750006E20004F666600536F667420656E64737A
:10176000746F70733A2000426564204C6576656C36
:10177000696E6720004661696C656420746F20653E
:101780006E61626C6520426564204C6576656C69AB
:101790006E670A00426564204C6576656C20436F75
:1017A0007272656374696F6E204D61747269783A04
:1017B000004F666673657473206170706C69656450
:1017C000004572723A20546F6F2066617221005496
:1017D0006F6F206661722066726F6D20726566653C
:1017E00072656E636520706F696E740A00454550BE
:1017F000524F4D204F4B0A0024F4D43050C38E205A
:10180000C2A24017828B7011127A910D816CD90A95
:10181000A861E108C7586607615143061E4B5D0584
:10182000C145A7041A411104093D980371393103D8
:101830004036DB0265339102D4305402802E1D0203
:10184000632CEE01752AC501B028A0011027810183
:101850008F2564012B244B01E0223401AC211F01B0
:101860008D200D01801FFC00841EED00971DDF0000
:10187000B81CD200E61BC600201BBC00641AB200D4
:10188000B219A8000A19A0006A189900D11791008E
:1018900040178B00B516840031167E00B315790011
:1018A0003A157300C7146F0058146A00EE136600EF
:1018B0008813630025135E00C7125B006C1257008B
:1018C00015125400C111510070114F0021114B002D
:1018D000D61049008D104700461044000210420007
:1018E000C00F4000800F3E00420F3C00060F3B003F
:1018F000CB0E3800930E37005C0E3500270E3400F7
:10190000F30D3200C10D3100900D3000600D2E003E
:10191000320D2D00050D2C00D90C2B00AE0C29002A
:10192000850C29005C0C2700350C27000E0C2600C6
:10193000E80B2400C40B2400A00B23007D0B230024
:101940005A0B2100390B2100180B2000F80A1F0048
:10195000D90A1E00BB0A1E009D0A1D00800A1D0038
:10196000630A1C00470A1B002C0A1B00110A1A00FC
:10197000F7091A00DD091900C4091900AB0919009B
:10198000920917007B091800630917004C0916001B
:1019900036091600200916000A091500F508150079
:1019A000E0081400CC081400B8081400A4081400BF
:1019B000900813007D0812006B08130058081200ED
:1019C0004608120034081100230811001208110003
:1019D00001081100F0071000E0071000D007100008
:1019E000C0071000B0070F00A107100091070E00FC
:1019F00083070F0074070F0065070E0057070E00DE
:101A000049070E003B070D002E070E0020070D00B2
:101A100013070D0006070D00F9060C00ED060D007A
:101A2000E0060C00D4060C00C8060C00BC060C0036
:101A3000B0060C00A4060B0099060C008D060B00E6
:101A400082060B0077060B006C060B0061060A008D
:101A500057060B004C060A0042060A0038060A0028
:101A60002E060A0024060A001A060A0010060900BB
:101A700007060A00FD050900F4050900EB05090049
:101A8000E2050900D9050900D0050900C7050900CC
:101A9000BE050900B5050800AD050800A50509004B
:101AA0009C050800940508008C05080084050800C2
:101AB0007C050800740508006C0507006505080032
:101AC0005D050700560508004E050700470507009D
:101AD0004005080038050700310507002A05070002
:101AE000230507001C050600160507000F05070063
:101AF0000805060002050700FB040600F5040700C0
:101B0000EE040600E8040600E2040700DB04060019
:101B1000D5040600CF040600C9040600C30406006D
:101B2000BD040600B7040600B1040500AC040600BD
:101B3000A6040600A00405009B0406009504050009
:101B4000900406008A040500850405008004060050
:101B50007A04050075040500700405006B04050097
:101B600066040500610405005C04050057040500D7
:101B7000520405004D040500480405004304050017
:101B80003E0404003A040500350405003004040056
:101B90002C04050027040400230405001E0404008F
:101BA0001A04040016040500110404000D040400C6
:101BB000090405000404040000040400FC030400FC
:101BC000F8030400F4030400F0030400EC03040031
:101BD000E8030400E4030400E0030400DC03040061
:101BE000D8030400D4030400D0030400CC03040091
:101BF000C8030300C503030024F404D9201BC40C4C
:101C00005C0E9804C4095F0265077101F405F900D0
:101C1000FB04B30048048700C10369005803550062
:101C200003034500BE023A008402310053022A0039
:101C30002902250004022000E4011C00C80119004B
:101C4000AF01170098011400840113007101100006
:101C50006101100051010E0043010D0036010B001F
:101C60002B010B0020010B00150109000C010900DC
:101C700003010800FB000800F3000800EB00070068
:101C8000E4000600DE000600D8000600D2000600D0
:101C9000CC000500C7000500C2000500BD0004001F
:101CA000B9000400B5000400B1000400AD00040058
:101CB000A9000400A5000300A20003009F00040087
:101CC0009B000300980003009500020093000300AE
:101CD000900003008D0002008B00030088000200CA
:101CE0008600020084000300810002007F000200E1
:101CF0007D0002007B0002007900020077000100F5
:101D000076000200740002007200010071000200FF
:101D10006F0002006D0001006C0002006A0001000B
:101D20006900020067000100660001006500010013
:101D30006400020062000100610001006000010017
:101D40005F0002005D0001005C0001005B0001001B
:101D50005A0001005900010058000100570001001D
:101D6000560001005500010054000100530000001E
:101D70005300010052000100510001005000010019
:101D80004F0001004E0000004E0001004D00010018
:101D90004C0001004B0000004B0001004A00010014
:101DA0004900010048000000480001004700010010
:101DB000460000004600010045000000450001000B
:101DC0004400010043000000430001004200000005
:101DD00042000100410000004100010040000100FC
:101DE0003F0000003F0001003E0000003E000100F7
:101DF0003D0000003D0001003C0000003C000000F0
:101E00003C0001003B0000003B0001003A000000E4
:101E10003A000100390000003900010038000000DC
:101E200038000000380001003700000037000100D2
:101E300036000000360000003600010035000000CA
:101E400035000000350001003400000034000000BF
:101E500034000100330000003300000033000100B3
:101E600032000000320000003200010031000000AA
:101E7000310000003100010030000000300000009F
:101E8000300001002F0000002F0000002F00000094
:101E90002F0001002E0000002E0000002E00010087
:101EA0002D0000002D0000002D0000002D0001007D
:101EB0002C0000002C0000002C0000002C00010071
:101EC0002B0000002B0000002B0000002B00010065
:101ED0002A0000002A0000002A0000002A00010059
:101EE000290000002900000029000000290000004E
:101EF0002900010028000000280000002800000040
:101F00002800000028000100270000002700000032
:101F10002700000027000000270001002600000025
:101F20002600000026000000260000002600010018
:101F3000250000002500000025000000250000000D
:101F400025000000250001002400000024000000FE
:101F500024000000240000002400010023000000F1
:101F600023000000230000002300000023000000E5
:101F700023000000230001002200000022000000D6
:101F800022000000220000002200000022000100C8
:101F900021000000210000002100000021000000BD
:101FA00021000000210000002100010020000000AD
:101FB00020000000200000002000000020000000A1
:101FC0002000000020000000200001001F00000091
:101FD0001F0000001F0000001F0000001F00000085
:101FE0001F0000001F0001001E0000001E00000076
:101FF0001E0000001E000000C23100001C26000070
:10200000F4190000D80F0000EB080000C004000025
:1020100075020000400100002569730025696D20EC
:10202000256973002569682025696D20256973007D
:10203000256964202569682025696D20256973005C
:1020400025697920256964202569682025696D2026
:1020500025697300486F6D696E67206661696C65FC
:10206000640001050800FF060121023520FFFF077B
:10207000FF06FF09005022165680808080008015E0
:102080003353A0A0A00257575050F850F8505002B8
:1020900057572070A07028702013355580A040A09D
:1020A0002002475740A0A040A0A050251353808095
:1020B0008012265640808080804012265680404004
:1020C0004040800245559060F060900255552020B8
:1020D000F82020113353604080044151F0113353F4
:1020E00040E0400246561010204080801236564094
:1020F000A0A0A0A04012365640C0404040E002469A
:10210000566090106080F0024656F020601090609B
:102110000246562060A0F02020024656F080E010D3
:1021200090600246566080E0909060024656F01043
:1021300020204040024656609060909060024656D3
:10214000609090701060122555C0C000C0C011365C
:1021500056606000604080123656204080804020EB
:10216000034353F000F01236568040202040801286
:10217000365640A020400040015858304898A8A842
:10218000904030024656609090F09090024656E0A3
:1021900090E09090E0024656609080809060024609
:1021A00056E090909090E0024656F080E08080F0FB
:1021B000024656F080E0808080024656609080B0F3
:1021C00090600246569090F0909090123656E04003
:1021D000404040E002465670202020A04002465673
:1021E00090A0C0A0A0900246568080808080F0021F
:1021F000465690F0F090909002465690D0F0B0B0D5
:1022000090024656609090909060024656E0909002
:10221000E08080014757609090D0B0601002465631
:10222000E09090E0909002465660904020906012BE
:102230003656E04040404040024656909090909084
:102240006002465690909090606002465690909042
:10225000F0F090024656909060609090025656883A
:102260008850202020024656F010204080F0123680
:1022700056E080808080E00246568080402010102A
:10228000123656E020202020E016325240A00141B4
:1022900051F01622528040024454709090700246D1
:1022A000568080E09090E012345460808060024656
:1022B0005610107090907002445460B0C060024696
:1022C00056205040E040400145556090701060023B
:1022D00046568080E09090901236564000C04040B4
:1022E000E01137572000202020A040024656808071
:1022F00090E09090123656C040404040E002545466
:10230000D0A8A8A8024454E0909090024454609051
:102310009060014555E090E08080014555709070D7
:102320001010024454A0D0808012345460C020C0E9
:102330000246564040E04050200244549090907035
:10234000123454A0A0A04002545488A8A8500244BB
:102350005490606090014555909070906002445494
:10236000F02040F0024757304020C0204030221675
:1023700056808080808080024757C02040304020B7
:10238000C006425250A0FFFFFFFFFFFFFFFFFFFF0D
:10239000FFFFFFFFFFFFFFFFFFFFFFFFFFFFFFFF4D
:1023A000FFFFFFFFFFFFFF0900502216568000804D
:1023B0008080800146562070A0A0702002465620E2
:1023C00050E04050A0025555887050708802565613
:1023D0008850F820F8202217578080800080808065
:1023E0000247577080E0907010E0173151A00256FC
:1023F0005670A8C8C8A87014355560A06000E003E6
:10240000435350A050123353E02020143151E002C6
:10241000565670E8D8E8D870173151E0153353405C
:10242000A04012355540E04000E014355540A02052
:1024300040E0143555C020C020C016225240800113
:102440004555909090E08002565678E8E868282834
:1024500024115180112252408014355540C0404013
:10246000E014355540A04000E0034353A050A002C3
:102470004757808080A060F0200247578080A0D01E
:1024800010207002475780408060A0F0201236561E
:1024900040004080A04002475740206090F090905C
:1024A00002475720406090F090900247576090603C
:1024B00090F0909002475750A06090F090900247A3
:1024C0005790006090F0909002475760906090F0B5
:1024D000909002465670A0A0F0A0B00147576090BF
:1024E00080809060400247574020F080E080F002FA
:1024F00047572040F080E080F00247576090F0801E
:10250000E080F00247579000F080E080F0123757EB
:102510008040E0404040E01237572040E0404040DB
:10252000E012375740A0E0404040E0123757A0008B
:10253000E0404040E00256567048E8484870024784
:102540005750A090D0B09090024757402060909094
:10255000906002475720406090909060024757601B
:1025600090609090906002475750A060909090606B
:1025700002475790006090909060123353A040A0A3
:1025800002465670B0B0D0D0E0024757402090903D
:10259000909060024757204090909090600247577B
:1025A000609090909090600247579000909090902B
:1025B000600257571020885020202002465680E0A5
:1025C0009090E0800246566090A0A090A0024757ED
:1025D000402000709090700247572040007090900B
:1025E000700247572050007090907002475750A0DB
:1025F00000709090700246565000709090700247A4
:102600005760906070909070025454F068B07811E8
:102610003555608080604002475740200060B0C060
:102620006002475720400060B0C06002475760908A
:102630000060B0C060024656500060B0C060123703
:1026400057804000C04040E0123757204000C04053
:1026500040E012375740A000C04040E0123656A07C
:1026600000C04040E0024757A040A01070906002B8
:10267000475750A000E090909002475740200060DC
:10268000909060024757204000609090600247574A
:102690006090006090906002475750A0006090905A
:1026A000600246569000609090601235554000E000
:1026B000004002445470B0D0E002475740200090E0
:1026C00090907002475720400090909070024757BA
:1026D000609000909090700246569000909090709C
:1026E00001485820400090907090600147578080CA
:1026F000E090E080800147579000909070906001DA
:10270000050700FE0500FB01F220FFFE05FE05FEA9
:102710000200400215258080800080053242A0A082
:1027200002556550F850F8500146562070C030E010
:1027300020025565901020404802556560806890E1
:102740006805122280800225354080808040022565
:10275000358040404080043343A040A003334340D1
:10276000E0400122324080043141E0021121800228
:102770005565081020408002455560909090600299
:102780002535C040404040024555E0106080F002D1
:102790004555E0106010E00245552060A0F0200291
:1027A0004555F080E010E00245556080E090600201
:1027B0004555F01020404002455560906090600201
:1027C000455560907010600313238000800214242C
:1027D000800080800235452040804020033343E064
:1027E00000E00235458040204080024555E0106001
:1027F00000400255657088B8A870024555609090F9
:10280000F090024555E090E090E002354560808010
:102810008060024555E0909090E0023545E080E010
:1028200080E0023545E080E080800245557080B050
:1028300090700245559090F09090023545E04040F0
:1028400040E0024555301010906002455590A0C000
:10285000A09002354580808080E002556588D8A828
:10286000888802455590D0B0909002455560909070
:102870009060024555E09090E0800146566090904F
:10288000906010024555E09090E0900245557080B0
:102890006010E0023545E0404040400245559090D0
:1028A0009090600245559090A0A04002556588A880
:1028B000A8A8500245559090609090024555909080
:1028C000701060023545E0204080E0022535C08070
:1028D0008080C00255658040201008022535C04028
:1028E0004040C005324240A0024151F005223280F2
:1028F000400244547090907002455580E09090E002
:1029000002344460808060024555107090907002DF
:10291000445460B0C0600235452040E0404000466D
:102920005670909070106002455580E09090900233
:1029300015258000808080002737400040404040BF
:10294000800245558090A0E090021525808080800F
:1029500080025464F0A8A8A8024454E09090900229
:10296000445460909060004656E09090E080800073
:102970004656709090701010023444A0C0808002BF
:10298000445470C030E002354540E04040200244ED
:1029900054909090700244549090A040025464A8C7
:1029A000A85050023444A04040A000465690909059
:1029B000701060024454F02040F0023545604080C1
:1029C00040600215258080808080023545C040200F
:1029D00040C005425250A0FFFFFFFFFFFFFFFFFF77
:1029E000FFFFFFFFFFFFFFFFFFFFFFFFFFFFFFFFF7
:1029F000FFFFFFFFFFFFFFFF020040FFFFFFFFFFA2
:102A0000FFFFFFFFFFFFFFFFFFFFFFFFFFFFFFFFD6
:102A1000FFFFFFFFFFFFFFFFFFFFFFFFFFFFFFFFC6
:102A2000FFFFFFFFFFFFFFFFFFFFFFFFFFFFFFFFB6
:102A3000FFFFFFFFFFFFFFFFFFFFFFFFFFFFFFFFA6
:102A4000FFFFFFFFFFFFFFFFFFFFFFFFFFFFFFFF96
:102A5000FFFFFFFFFFFFFFFFFFFF01060D00FE0965
:102A6000016602D620FFFE0BFE0AFE0D0060221951
:102A700069808080808080800080183363A0A0A05F
:102A80000357675050F850F850500259692078A009
:102A9000A0702828F02002596948A8501020405002
:102AA000A89002586840A0A040A09890682813639E
:102AB000808080113B6B204040808080808040403F
:102AC00020113B6B80404020202020204040800689
:102AD000556520A870A8200455652020F8202011F5
:102AE0003363604080065161F811336340E0400277
:102AF0005969080810102040408080025969205010
:102B0000888888888850200259692060A020202069
:102B10002020F80259697088880810204080F80247
:102B20005969F80810207008088870025969101057
:102B300030505090F81010025969F88080B0C808E1
:102B400008887002596970888080F08888887002CF
:102B50005969F808101020204040400259697088D7
:102B60008888708888887002596970888888780891
:102B700008887011386840E040000040E04011389B
:102B80006840E04000006040800259690810204021
:102B90008040201008045464F80000F8025969804D
:102BA0004020100810204080025969708888081061
:102BB0002020002002596970888898A8A8B08078E1
:102BC0000259692050888888F8888888025969F0F5
:102BD00048484870484848F00259697088808080A9
:102BE00080808870025969F048484848484848F051
:102BF000025969F8808080F0808080F8025969F875
:102C0000808080F080808080025969708880808018
:102C10009888887002596988888888F888888888A0
:102C2000123969E040404040404040E00259693874
:102C30001010101010109060025969888890A0C080
:102C4000A09088880259698080808080808080F888
:102C50000259698888D8A8A888888888025969880C
:102C6000C8C8A8A8989888880259697088888888F0
:102C700088888870025969F0888888F08080808010
:102C8000015A6A70888888888888A87008025969FB
:102C9000F0888888F0A090888802596970888080C0
:102CA0007008088870025969F82020202020202010
:102CB00020025969888888888888888870025969BC
:102CC00088888888505050202002596988888888D0
:102CD000A8A8A8A850025969888850502050508848
:102CE0008802596988885050202020202002596984
:102CF000F808101020404080F8113B6BE080808085
:102D0000808080808080E00259698080404020106F
:102D1000100808113B6BE0202020202020202020DC
:102D2000E0085363205088015161F82A22628040F4
:102D3000025666700878889868025969808080F029
:102D400088888888F002566670888080887002596A
:102D5000690808087888888888780256667088F834
:102D600080887002596930484040F040404040003F
:102D700058687088888878088870025969808080CF
:102D8000B0C8888888881238684000C040404040F9
:102D9000E0004A6A10003010101010909060025944
:102DA0006980808090A0C0A09088123969C040409E
:102DB0004040404040E0025666D0A8A8A8A888023B
:102DC0005666B0C888888888025666708888888861
:102DD00070005868F0888888F08080800058687893
:102DE00088888878080808025666B0C88080808085
:102DF0000256667088601088700258684040F04043
:102E0000404048300256668888888898680256662E
:102E10008888885050200256668888A8A8A8500242
:102E2000566688502020508800586888888898689E
:102E3000088870025666F810204080F8015B6B1815
:102E400020202020C0202020201822196980808086
:102E5000808080808080015B6BC020202020182033
:102E6000202020C008536348A890FFFFFFFFFFFF0A
:102E7000FFFFFFFFFFFFFFFFFFFFFFFFFFFFFFFF62
:102E8000FFFFFFFFFFFFFFFFFFFFFF0D00602219A5
:102E9000698000808080808080800358682070A8CE
:102EA000A0A0A8702002596930484040E040404846
:102EB000B0035666887050507088025969888850EF
:102EC00050F820F8202022196980808080008080BE
:102ED0008080124A6A609080609090601090601AC2
:102EE0003262A0A00359697088A8D8C8D8A8887091
:102EF000045767700878887800F80356662850A051
:102F0000A05028045363F80808163161E00359699A
:102F10007088E8D8D8E8D888700A5161F8174464F6
:102F2000609090600357672020F8202000F8073554
:102F30006540A02040E007356540A04020C02A221F
:102F40006240800058688888888898E880800259A4
:102F50006978E8E8E8E868282828262161C0202266
:102F600062408007356540C04040E0045767708884
:102F700088887000F8035666A050282850A0025A8E
:102F80006A40C04040E00818283808025A6A40C029
:102F90004040E01028081038025A6A40A04020A0A3
:102FA0004818283808025969200020204080888865
:102FB00070025A6A40200020508888F88888025A97
:102FC0006A10200020508888F88888025A6A3048A1
:102FD0000020508888F88888025A6A2850002050BB
:102FE0008888F88888025A6A50500020508888F8EB
:102FF0008888025A6A20502020508888F8888802E1
:10300000596958A0A0A0B0E0A0A0B8005B6B708880
:10301000808080808088702040025A6A402000F8BA
:103020008080F08080F8025A6A102000F88080F0DA
:103030008080F8025A6A304800F88080F08080F87A
:10304000025A6A505000F88080F08080F8123A6A84
:10305000804000E04040404040E0123A6A2040009A
:10306000E04040404040E0124A6A609000E040404A
:10307000404040E0123A6AA0A000E040404040409A
:10308000E0025969F0484848E8484848F0025A6A5E
:103090002850008888C8A8988888025A6A4020006A
:1030A00070888888888870025A6A10200070888822
:1030B00088888870025A6A304800708888888888B2
:1030C00070025A6A28500070888888888870025A6E
:1030D0006A505000708888888888700355658850C9
:1030E000205088015B6B08709898A8A8A8C8C87081
:1030F00080025A6A40200088888888888870025A2E
:103100006A10200088888888888870025A6A304847
:103110000088888888888870025A6A505000888899
:103120008888888870025A6A102000888850202079
:10313000202002596980F0888888F08080800259B8
:1031400069609090A0A0908888B0025969402000E2
:10315000700878889868025969102000700878888B
:103160009868025969304800700878889868025950
:103170006928500070087888986802596950500092
:10318000700878889868025A6A3048300070087869
:10319000889868025666702870A0A8500058687019
:1031A000888080887020400259694020007088F82B
:1031B0008088700259691020007088F88088700239
:1031C00059693048007088F88088700259695050F9
:1031D000007088F8808870123969804000C04040D3
:1031E0004040E0123969204000C040404040E012B9
:1031F0004969609000C040404040E0123969A0A099
:1032000000C040404040E0025A6A50206010708880
:1032100088888870025969285000B0C888888888D2
:1032200002596940200070888888887002596910A6
:10323000200070888888887002596930480070883A
:10324000888888700259692850007088888888703A
:103250000259695050007088888888700357672029
:103260002000F8002020015868087098A8A8C870AD
:1032700080025969402000888888889868025969C6
:10328000102000888888889868025969304800882A
:10329000888888986802596950500088888888987A
:1032A00068005B6B10200088888898680888700028
:1032B0005A6A8080B0C88888C8B08080005B6B5034
:1032C0005000888888986808887000000000000016
:1032D00000000000000000000000000000000000EE
:1032E000000000000000000000000000000C0000D2
:1032F00000000000000C00000000000000120000B0
:103300000000000000230000000000000021000079
:1033100000000000004C800000000000005E800003
:1033200000000000009240000000000000A14000EA
:10333000000000000121200000000000027F90003A
:1033400000000000020010000000000007FFF8006D
:103350000000000004000800000000000800040055
:10336000000000000800060000000000100002003D
:1033700000000000301E010000000000207F8100DE
:103380000000000041FFE0800000000043FCF080EE
:1033900000000000873B7840000000018EDBFC60ED
:1033A000000000010FEBCC20000000021FEDB61062
:1033B000000000021FDEB6100000000439CD7F08B7
:1033C0000000000436E0FF08000000087EC0BB8457
:1033D000000000187F005D86000000107FC0ED82B5
:1033E000000000203CC07301000000203B337F013F
:1033F000000000701BE77E03800000C81DEEDE04A5
:10340000C00000880FDEDC04400001240FDF3C090F
:103410002000012607DBF8192000027203E7F013F1
:103420009000025101FFE02290000489007F802477
:1034300048000904801E004824000BFE400000DF05
:10344000F40010004000008002001FFFFFFFFFFF9C
:10345000FE0000000000000000000000000000006E
:10346000000000000000000000001022103C3C0E94
:103470001F00102210042211040010221008221133
:103480000400102210083C11040010221010221118
:10349000040010221020221104001E1C1E3C3C0EB1
:1034A0000400000000000000000000000000000018
:1034B000000000000000000000000000000000000C
:1034C00000000000000000000000000000000000FC
:1034D00000000000000000000000000000000000EC
:1034E00000000000000000000000000000000000DC
:1034F00000000000000000000000000000000000CC
:1035000000000000000000001FFFFFFFFFFFFF6042
:103510000000000001FF400000000000FF800000EC
:103520000000007F83CF00000C303F87FF80000C3D
:10353000301F867980000C000F8C30C7838C30E7F9
:103540008C30CFC7CC31F38C30DCECEC33B98C3021
:10355000D86C6C33198C30D06C0C33198C30D86C1F
:103560000C33198C30DC6C0E3B198C30CF7C079FF0
:10357000198C30C77C038F194000000000000260E6
:103580000000000000061FFFFFFFFFFFF820205093
:103590006C616E6E657242756666657242797465BD
:1035A000733A20002046726565204D656D6F727913
:1035B0003A2000436F6D70696C65643A204A616E11
:1035C00020313020323031390A00207C204175749E
:1035D000686F723A2028416C657068204F626A6596
:1035E00063747320496E632E2C204C756C7A426F85
:1035F0007420476974205265706F7369746F7279B3
:10360000290A004A616E203130203230313931339D
:103610003A34303A313000204C6173742055706474
:10362000617465643A2000312E312E390A004D61F3
:10363000726C696E0020536F6674776172652052F8
:10364000657365740A00205761746368646F67204E
:1036500052657365740A002042726F776E206F7531
:10366000742052657365740A002045787465726E23
:10367000616C2052657365740A00506F77657255EE
:10368000700A0073746172740A006175746F256941
:103690002E67006572726F722077726974696E6747
:1036A00020746F2066696C650A00456E6473746FE0
:1036B0007073202563202563202563202563002067
:1036C0005A3A0020593A0020583A00656E647374E3
:1036D0006F7073206869743A2000446F6E652073C0
:1036E0006176696E672066696C652E0A004D323915
:1036F00000473238205A0A47302058383020593194
:1037000039302046333030300A4D31313720507255
:10371000696E742061626F727465642E000000200F
:10372000002300260029002C002F00320000010099
:1037300000030106010901020A0A426564204C6582
:1037400076656C20436F7272656374696F6E204D8D
:1037500061747269783A00202B000A436F727265B7
:1037600063746564204265642048656967687420F5
:1037700076732E2042656420546F706F6C6F67798A
:103780003A0A00202B000A42656420486569676890
:103790007420546F706F6772617068793A0A2020E4
:1037A000202B2D2D2D204241434B202D2D2B0A2047
:1037B00020207C20202020202020202020207C0A67
:1037C000204C207C20202020282B29202020207CF9
:1037D00020520A2045207C2020202020202020204C
:1037E00020207C20490A2046207C20282D29204E9C
:1037F00020282B29207C20470A2054207C202020B0
:1038000020202020202020207C20480A2020207CEE
:1038100020202020282D29202020207C20540A2010
:1038200020207C20202020202020202020207C0AF6
:103830002020204F2D2D2046524F4E54202D2D2B31
:103840000A2028302C30290A004D65616E206F66F1
:103850002073616D706C656420706F696E74733A6B
:10386000200020643A200020623A200045716E203A
:10387000636F656666696369656E74733A20613A61
:1038800020003474682070726F626520706F696EFA
:10389000742C2064697374616E63652066726F6D49
:1038A00020706C616E653A200020284452595255B0
:1038B0004E2900473239204175746F2042656420DB
:1038C0004C6576656C696E67003F20284C2C522C45
:1038D000462C4229206F7574206F6620626F756ECA
:1038E00064732E0A003F50726F626520706F696EBC
:1038F00074732028592920697320696D706C617573
:103900007369626C652028322D32292E0A003F50DF
:10391000726F626520706F696E7473202858292059
:10392000697320696D706C61757369626C652028BC
:10393000322D32292E0A003F2856296572626F7394
:1039400065206C6576656C20697320696D706C61AB
:10395000757369626C652028302D34292E0A002089
:10396000204E6F7A7A6C653A2000200066696C619F
:103970006D656E742070757267650057616974209B
:10398000666F7200506C6561736520776169742E93
:103990000000436172642072656D6F766564004358
:1039A00061726420696E7365727465640000060953
:1039B00000FE06018902FE20FFFE07FE06FE000053
:1039C0000006000701060606020080808080008055
:1039D000030303060103A0A0A00507070600FF508C
:1039E00050F850F850500509090600FE2070A8A0B4
:1039F0007028A870200608080600FF40A84810207C
:103A00004854080507070600FF609090609890688A
:103A10000103030602038080800207070602FF40BD
:103A20008080808080400207070602FF804040407F
:103A30004040800505050600008850F850880505BF
:103A4000050600002020F820200204040602FEC023
:103A5000404080050101060002F802020206020051
:103A6000C0C0040606060100101020408080040635
:103A70000606010060909090906003060606010023
:103A800040C0404040E0040606060100609010205F
:103A900040F0040606060100F020601010E0050664
:103AA0000606000010305090F810040606060100CB
:103AB000F080E01010E00406060601006080E0904F
:103AC0009060040606060100F01010204040040635
:103AD00006060100609060909060040606060100F2
:103AE000609090701060020505060200C0C000C022
:103AF000C00207070602FEC0C000C04040800505A6
:103B0000050600001860806018050303060001F830
:103B100000F8050505060000C0300830C00407079E
:103B20000601006090106040004005060606000097
:103B30007090A8B08070050606060000205088F836
:103B40008888050606060000F088F08888F00406DC
:103B50000606010060908080906004060606010061
:103B6000E090909090E0040606060100F080E0806E
:103B700080F0040606060100F080E08080800406E4
:103B800006060100609080B0906004060606010001
:103B90009090F0909090030606060100E0404040AF
:103BA00040E005060606000038101010906004067C
:103BB0000606010090A0C0A0909004060606010031
:103BC0008080808080F005060606000088D8A8A8BE
:103BD000888804060606010090D0B09090900506F3
:103BE00006060000708888888870040606060100B2
:103BF000E09090E080800407070601FF609090D07D
:103C0000B06010040606060100E09090E090900479
:103C1000060606010060904020906005060606003A
:103C200000F8202020202004060606010090909035
:103C3000909060040606060100909090F060600588
:103C400006060600008888A8A8D88805060606008B
:103C500000885020205088050606060000888850FD
:103C6000202020040606060100F010204080F0030A
:103C70000606060100E080808080E004060606015A
:103C800000808040201010030606060100E020207E
:103C90002020E005030306000320508805010106EB
:103CA00000FEF80202020602048040040404060139
:103CB00000709090700406060601008080E09090ED
:103CC000E00404040601007080807004060606010A
:103CD0000010107090907004040406010060B0C0E1
:103CE00070040606060100205040E040400406062D
:103CF0000601FE60909070106004060606010080C8
:103D000080E09090900306060601004000C040400D
:103D1000E00308080601FE200060202020A04004E7
:103D200006060601008080A0C0A0900306060601DA
:103D300000C040404040E0050404060000D0A8A8B0
:103D400088040404060100E0909090040404060135
:103D500000609090600406060601FEE09090E0800E
:103D6000800406060601FE70909070101004040492
:103D7000060100A0D0808004040406010070C03059
:103D8000E00406060601004040E040502004040420
:103D90000601009090907004040406010090906069
:103DA0006005040406000088A8A850040404060165
:103DB00000906060900406060601FE90909070905E
:103DC00060040404060100F02040F0030707060128
:103DD00000204040804040200107070602FF80800D
:103DE00080808080800307070601008040402040DB
:103DF000408004020206010350A0FFFFFFFFFFFF07
:103E0000FFFFFFFFFFFFFFFFFFFFFFFFFFFFFFFFC2
:103E1000FFFFFFFFFFFFFFFFFFFFFF0000000600A7
:103E200007010606060200800080808080040606E6
:103E30000601FF2070A0A070200507070600FF30D4
:103E40004840F04040F8050505060000A85088509D
:103E5000A80506060600008850F820F8200107078C
:103E60000602FF808080008080800407070601FF33
:103E7000708060906010E0030101060105A0060754
:103E800007060000788494A494847803050506014D
:103E90000160A06000E00505050600002850A05064
:103EA00028040303060100F01010040101060102BA
:103EB000F00607070600007884B4A4A484780401FF
:103EC00001060105F0040303060102609060050786
:103ED000070600FF2020F8202000F8030505060152
:103EE0000140A02040E0030505060101C02040205C
:103EF000C002020206020440800405050601FF908C
:103F000090B0D08005060606000078E8E86828280A
:103F1000010101060202800202020602FE40800345
:103F2000050506010140C04040E00305050601010A
:103F300040A04000E0050505060000A0502850A064
:103F40000508080600FF40C0405070307810050892
:103F5000080600FF40C040506808103805080806F1
:103F600000FFC0204030F030781004070706010041
:103F70002000206080906005070706000040202098
:103F800050708888050707060000102020507088B0
:103F90008805070706000020502050708888050714
:103FA0000706000028502050708888050707060083
:103FB0000050002050708888050707060000205038
:103FC000205070888805060606000078A0F0A0A0A2
:103FD000B80408080601FE609080809060204004CC
:103FE00007070601004020F080E080F00407070684
:103FF00001002040F080E080F00407070601002067
:1040000050F080E080F00407070601005000F080C7
:10401000E080F00307070601008040E0404040E0F8
:104020000307070601002040E0404040E003070787
:1040300006010040A0E0404040E003070706010001
:10404000A000E0404040E00506060600007048E899
:1040500048487004070706010050A090D0B0909027
:104060000407070601004020609090906004070755
:104070000601002040609090906004070706010050
:104080002050609090906004070706010050A060E7
:104090009090906004070706010050006090909097
:1040A00060050505060000885020508804080806B1
:1040B00001FF1070B0B0D0D0E08004070706010007
:1040C00040209090909060040707060100204090E7
:1040D0009090906004070706010020509090909007
:1040E000600407070601005000909090906005075B
:1040F0000706000010208850202020040606060134
:104100000080E09090E0800406060601006090A028
:10411000A090A00407070601004020007090907056
:104120000407070601002040007090907004070704
:1041300006010020500070909070040707060100EF
:1041400050A00070909070040606060100500070A8
:104150009090700407070601002050207090907026
:1041600005040406000070A8B0780406060601FEE7
:104170007080807020400407070601004020006026
:10418000B0C07004070706010020400060B0C07096
:1041900004070706010020500060B0C07004060646
:1041A000060100500060B0C07003070706010080E0
:1041B0004000C04040E0030707060100204000C067
:1041C0004040E003070706010040A000C04040E077
:1041D000030606060100A000C04040E004070706F1
:1041E00001003060107090906004070706010050D5
:1041F000A000E090909004070706010040200060B6
:1042000090906004070706010020400060909060D5
:104210000407070601002050006090906004070723
:1042200006010050A00060909060040606060100A0
:104230005000609090600505050600002000F80021
:104240002004040406010070B0D0E0040707060152
:104250000040200090909070040707060100204065
:104260000090909070040707060100205000909085
:1042700090700406060601005000909090700409AA
:10428000090601FE2040009090907090600408089C
:104290000601FE8080E09090E0808004080806011E
:1042A000FE50009090907090604D3530320A4D3540
:1042B0003030004C6F61642073657474696E67738D
:1042C00000526573746F7265206661696C73616614
:1042D000650053746F72652073657474696E6773DB
:1042E00000416476616E6365642053657474696E21
:1042F0006773004D61696E005072696E746572205B
:104300005374617473004669726D776172652056EB
:10431000657273696F6E004D61696E000A003B2023
:10432000454550524F4D20496E6465783A200055FE
:1043300070646174696E67207A6F66667365742055
:10434000696E20454550524F4D3A20000E000E0038
:104350000E000E000E000E000E000E007FC03F800B
:104360001F000E00040004000E001F003F807FC0ED
:104370000E000E000E000E000E000E000E000E00CD
:1043800003F8000FFE001E0F00380700380380708E
:104390000380700FE07007C0700380700100700030
:1043A000003800003807001E0F000FFE0003F80061
:1043B00000FE0003FF800783C00E01C00E00E01C5A
:1043C00000E07F00E03E00E01C00E00800E00000AC
:1043D000E00001C00E01C00F078007FF0001FC00D4
:1043E000FFFFFF7F80FFC0FFC0FFC07F807F80FF97
:1043F000C0FFC0FFC03F001E000C0050726F62651E
:10440000205A204F66667365740050726F62652093
:104410005A204F666673657400466C6F7700466C71
:104420006F770046616E2073706565640046616E4B
:104430002073706565640042656400426564004EE7
:104440006F7A7A6C65004E6F7A7A6C65005370658E
:104450006564005370656564004D61696E004D6F61
:1044600076652058004D6F76652059004D6F766552
:10447000205A00457874727564657220004D6F761D
:104480006520302E316D6D004D6F766520316D6D7C
:10449000004D6F76652031306D6D004D6F76652073
:1044A0006178697300457874727564657220004D97
:1044B0006F7665205A004D6F76652059004D6F76F6
:1044C000652058007C3C3E5E2B3D3F2F5B5D3B2CC6
:1044D0002A225C006F70656E206661696C65642CD1
:1044E0002046696C653A200043616E6E6F74206FE0
:1044F00070656E2073756264697220006563686F11
:104500003A00453120544845524D414C2052554EB9
:10451000415741590042454420544845524D414C71
:104520002052554E4157415900546865726D616C77
:104530002052756E61776179000000220025002805
:10454000002B002E0031003400020100000501089C
:10455000010B0100002100240027002A002D00305B
:1045600000330001010000040107010A01050505EF
:1045700005070508080808020202020A0A080804DA
:104580000404040101010101010101030303030308
:10459000030303040707070C0C0C0C0C0C0C0C0297
:1045A00002020206060606060606060B0B0B0B0B9E
:1045B0000B0B0B0102102020080810204010204097
:1045C00080020102010804020101020408102040D7
:1045D00080804020100804020180040201804020F5
:1045E000100804020108040201010204081020401E
:1045F000800102040810204080486F6D65202573FB
:10460000257325732066697273740020666972735E
:10461000740A005A0059005800486F6D6520004D1B
:104620003234004D323320257300534420636172CD
:1046300064206F6B0A006F70656E526F6F74206636
:1046400061696C65640A00766F6C756D652E696EC4
:104650006974206661696C65640A00534420696E60
:104660006974206661696C0A0057726974696E67C3
:1046700020746F2066696C653A20006F70656E204B
:104680006661696C65642C2046696C653A20006F30
:1046900070656E206661696C65642C2046696C6586
:1046A0003A200046696C652073656C6563746564C7
:1046B0000A002053697A653A200046696C65206FCC
:1046C00070656E65643A20002066696C653A20006A
:1046D000646F696E67006672657368004E6F77205D
:1046E00000454E4420535542524F5554494E450AB9
:1046F000002220706F73002220706172656E743A20
:104700002200535542524F5554494E452043414C87
:104710004C207461726765743A22004B494C4C45D9
:10472000442E2000747279696E6720746F20636173
:104730006C6C207375622D67636F64652066696CAD
:104740006573207769746820746F6F206D616E796E
:10475000206C6576656C732E204D4158206C657613
:10476000656C2069733A004572726F723A004D6948
:1047700063726F737465707320756E617661696CB6
:1047800061626C650A0045303A20005A3A200059AF
:104790003A2000583A20004D53312C4D53322050CE
:1047A000696E730A004572726F722077726974695C
:1047B0006E6720746F20454550524F4D210A0045C9
:1047C0004550524F4D206461746173697A6520656C
:1047D00072726F722E0A00290A0020627974657362
:1047E0003B20637263200053657474696E677320A5
:1047F00053746F726564202800290A00206279745E
:1048000065733B2063726320002073746F7265646C
:104810002073657474696E6773207265747269655C
:10482000766564202800202863616C63756C617470
:10483000656429210A0020213D2000454550524F42
:104840004D20435243206D69736D61746368202D60
:10485000202873746F7265642920002053697A657B
:104860003A2000496E6465783A2000204D61726CF0
:10487000696E3D563535290A0028454550524F4D41
:104880003D00454550524F4D2076657273696F6EFD
:10489000206D69736D61746368200045787472756A
:1048A00064657220004D6F7665205A004D6F766505
:1048B0002059004D6F76652058004D6F76656D6507
:1048C0006E7400436F6F6C646F776E0046616E208C
:1048D00073706565640046616E2073706565640081
:1048E00042656400426564004E6F7A7A6C65004EE2
:1048F0006F7A7A6C65004D61696E0056547261760C
:10490000206D696E005654726176206D696E005696
:1049100054726176206D696E00566D696E00566D39
:10492000696E00566D696E00566D617820450056BF
:104930006D6178204500566D6178204500566D61A7
:1049400078205A00566D6178205A00566D617820A3
:104950005A00566D6178205900566D6178205900D3
:10496000566D6178205900566D6178205800566D5B
:104970006178205800566D61782058004D6F746939
:104980006F6E00416D6178204500416D6178204572
:1049900000416D6178205A00416D6178205A0041D4
:1049A0006D6178205900416D6178205900416D6139
:1049B00078205800416D6178205800412D74726153
:1049C00076656C00412D74726176656C00412D72C4
:1049D00065747261637400412D72657472616374F1
:1049E00000416363656C00416363656C004D6F74E7
:1049F000696F6E00506C65617365207265736574D4
:104A0000005052494E5445522048414C54454400B0
:104A10005072696E7465722068616C7465642E20D2
:104A20006B696C6C28292063616C6C6564210A00D9
:104A3000656E7175657565696E67202200000040BE
:104A4000C000003E4300001F430000F0410000F0A2
:104A50004100000041000000005761726E696E67FE
:104A60003A20486F6D696E672042756D7020446909
:104A70007669736F72203C20310A00020204000044
:104A8000A0400000A04000000040000025430000BE
:104A9000454300002143FF010120643A0020693AA8
:104AA0000020703A00496E736572742066696C610B
:104AB0006D656E7420616E64207072657373206220
:104AC0007574746F6E20286F72204D313038290A4A
:104AD000002F2F616374696F6E3A726573756D652F
:104AE0000A004D3630303A20546F6F20636F6C648B
:104AF00000486F74656E6420746F6F20636F6C6420
:104B00000A002F2F616374696F6E3A706175736567
:104B10000A00436C69636B20746F20726573756D56
:104B2000652E2E2E004E6F206D6F76652E00286E3E
:104B30006F2066696C6529005344207072696E7439
:104B4000696E67206279746520004E6F742053444B
:104B5000207072696E74696E670A004375727265BF
:104B60006E742066696C653A200046696C65206445
:104B7000656C657465643A0044656C6574696F6E54
:104B8000206661696C65642C2046696C653A20007A
:104B9000000125301D0C1E2829FF24311C0B18454F
:104BA00027FF232F1B0A174443FFFFFFFF040806BC
:104BB000FF06222B1A4142FF043803FF3650726F62
:104BC0007465637465642050696E0A0046696C619F
:104BD0006D656E7420757365643A2000537461745A
:104BE000733A20002C204C6F6E67657374206A6FD7
:104BF000623A2000546F74616C2074696D653A20CC
:104C00000053746174733A20002C204661696C650E
:104C1000643A20002C2046696E69736865643A2006
:104C2000005072696E74733A200053746174733A61
:104C300020006F6B000045787472756465642074A1
:104C40006F74616C3A2000256C642E25696D00003C
:104C50004C6F6E67657374206A6F622074696D654E
:104C60003A200000546F74616C207072696E742079
:104C700074696D653A2000436F6D706C657465648E
:104C80003A20005072696E7420436F756E743A203A
:104C9000004D36303020423020542564004D3730EE
:104CA0003120542564004D373032203B2564004DBF
:104CB00037303220542564004368616E6765206692
:104CC000696C616D656E7400507265686561742011
:104CD000437573746F6D005072656865617420432D
:104CE0007573746F6D005072656865617420414220
:104CF00053005072656865617420504C41004D61ED
:104D0000696E005052494E5420504155534544005D
:104D1000554E4C4F41442046494C414D454E540060
:104D20004C4F41442046494C414D454E540050752E
:104D3000726765206D6F726500456E642066696CF0
:104D4000616D656E74206368616E67650000202088
:104D50004E6F7A7A6C653A20006368616E67650011
:104D60006F66207468652066696C616D656E74009D
:104D70005761697420666F722073746172740020C9
:104D8000204E6F7A7A6C653A2000200066696C616B
:104D90006D656E7420756E6C6F6164005761697427
:104DA00020666F720020204E6F7A7A6C653A200080
:104DB0002000506C6561736520776169742E2E2E1A
:104DC0000048656174696E67206E6F7A7A6C650061
:104DD00020204E6F7A7A6C653A2000200068656169
:104DE00074206E6F7A7A6C652E0050726573732032
:104DF000627574746F6E20746F0020204E6F7A7A23
:104E00006C653A2000746F20636F6E74696E75650F
:104E10002E2E2E00616E6420707265737320627591
:104E200074746F6E00496E736572742066696C618C
:104E30006D656E740020204E6F7A7A6C653A2000A2
:104E4000200066696C616D656E74206C6F61640032
:104E50005761697420666F720056652D6A65726BC2
:104E60000056652D6A65726B0056652D6A65726B1A
:104E700000567A2D6A65726B00567A2D6A65726BE0
:104E80000056792D6A65726B0056792D6A65726BD2
:104E90000056792D6A65726B0056782D6A65726BC3
:104EA0000056782D6A65726B0056782D6A65726BB4
:104EB000004D6F74696F6E004573746570732F6D6C
:104EC0006D004573746570732F6D6D005A73746552
:104ED00070732F6D6D005A73746570732F6D6D0054
:104EE0005973746570732F6D6D00597374657073A9
:104EF0002F6D6D005873746570732F6D6D0058734E
:104F0000746570732F6D6D004D6F74696F6E004F17
:104F10006666004F6E2000456E6473746F7020618A
:104F2000626F72740053746570732F6D6D004A6503
:104F3000726B00416363656C65726174696F6E00CA
:104F400056656C6F636974790050726F6265205AA0
:104F5000204F666673657400416476616E636564B4
:104F60002053657474696E67730043616E6E6F746D
:104F700020656E746572207375626469723A2000F0
:104F8000022E2E004D61696E0048617264636F6489
:104F900065642044656661756C742053657474693A
:104FA0006E6773204C6F616465640A0028230000FB
:104FB0002823000064000000E8030000000096437E
:104FC0000000964300000041000020420000C9425A
:104FD0000000C9420000C8440000D2433A0A002041
:104FE000286D6D290020204D3630332000205500DB
:104FF0004C0046696C616D656E74206C6F61642F46
:10500000756E6C6F6164206C656E677468733A0AC4
:1050100000204500205A0020204D3930372058000C
:1050200053746570706572206D6F746F7220637554
:105030007272656E74733A0A0020204D3930302048
:105040004B004C696E65617220416476616E6365E8
:105050003A0A0020204D383531205A005A2D50721E
:105060006F6265204F6666736574002044002049B6
:105070000020204D333034205000204400204900CF
:1050800020204D3330312050005049442073657446
:1050900074696E67733A0A00204600204200204877
:1050A0000020204D3134352053004D617465726904
:1050B000616C2068656174757020706172616D65E6
:1050C000746572733A0A0020204D34323020530048
:1050D0004175746F20426564204C6576656C696E1D
:1050E000673A0A00205A0020590020204D323036FD
:1050F000205800486F6D65206F66667365743A0AC4
:1051000000204500205A002059002058002054005B
:1051100020530020204D32303520420020453C6D88
:1051200061785F655F6A65726B3E0020583C6D6117
:10513000785F785F6A65726B3E20593C6D61785F7D
:10514000795F6A65726B3E205A3C6D61785F7A5F69
:105150006A65726B3E00416476616E6365643A20F5
:10516000423C6D696E5F7365676D656E745F7469EF
:105170006D655F75733E20533C6D696E5F66656556
:1051800064726174653E20543C6D696E5F74726137
:1051900076656C5F66656564726174653E00205477
:1051A0000020520020204D323034205000416363F3
:1051B000656C65726174696F6E2028756E697473B1
:1051C0002F7332293A20503C7072696E745F6163AC
:1051D00063656C3E20523C726574726163745F61FA
:1051E0006363656C3E20543C74726176656C5F61EC
:1051F0006363656C3E0A00204500205A0020590078
:1052000020204D3230312058004D6178696D756D28
:1052100020416363656C65726174696F6E202875E7
:105220006E6974732F7332293A0A00204500205AA0
:105230000020590020204D3230332058004D617835
:10524000696D756D2066656564726174657320288B
:10525000756E6974732F73293A0A00204500205A2D
:105260000020590020204D393220580053746570B9
:10527000732070657220756E69743A0A0020204DA3
:105280003230302044300A0020204D32303020446B
:10529000002044697361626C65640A0046696C6150
:1052A0006D656E742073657474696E67733A00205F
:1052B000204D3134392043203B20556E69747320D2
:1052C000696E2043656C736975730A00202047324C
:1052D00031202020203B00526573656E643A200027
:1052E0002042002050006F6B00627573793A207085
:1052F000617573656420666F7220696E7075740ADB
:1053000000627573793A2070617573656420666F09
:105310007220757365720A00627573793A20707233
:105320006F63657373696E670A004B494C4C454463
:105330002E20004B494C4C206361757365642062DC
:105340007920746F6F206D75636820696E61637476
:105350006976652074696D65202D206375727265AC
:105360006E7420636F6D6D616E643A20004C756CD5
:105370007A426F74204D696E692072656164792E7E
:10538000005072696E74696E672E2E2E005072691D
:105390006E7420706175736564004D313235004D57
:1053A0003234005072696E742061626F7274656489
:1053B000005072696E742066726F6D205344005302
:1053C000746F70207072696E7400526573756D65CC
:1053D000207072696E74004E6F20534420636172B6
:1053E00064005061757365207072696E740041626B
:1053F0006F7574205072696E746572004368616ED7
:1054000067652066696C616D656E74004368616EE6
:1054100067652066696C616D656E74004D3630306D
:1054200020423000436F6E66696775726174696F00
:105430006E0054656D7065726174757265004D6FB4
:1054400076656D656E740054756E6500496E666FA5
:105450002073637265656E004D6F766520617869B3
:10546000730044697361626C652073746570706564
:105470007273004D3834004175746F20686F6D652C
:1054800000473238004D61696E00556E6B6E6F7764
:105490006E20636F6D6D616E643A202200486F74F8
:1054A000656E6420746F6F20636F6C640A00000087
:1054B0000A0B02090C0D0E0807030401000000008E
:1054C00000000000000000000000000000000000DC
:1054D0000000000000000000000012111000000099
:1054E00000000000000000000000000000000000BC
:1054F0000000000050726F62696E67206661696C1F
:1055000065640A0050726F62696E67206661696C3B
:10551000656400205A3A200020593A200042656410
:1055200020583A20000038D30A0111241FBECFEFC3
:10553000D1E2DEBFCDBF00E00CBF13E0A0E0B2E0DF
:10554000E2EDFFE602E00BBF02C007900D92AC3A1D
:10555000B107D9F726E1ACEAB3E001C01D92A33749
:10556000B207E1F71AE2C4E9DAE200E006C02197E7
:105570000109802FFE010F945437C339D10780E011
:105580000807A9F70E9450950D94D8370C94000095
:105590002F923F924F925F926F927F928F929F9243
:1055A000AF92BF92CF92DF92EF92FF920F931F9331
:1055B000CF93DF93CDB7DEB7C15AD1090FB6F894B8
:1055C000DEBF0FBECDBFC356DF4F8883CD59D0405D
:1055D00021E02093BB148091A5148D3411F40C9418
:1055E0002B33843511F40C947344873411F00C94EC
:1055F000B7448091A3149091A4148A31910509F4C1
:105600006AC6B4F4843091053CF4823091059CF56F
:1056100097FF2AC00C9427338430910509F41CC6E7
:105620000C9711F00C9427330E94EE6A0C94B94445
:105630008E31910509F4CCC63CF48C31910509F406
:1056400080C60CF44EC682C68B35910509F493C70B
:105650008C35910509F493C78A35910509F0F7C790
:105660001092B2030C94B94480910A0281110C94F7
:10567000C6440C94B94420910A02222311F40C94DC
:10568000B94411E0029709F010E00E942E6C82E507
:105690000E94E26A882309F45CC10E94646A6B017B
:1056A0007C018091231290912412A0912512B09137
:1056B00026128CAF9DAFAEAFBFAF209127123091B5
:1056C00028124091291250912A1224962CAF3DAFF6
:1056D0004EAF5FAF24978091BC149091BD14A09100
:1056E000BE14B091BF1428968CAF9DAFAEAFBFAFC4
:1056F00028972091C0143091C1144091C214509148
:10570000C3142C962CAF3DAF4EAF5FAF2C9720E06B
:1057100030E0A901C701B6010F94FB2F882309F4DB
:1057200081C52CAD3DAD4EAD5FAD28966CAD7DAD68
:105730008EAD9FAD28970F94FB2F811111C0249639
:105740002CAD3DAD4EAD5FAD24972C966CAD7DADCF
:105750008EAD9FAD2C970F94FB2F882309F462C563
:1057600020E030E0A901C701B6010F94FB2F881F8C
:105770008827881F181307C0412C512C00E8602E81
:105780000FE3702E06C0412C512CB0E86B2EBFEBFE
:105790007B2E2CAD3DAD4EAD5FAD28966CAD7DAD95
:1057A0008EAD9FAD28970F94643464966CAF7DAF37
:1057B0008EAF9FAF649724962CAD3DAD4EAD5FADDF
:1057C00024972C966CAD7DAD8EAD9FAD2C970F942C
:1057D000643468966CAF7DAF8EAF9FAF6897649668
:1057E0002CAD3DAD4EAD5FAD6497CA01B9010F94CC
:1057F00060304B015C0168962CAD3DAD4EAD5FADA8
:105800006897CA01B9010F9460309B01AC01C501D2
:10581000B4010F9465340F94D03660966CAF7DAFB1
:105820008EAF9FAF609720E030E040E05FE30F94E1
:1058300060304B015C01A7019601C701B6010F94CE
:1058400060306B017C01A5019401C501B4010F9486
:1058500060309B01AC01C701B6010F9464340F9412
:10586000D0369B01AC01C301B2010F9460302B0113
:105870003C0128962CAD3DAD4EAD5FAD28976CAD8B
:105880007DAD8EAD9FAD0F94653420E030E040E0FB
:105890005FE30F9460306B017C0168966CAD7DAD69
:1058A0008EAD9FAD6897905860962CAD3DAD4EADD6
:1058B0005FAD60970F9441359B01AC01C301B2010C
:1058C0000F9460309B01AC01C701B6010F946534A1
:1058D0002CAD3DAD4EAD5FAD0F9464346B017C01DA
:1058E0002C962CAD3DAD4EAD5FAD2C9724966CAD96
:1058F0007DAD8EAD9FAD24970F94653420E030E0F0
:1059000040E05FE30F9460304B015C0160962CAD8A
:105910003DAD4EAD5FAD609764966CAD7DAD8EAD27
:105920009FAD64970F9441359B01AC01C301B20157
:105930000F9460309B01AC01C501B4010F94653434
:1059400024962CAD3DAD4EAD5FAD24970F946434DD
:1059500014C089E40E94E26A882329F00E94646AE4
:105960006B017C0103C0C12CD12C76018AE40E941A
:10597000E26A8823F9F00E94646A28966CAF7DAFD2
:105980008EAF9FAF289720E030E0A901C701B60194
:105990000F94FB2F81111EC020E030E0A901289652
:1059A0006CAD7DAD8EAD9FAD28970F94FB2F81110F
:1059B00011C038C420E030E0A901C701B6010F943E
:1059C000FB2F882309F42EC428961CAE1DAE1EAEF4
:1059D0001FAE2897D701C601B0588CAF9DAFAEAFB0
:1059E000BFAF28962CAD3DAD4EAD5FAD289750585A
:1059F00024962CAF3DAF4EAF5FAF24979C01AD0115
:105A0000BC01CD010F9460304B015C0124962CAD9C
:105A10003DAD4EAD5FAD2497CA01B9010F94603022
:105A20009B01AC01C501B4010F9465340F94D036CD
:105A3000A4966CAF7DAF8EAF9FAFA49780912312D9
:105A400090912412A0912512B09126122C968CAF21
:105A50009DAFAEAFBFAF2C97A7019601BC01CD01A2
:105A60000F94653468966CAF7DAF8EAF9FAF68972B
:105A700020912712309128124091291250912A1218
:105A800060962CAF3DAF4EAF5FAF609728962CADC0
:105A90003DAD4EAD5FAD289760966CAD7DAD8EADE2
:105AA0009FAD60970F946534E0966CAF7DAF8EAF7D
:105AB0009FAFE0978091BC149091BD14A091BE144B
:105AC000B091BF1464968CAF9DAFAEAFBFAF64977B
:105AD00068962CAD3DAD4EAD5FAD6897BC01CD0174
:105AE0000F9464346B017C012091C0143091C11477
:105AF0004091C2145091C3146C962CAF3DAF4EAF81
:105B00005FAF6C97E0962CAD3DAD4EAD5FADE097CD
:105B10006C966CAD7DAD8EAD9FAD6C970F9464347B
:105B20004B015C0180912B1290912C12A0912D12AF
:105B3000B0912E12A0968CAF9DAFAEAFBFAFA09725
:105B40009C01AD016091C4147091C5148091C6147C
:105B50009091C7140F9464342B013C012091C81418
:105B60003091C9144091CA145091CB14A8962CAF0F
:105B70003DAF4EAF5FAFA89780912F12909130123A
:105B8000A0913112B0913212E4968CAF9DAFAEAFBE
:105B9000BFAFE497A70196016CAD7DAD8EAD9FAD13
:105BA0000F946030AC966CAF7DAF8EAF9FAFAC976B
:105BB000A501940124966CAD7DAD8EAD9FAD24976B
:105BC0000F9460309B01AC01AC966CAD7DAD8EAD99
:105BD0009FADAC970F946534AC966CAF7DAF8EAF34
:105BE0009FAFAC97A50194016CAD7DAD8EAD9FAD1F
:105BF0000F9460304B015C01A701960124966CADB7
:105C00007DAD8EAD9FAD24970F9460309B01AC01AC
:105C1000C501B4010F946434AC962CAD3DAD4EADCE
:105C20005FADAC970F94D8346B017C0120E030E07D
:105C3000A9010F94FB2F87FF0AC02BED3FE049EC31
:105C400050E4C701B6010F9465346B017C01112348
:105C500051F02BED3FE049EC50E4C701B6010F9441
:105C600064346B017C0120E030E0A901C701B6017A
:105C70000F94FB2F811128C064962CAD3DAD4EAD25
:105C80005FAD64972C966CAD7DAD8EAD9FAD2C97BE
:105C90000F94FB2F811118C06C962CAD3DAD4EAD0D
:105CA0005FAD6C9760966CAD7DAD8EAD9FAD60972E
:105CB0000F94FB2F811108C0ABEDCA2EAFE0DA2E96
:105CC000A9ECEA2EA0E4FA2EA7019601A4966CADE9
:105CD0007DAD8EAD9FADA4970F9460304B015C01FC
:105CE00020E030E0A901C301B2010F94FB2F88230B
:105CF000C9F0A5019401C501B4010F9460304B01B6
:105D00005C01A3019201C301B2010F9460309B01B9
:105D1000AC01C501B4010F9465340F94D0364B012A
:105D20005C010DC020E030E0A901C501B4010F9471
:105D30008B3687FF04C0B7FAB094B7F8B0942FE65B
:105D400032E143E85AE3C501B4010F94FB2F87FF0A
:105D500002C00C94B944C501B4010F94DA350F9414
:105D6000AE351B01672B19F422242394312CB10189
:105D700080E090E00F94FF2F4B015C019B01AC0190
:105D8000C701B6010F9441352C966CAF7DAF8EAF35
:105D90009FAF2C97A5019401C301B2010F94413527
:105DA000A4966CAF7DAF8EAF9FAFA497E4962CAD59
:105DB0003DAD4EAD5FADE497A8966CAD7DAD8EADBB
:105DC0009FADA8970F946434A50194010F944135B9
:105DD000A8966CAF7DAF8EAF9FAFA8972C962CADD9
:105DE0003DAD4EAD5FAD2C97CA01B9010F94603047
:105DF00020E030E040E05FE30F9460309B01AC01B5
:105E000060E070E080E89FE30F9464346C966CAFC0
:105E10007DAF8EAF9FAF6C97A0962CAD3DAD4EADD4
:105E20005FADA09729873A874B875C87E4968CAD56
:105E30009DADAEADBFADE4978D879E87AF87B88B24
:105E40006091000270910102072E000C880B990BE3
:105E50000F940130209170023091710240917202D2
:105E6000509173020F9460302AE037ED43E25CE317
:105E70000F9460306CAB7DAB8EAB9FAB0E948EA35A
:105E80009B01AC0128533F4F4F4F5F4FA0962CAF63
:105E90003DAF4EAF5FAFA0974CAC5DAC6EAC7FAC8E
:105EA00041E050E062965FAF4EAF629759E12D96A8
:105EB0005FAF2D9762962EAD3FAD629722153305E9
:105EC00009F455C10E94A5770E948EA3DC01CB0185
:105ED000A0962CAD3DAD4EAD5FADA097821B930B50
:105EE000A40BB50BB7FD11C00E948EA39B01AC01A2
:105EF00028533F4F4F4F5F4FA0962CAF3DAF4EAF53
:105F00005FAFA09780E00F94BB1E2D963FAD2D97FD
:105F100031502D963FAF2D97332309F44BC06C962B
:105F20002CAD3DAD4EAD5FAD6C9724966CAD7DADA7
:105F30008EAD9FAD24970F9460306B017C012C9641
:105F40002CAD3DAD4EAD5FAD2C97B201C3010F94AA
:105F50006030A70196010F9465347B018C016C962B
:105F60002CAD3DAD4EAD5FAD6C97B201C3010F944A
:105F700060304B015C012C962CAD3DAD4EAD5FAD5C
:105F80002C9724966CAD7DAD8EAD9FAD24970F946C
:105F900060309B01AC01C501B4010F9464342B0146
:105FA0003C01C701D80124968CAF9DAFAEAFBFAF07
:105FB00024975DC062964EAD5FAD6297BA0180E0F6
:105FC00090E00F94FF2F2C962CAD3DAD4EAD5FAD04
:105FD0002C970F9460304B015C010F943E356B01A0
:105FE0007C01C501B4010F94C6364B015C01A701C9
:105FF00096016CAD7DAD8EAD9FAD0F9460302B01E1
:106000003C01A501940128966CAD7DAD8EAD9FAD90
:1060100028970F9460309B01AC01C301B2010F942B
:1060200065342B013C01A50194016CAD7DAD8EADB5
:106030009FAD0F9460304B015C01A701960128963B
:106040006CAD7DAD8EAD9FAD28970F9460309B01F8
:10605000AC01C501B4010F94643424966CAF7DAFDC
:106060008EAF9FAF249759E12D965FAF2D97920188
:10607000A30168966CAD7DAD8EAD9FAD68970F9412
:10608000653469837A838B839C8324962CAD3DADE4
:106090004EAD5FAD2497E0966CAD7DAD8EAD9FADFE
:1060A000E0970F9465346D837E838F839887A496E1
:1060B0002CAD3DAD4EAD5FADA49769857A858B85DE
:1060C0009C850F94653469877A878B879C87A8960F
:1060D0002CAD3DAD4EAD5FADA8976D857E858F85AE
:1060E00098890F9465346D877E878F87988BCE0152
:1060F00001960F94CE21E09058161CA61DA61EA650
:106100001FA689819A81AB81BC8188A399A3AAA388
:10611000BBA38D819E81AF81B8858CA39DA3AEA3C7
:10612000BFA389859A85AB85BC8588A799A7AAA7AF
:10613000BBA7AE01485D5F4FBE016C5D7F4FCE01D6
:1061400080960E94FD6FCE018C966C018E010C5CD6
:106150001F4F9E01235F3F4FAE01485D5F4FBE0161
:106160006C5D7F4F0C970E947A50811151C0E09076
:10617000581618AA19AA1AAA1BAA8091BC149091A1
:10618000BD14A091BE14B091BF1488A399A3AAA373
:10619000BBA38091C0149091C114A091C214B0917E
:1061A000C3148CA39DA3AEA3BFA38091C4149091EC
:1061B000C514A091C614B091C71488A799A7AAA71F
:1061C000BBA7AE01485D5F4FBE016C5D7F4FCE0146
:1061D00080960E94FD6FDE01D0966D018E010C5CF1
:1061E0001F4F28EC34E1AE01485D5F4FBE016C5D8E
:1061F0007F4FCE0180960E947A5080E1ECEBF4E173
:10620000A3E2B2E101900D928A95E1F70C94B944B2
:106210006296EEADFFAD629731966296FFAFEEAF3C
:10622000629748CEE7E6F7E484918F010F5F1F4F36
:10623000882321F00F943F26F801F6CFEDEBF2E032
:1062400084918F010F5F1F4F882311F40C94B94480
:106250000F943F26F801F4CF80E50E94E26A88237C
:1062600029F00E94246A6B017C0103C0C12CD12C4F
:10627000760183E50E94E26A882361F00E94646AE5
:1062800020E030E04AE754E40F9460300F94AE35DC
:106290006B017C010E9427628091690E811105C00B
:1062A00060E083ED92E00E94E1BB0E948EA3C60EE7
:1062B000D71EE81EF91E0E948EA3DC01CB018C19AB
:1062C0009D09AE09BF09B7FD02C00C94B94480E036
:1062D0000F94BB1EF0CF20930A02109271120C94FF
:1062E000B9440E9443E281110C94B94480E090E0EB
:1062F000A0E2B1E489839A83AB83BC8380E090E021
:10630000A4E3B3E48D839E83AF83B88780E090E0FD
:10631000A0EAB1E489879A87AB87BC8780E50E94B1
:10632000E26A882319F00E94346A01C060E068A321
:10633000BE016F5F7F4FCE0180960E9474D20C9495
:10634000B94480E00E94ABB30C94B94480E00E9451
:10635000E26913E001E010925D1610925E16109251
:106360005F16109260160093140C24982C9A149ABD
:106370000E94E4A31092140C249A2C9814988091F3
:106380002215882351F080912215882369F08AE52F
:1063900093E00F9475050C94B9448AE893E00F9448
:1063A00075051150C1F6EFCFE1E7F3E084918F015D
:1063B0000F5F1F4F882321F00F943F26F801F6CF7F
:1063C0008BEE92E00F9475058CED92E00F94DA0558
:1063D000C0902312D0902412E0902512F090261243
:1063E00088E50E94E26A811108C020E030E0A9013E
:1063F000C701B6010F94653402C00E94646A68A3A5
:1064000079A38AA39BA3C0902712D0902812E09072
:106410002912F0902A1289E50E94E26A811108C0CF
:1064200020E030E0A901C701B6010F94653402C035
:106430000E94646A9B01AC0169837A838B839C838D
:1064400068A179A18AA19BA10F94FC04882311F46F
:106450000C94B94480E00E94E2690E94586585E48A
:106460000E94E26A882321F00E94556A182F04C016
:1064700085E40E949B6A11E086E50E94E26A882317
:1064800021F00E94346A262F01C021E0412FBE0175
:106490006F5F7F4FCE0180960F9457286B017C0170
:1064A0009B01AC010F94113781115FC088A099A0A6
:1064B000AAA0BBA020E030E0A901C501B4010F945F
:1064C000FB2F87FD05C027E137EB41E558E304C00A
:1064D00027E137EB41E558EBC501B4010F94653472
:1064E000AB01BC0186E194E00E9445FE89809A8060
:1064F000AB80BC8020E030E0A901C501B4010F945D
:10650000FB2F87FD05C027E137EB41E558E304C0C9
:1065100027E137EB41E558EBC501B4010F94653431
:10652000AB01BC0181E194E00E9445FE20E030E037
:10653000A901C701B6010F94FB2F87FD05C027E114
:1065400037EB41E558E304C027E137EB41E558EB71
:10655000C701B6010F946534AB01BC018CE094E037
:106560000E9445FE8AE00F943F260E943F650E94EC
:10657000187C0C94B9442093B2030C94B94443E1C1
:1065800053E05DAF4CAF73E2E72E72E1F72EE1E628
:10659000CE2EE6E1DE2E312C00E010E0ACADBDAD3C
:1065A0008D91BDAFACAF0E94E26A8823B9F10E9421
:1065B000646A2B013C01133049F0F60120813181DE
:1065C000428153810F9464342B013C01D7012D91FA
:1065D0003D914D915C91C301B2010F9464344B0124
:1065E0005C012DEB37E346E855EB0F948B3687FDC6
:1065F0000AC02DEB37E346E855E3C501B4010F941B
:10660000FB2F18165CF4133011F001E002C03324A4
:106610003394F70140825182628273821F5FF4E0FB
:10662000EF0EF11C24E0C20ED11C143009F0B6CFDD
:10663000002319F00E94DB6806C0332021F08FE2AE
:1066400092E10E94E4E20E94187C0C94B9440F94F9
:106650005A2B0C94B9448091A3149091A4148937B7
:10666000910509F414C60CF00DC18D34910509F49F
:10667000C6C20CF07CC08A31910509F47AC20CF0D4
:1066800040C08431910509F413C294F4813191051D
:1066900009F40AC244F4029710F00C9470440F9469
:1066A000430B0C94B944429709F48DC30C94704485
:1066B0008731910509F443C274F48531910509F4D9
:1066C0003AC2469711F00C94704410922D0F10921C
:1066D0002E0F0C94B9448831910509F446C24997AC
:1066E00011F00C94704410922D0F0E94A1938EE330
:1066F00094E090935912809358120E940A660C9469
:10670000B9448F31910509F448C29CF48C3191054C
:1067100009F437C20CF431C28D31910511F40C9497
:10672000B9444E9711F00C9470440F949A080C944D
:10673000B9448934910509F45AC264F48032910550
:1067400009F423C28A9711F00C9470440F94E8075F
:106750000C94B9448B34910509F44DC28C349105E5
:1067600011F00C9470440E94A1930C94B9448B36A0
:10677000910509F471C20CF046C08435910509F405
:1067800022C3E4F48135910509F404C34CF48E343A
:10679000910511F00C9470440F94BD060C94B9440B
:1067A0008235910509F40BC38335910511F00C94E2
:1067B000704481E08093B1030C94B944883691050C
:1067C00009F421C29CF48535910509F431C38C3557
:1067D000910511F00C94704443E1C42E43E0D42E93
:1067E00057E4E52E52E1F52E10E03DC389369105C0
:1067F00009F424C28A36910511F00C9470440F9468
:106800003B060C94B9448237910509F4ADC3DCF41E
:106810008E36910509F4FBC14CF48D36910511F0CB
:106820000C9470440E94C9810C94B9448F36910530
:1068300009F400C28137910511F00C9470440E9454
:10684000507F0C94B9448637910509F402C454F47E
:106850008337910509F48EC38537910509F4E8C3A0
:106860000C9470448737910509F444C48837910526
:1068700011F00C94704481E08093120C8093110C01
:106880000C94B9448E3531E0930711F40C94C93F50
:106890000CF07CC08E3C910509F40FC5E4F58E3BED
:1068A000910509F4D5C1C4F48C38910509F4CCC123
:1068B00034F48D37910509F4E1C10C9470448139A9
:1068C000910509F4EAC48B39910511F00C947044D8
:1068D0000F9457060C94B9448B3C910509F4E5C418
:1068E0006CF4883C910509F4DCC4893C910511F0F5
:1068F0000C9470440E94667B0C94B9448C3C9105C6
:1069000009F4D7C48D3C910511F00C9470440E9499
:10691000637A0C94B944823251E0950709F49CC51E
:10692000C4F48C3D910509F4D0C44CF4833D910529
:1069300011F00C9470440E9485790C94B9448D3DFB
:10694000910509F4D1C4823E910509F43EC50C9429
:1069500070448E32B1E09B0709F4DDC55CF48C32E3
:10696000F1E09F0709F486C58D32914009F4ACC56A
:106970000C9470448F3231E0930709F423C68033BE
:10698000914011F40C944C3F0C947044863F51E0BC
:10699000950711F40C94E8400CF049C08239B1E03D
:1069A0009B0711F40C945E4004F58336F1E09F07D9
:1069B00011F40C9442403CF48F35914011F40C9446
:1069C000FE3F0C947044803941E0940711F40C941C
:1069D0005B408139914011F00C94704481E00E9439
:1069E000F9640E94187C0C94B9448C3AA1E09A078F
:1069F00009F467C46CF4843AE1E09E0711F40C9446
:106A00006440893A914011F40C9467400C947044AE
:106A1000843F21E0920711F40C94E540853F9140BA
:106A200011F00C9470440F94AE1E0C94B9448B3545
:106A300042E0940711F40C94DC42B4F4883FA1E0E6
:106A40009A0711F40C94F74014F40C94EB408C3139
:106A5000E2E09E0711F40C94FA408835924011F45C
:106A60000C9405410C9470448B3823E0920711F488
:106A70000C9422446CF4833543E0940711F40C9495
:106A800065438438934011F40C94CB430C947044C8
:106A9000803AA3E09A0709F47CC0873E934011F442
:106AA0000C945B440C9470440F94390B0C94B944CF
:106AB000EDE2F4E084918F010F5F1F4F882321F0F6
:106AC0000F943F26F801F6CF1092D11140E050E02C
:106AD000BA0184E89FE00E943FCB8BE1E4E8FFE04D
:106AE000DE01159601900D928A95E1F78091820F53
:106AF0009091830F9C838B838AE993E09A838983A7
:106B000040E050E0BE016F5F7F4F80E090E00E9468
:106B1000C0D7CE0101960F946D05EEE1F4E08491AB
:106B20008F010F5F1F4F882311F40C94B9440F9409
:106B30003F26F801F4CF0E94FADD0C94B944E091AD
:106B4000A114F091A2148081882329F0803209F4E5
:106B500010823196F8CF40E061E08091A1149091CD
:106B6000A2140E940CDC0C94B9440F94F4090C9408
:106B7000B9440F94DA090C94B9440F9452090C9457
:106B8000B9440F944A090C94B9440F9459080C94D1
:106B9000B9440F944E080C94B9440E946D9368A3B5
:106BA00079A38AA39BA3BE016F5F7F4FCE0180961E
:106BB0000E94909460E0CE0101960E941BBCECEF15
:106BC000F4E484918F010F5F1F4F882321F00F940D
:106BD0003F26F801F6CFBE016F5F7F4F83E494E05C
:106BE0000E94A2FE8AE00F943F260C94B9440F94B1
:106BF000D6070C94B9440E94B6930C94B9440E94F1
:106C000013940C94B9440F94A2060C94B9448EE4E6
:106C10000E94E26A882311F40C94B9440E94346AF9
:106C200060937F14709380148093811490938214E6
:106C30000C94B9440E947A7F0C94B9440F94850651
:106C40001092BB140C94A0480E94B0810C94B944DB
:106C50000E94F17F0C94B94480E50E94E26A8111A0
:106C600006C010920C0E10920B0E0C94B9440E94A8
:106C7000346A672B11F00C94B944F3CF8CE40E9472
:106C80009B6A882381F00E94646A6B017C0120E08A
:106C900030E0A9010F948B3687FF0AC0F7FAF09411
:106CA000F7F8F09405C0C12CD12CE12C60E4F62E4D
:106CB000F7FAF094F7F8F094CCA6DDA6EEA6FFA6BE
:106CC00080E090E0A0E2B1E489839A83AB83BC8347
:106CD00080E090E0A4E3B3E48D839E83AF83B88724
:106CE00080E090E0A0EAB1E489879A87AB87BC870F
:106CF00088E50E94E26A882379F088E50E94E26ACA
:106D0000882319F00E94646A03C060E070E0CB0140
:106D100069837A838B839C8389E50E94E26A882356
:106D200079F089E50E94E26A882319F00E94646A7A
:106D300003C060E070E0CB016D837E838F83988712
:106D40008AE50E94E26A882379F08AE50E94E26A75
:106D5000882319F00E94646A03C060E070E0CB01F0
:106D600069877A878B879C8718A219A21AA21BA20F
:106D70008091540E81110C94B94420E0AE01405E24
:106D80005F4FBE016F5F7F4FCE018C960F948A00DC
:106D90000C94B9440E94C3740E94386210920C0E85
:106DA00010920B0E68EE73E080E090E00E94C7E95D
:106DB00060E080E594E00E94E1BB0C94B94410923D
:106DC000B1030C94B94483E50E94E26A8823A1F0E0
:106DD0000E94646A20E030E04AE754E40F94603097
:106DE0000F94AE35609365027093660280936702DC
:106DF000909368020C94B94488E50E949B6A8111C3
:106E00000C94DC4589E50E949B6A81110C94DC4559
:106E10008AE50E949B6A81110C94DC4585E40E94FE
:106E20009B6A81110C94DC450E9438620C94B94431
:106E300083E50E949B6A882311F40C94B9440E9454
:106E4000646A20E030E04AE754E40F9460300F9425
:106E5000AE3560938615709387158093881590934F
:106E600089150C94B944F60181916F010E949B6AC7
:106E7000882309F46EC0133009F063C00E94646A6D
:106E80004B015C0120E030E040EA51E40F94FB2F1D
:106E900087FF4EC0A5019401609153127091541266
:106EA00080915512909156120F9441352B013C015F
:106EB0009B01AC0160912F157091301580913115B7
:106EC000909132150F94603060932F1570933015A8
:106ED0008093311590933215A3019201609167154B
:106EE000709168158091691590916A150F946030C2
:106EF00060936715709368158093691590936A1570
:106F00006091ED047091EE048091EF049091F00493
:106F10000F94FF2FA30192010F9460300F94AE35B0
:106F20006093ED047093EE048093EF049093F0046B
:106F30008092531290925412A0925512B09256120F
:106F400008C00E94646AD7016D937D938D939C93D2
:106F500013971F5FB4E0EB0EF11C143009F083CFE0
:106F60000E941E8F0C94B9440E9427620E94187CD4
:106F70000C94B944E5E4F5E084918F010F5F1F4F55
:106F8000882321F00F943F26F801F6CF60E085E3D7
:106F900095E00E94D47B61E08EE295E00E94D47B74
:106FA00061E083E295E00E94D47B61E083E195E0BB
:106FB0000E94D47B60E08AE095E00E94D47B61E08F
:106FC00080E095E00E94D47B61E086EF94E00E942F
:106FD000D47B61E08EEE94E00E94D47B61E080EE91
:106FE00094E00E94D47B61E082ED94E00E94D47B27
:106FF00060E083EC94E00E94D47B60E085EB94E059
:107000000E94D47B60E08FE994E00E94D47B61E031
:107010008EE894E00E94D47B60E089E794E00E94CF
:10702000D47B61E086E694E00E94D47B0C94B94462
:107030008091A1149091A214FC012081222329F0B7
:1070400060E00E941BBC0C94B9440F94AE230C94D6
:10705000B9440091A1141091A21483E0D12C40E016
:107060008150E9F0D8019C91292F2B7F2134C1F761
:1070700011962C912133A1F7913421F0953421F40C
:1070800041E002C0DD24D39498012E5F3F4F890177
:107090002F5F3F4FF80190819032C9F3E1CF442335
:1070A00069F0ECEFF4E484917F012FEFE21AF20A29
:1070B000882321F00F943F26F701F5CFDD2069F0FA
:1070C000EDE3F6E084917F013FEFE31AF30A8823B2
:1070D00021F00F943F26F701F5CFD8018D918D0156
:1070E000882319F00F943F26F8CF8AE00F943F26AB
:1070F0000C94B94481E08093140C24982C9A149A2F
:10710000E1E7F6E084918F010F5F1F4F882321F0A4
:107110000F943F26F801F6CFE9E6F6E084918F015F
:107120000F5F1F4F882321F00F943F26F801F6CF01
:107130001E9B03C00CEF12E002C001E013E0F80157
:1071400081918F01882319F00F943F26F8CF8AE0B0
:107150000F943F26E1E6F6E084918F010F5F1F4F09
:10716000882321F00F943F26F801F6CF379B03C008
:107170000CEF12E002C001E013E0D8018D918D0107
:10718000882319F00F943F26F8CF8AE00F943F260A
:10719000E9E5F6E084918F010F5F1F4F882321F00E
:1071A0000F943F26F801F6CF1D9B03C00CEF12E0B1
:1071B00002C001E013E0F80181918F01882319F0EA
:1071C0000F943F26F8CF8AE00F943F26E1E5F6E0E2
:1071D00084918F010F5F1F4F882321F00F943F266A
:1071E000F801F6CF029B03C00CEF12E002C001E0F1
:1071F00013E0D8018D918D01882319F00F943F265B
:10720000F8CF8AE00F943F26E9E4F6E084918F01FD
:107210000F5F1F4F882321F00F943F26F801F6CF10
:107220001C9B03C00CEF12E002C001E013E0F80168
:1072300081918F01882319F00F943F26F8CF8AE0BF
:107240000F943F26E1E4F6E084918F010F5F1F4F1A
:10725000882321F00F943F26F801F6CF019B03C04D
:107260000CEF12E002C001E013E0D8018D918D0116
:10727000882319F00F943F26F8CF8AE00F943F2619
:107280001092140C249A2C9814980C94B9441092CF
:10729000120C1092110C0C94B9440E94D97E0C94DB
:1072A000B9440E948B7B0C94B9440E94447B0C949B
:1072B000B9440E94CD7A0C94B9440E94B17E0C94DA
:1072C000B9440E94057D0C94B94483E50E94E26AAA
:1072D000882311F40C94B9440E94346A709301021B
:1072E000609300020C94B9448DED90E00E94DC6C38
:1072F00081110C94B94483E50E94E26A8823E1F18C
:107300000091D20410E00E94346A000F111FF801AE
:10731000E05FFD4F718360838091D20490E08C0127
:10732000000F111F000F111FF801EA5FFD4F7F01D1
:10733000880F991FFC01E05FFD4F60817181072E6E
:10734000000C880B990B0F9401302AE037ED43E2D3
:107350005CE30F946030F801E752FB4F20813181EC
:10736000428153810F946030D7016D937D938D934B
:107370009C9313970C94B944ECEFF4E484918F013F
:107380000F5F1F4F882321F00F943F26F801F6CF9F
:1073900085E40F943F268091D204805D0F943F26B0
:1073A000E091D204F0E0EE0FFF1FE05FFD4F60813F
:1073B00071818BE896E00E9489FE85E20F943F265A
:1073C0008AE00F943F260C94B94480E50E949B6AA2
:1073D000882311F40C94B9440E94346A6B017C0137
:1073E00083E50E94E26A882321F00E94346A8B01BF
:1073F00002C00FEF1FEF98012F5F3F4F2330310581
:1074000010F00C94B944D7FE02C00C94B9440E9409
:1074100027620F3FBFEF1B0731F00130110571F4F8
:1074200001E010E00DC08C2D0E949AA131E020E017
:10743000892B09F030E0032F122F02C000E010E08A
:107440008C2D0E949AA18017910711F40C94B944D5
:1074500080E00F94BB1EF4CF8AE50E94E26A81119E
:107460000C94074683E50E94E26A81110C9407465A
:107470000C94B94483E50E94E26A882319F00E94C3
:10748000346A02C064E071E079A368A380E50E94D9
:10749000E26A882339F00E94346A6938E3E17E07A2
:1074A00030F402C068EE73E07A83698304C088E830
:1074B00093E19A838983BE01605E7F4FCE0101967E
:1074C0000E942DDF0C94B94485E40E94E26A811188
:1074D00004C00F947E030C94B9440E94446A88232C
:1074E000C1F3E7E6F7E484918F010F5F1F4F882314
:1074F00021F00F943F26F801F6CFE4EAF6E08491FC
:107500008F010F5F1F4F882311F40C94B9440F941F
:107510003F26F801F4CF83E50E949B6A182F882349
:1075200071F00E94646A0F94A93570936B026093A6
:107530006A0221E0672B09F020E02093591680E5CC
:107540000E949B6A882361F020916A0230916B024D
:10755000232B11F00E94556A809359160C94B9445C
:1075600011110C94B944ECEFF4E484918F010F5F96
:107570001F4F882321F00F943F26F801F6CF80910A
:107580005916811103C06BE073E002C06EEF72E028
:107590008BEC96E00E94A2FE60916A0270916B02F1
:1075A0008AEB96E00E9489FEE6EBF6E084918F017B
:1075B0000F5F1F4F882311F40C94B9440F943F269A
:1075C000F801F4CF85E40E94E26A882321F00E944A
:1075D000346A7B0102C0E12CF12C83E40E94E26A50
:1075E000882331F00E94346AEB966FAFEB9704C0AA
:1075F00045E0EB964FAFEB9785E50E94E26A882362
:1076000019F00E94556A03C085E50E949B6ACA571B
:10761000DF4F8883C658D040F7FC07C0812C912CDF
:1076200066E1A62E63E4B62E06C0812C912C5CE8A0
:10763000A52E52E4B52E83E50E94E26A882321F04C
:107640000E94646A4B015C01E114F10411F4109290
:10765000D204ECAE0E948EA32B013C015CAD57FF1F
:107660000FC00CE310E080E090E0A0E0B1E4C95767
:10767000DF4F88839983AA83BB83C758D0400EC04D
:1076800004E110E020E030E040E551E4C957DF4F6D
:10769000288339834A835B83C758D04061E06E0DED
:1076A000623070F0E7E7F8E084918F010F5F1F4FC1
:1076B000882311F40C94B9440F943F26F801F4CFB9
:1076C000E1EAF8E084917F013FEFE31AF30A8823AF
:1076D00021F00F943F26F701F5CF0E94C3744CAD03
:1076E00047FF04C08FE78093D10408C05CADE52F4D
:1076F000550FFF0BE053FB4F8FE78083C501B401AB
:107700000F94A935072E000C880B990B0F940130AC
:1077100029966FAF29972D967FAF2D9761968FAFE2
:10772000619765969FAF65979801A8EEB3E00F94B7
:107730005534C557DF4F688379838A839B83CB5841
:10774000D040DC01CB01840D951DA61DB71DC95687
:10775000DF4F88839983AA83BB83C759D04081E0D8
:1077600080936902C258DF4F488259826A827B82C5
:10777000CE57D040C157DF4F488259826A827B8200
:10778000CF58D040EE961FAEEE97CD56DF4F188201
:1077900019821A821B82C359D040E1961FAEE1972D
:1077A00090E4A1969FAFA197ACE1A596AFAFA59746
:1077B000B6E4A996BFAFA997E5961FAEE597E69602
:1077C0001FAEE697E7961FAEE797E8961FAEE897DD
:1077D000A0961CAE1DAE1EAE1FAEA0976C961CAE42
:1077E0001DAE1EAE1FAE6C97C12CD12C76012FE7BB
:1077F00030E040E050E028962CAF3DAF4EAF5FAF99
:1078000028973FE7832E912CA12CB12CCE57DF4F28
:10781000188219821A821B82C258D04031E0ED963C
:107820003FAFED97AE961FAE1EAEAE9710E0212C87
:10783000312C00E04CAD842F440F990BDC01A05398
:10784000BB4FC556DF4FB983A883CB59D040880FB3
:10785000991F880F991FFC01EC5AF94EEA96FFAF69
:10786000EEAFEA97EB962FADEB97022E000C330BA1
:10787000EC963FAF2EAFEC9780916902882309F414
:1078800038C10E948EA324966CAF7DAF8EAF9FAFA0
:1078900024978091B904882309F407C10E947D755B
:1078A0003CAD37FF09C01091D3042090D404309030
:1078B000D5040091D6040DC0EA96AEADBFADEA97EF
:1078C0001C9111962C90119712963C90129713963A
:1078D0000C91212F322D432D502FE5966FADE5975A
:1078E000E6967FADE697E7968FADE797E8969FAD72
:1078F000E8970F94FB2F87FF0CC0E5961FAFE59725
:10790000E6962FAEE697E7963FAEE797E8960FAF7D
:10791000E897212F322D432D502FE1966FADE1973F
:10792000A1967FADA197A5968FADA597A9969FAD7E
:10793000A9970F948B36181664F4E1961FAFE19760
:10794000A1962FAEA197A5963FAEA597A9960FAF8A
:10795000A997ED96BFADED9729962FAD29972D9656
:107960003FAD2D9761964FAD619765965FAD659779
:10797000612F722D832D902FBB2309F476C00F94B5
:107980008B3618160CF091C024962CAD3DAD4EAD43
:107990005FAD24972419350946095709C256DF4FB0
:1079A000288339834A835B83CE59D040DA01C901E9
:1079B00088589341A109B109B7FD77C0D501C40129
:1079C00028962CAD3DAD4EAD5FAD2897821B930B35
:1079D000A40BB50B3CADB595A7959795879537FF4B
:1079E00003C08093D10407C0C556DF4FE881F981F9
:1079F000CB59D0408083C256DF4F288139814A81DC
:107A00005B81CE59D040CE57DF4F288339834A83DC
:107A10005B83C258D04029963FAD2997E5963FAF8A
:107A2000E5972D964FAD2D97E6964FAFE697619669
:107A30005FAD6197E7965FAFE79765968FAD659706
:107A4000E8968FAFE89724962CAD3DAD4EAD5FAD77
:107A50002497C258DF4F288339834A835B83CE57EC
:107A6000D040ED961FAEED9720C00F94FB2F87FFFF
:107A70001CC024968CAD9DADAEADBFAD2497C25851
:107A8000DF4F288139814A815B81CE57D040821BEC
:107A9000930BA40BB50BAC01BD01485853416109D0
:107AA000710977FD02C00C94814620E030E040EA85
:107AB00051E429966FAD29972D967FAD2D9761964C
:107AC0008FAD619765969FAD65970F9465349B0167
:107AD000AC01612F722D832D902F0F948B361816C9
:107AE0007CF4E3E0F8E084918F010F5F1F4F811178
:107AF00003C00E94C3743DC70F943F26F801F3CF23
:107B000024968CAD9DADAEADBFAD2497C157DF4F70
:107B1000288139814A815B81CF58D040821B930BE9
:107B2000A40BB50BB7FDCAC00E9473738AE00F9413
:107B30003F2624968CAD9DADAEADBFAD249780534E
:107B4000984FAF4FBF4FC157DF4F88839983AA83A8
:107B5000BB83CF58D040EE969FADEE97911185C074
:107B6000CD56DF4F288139814A815B81C359D0408E
:107B7000612F722D832D902F0F948B3618160CF0D9
:107B800055C020E030E040E050E4612F722D832D9D
:107B9000902F0F946534CD56DF4F688379838A83A5
:107BA0009B83C359D04024962CAD3DAD4EAD5FAD07
:107BB0002497C557DF4F88819981AA81BB81CB5813
:107BC000D040280F391F4A1F5B1FC956DF4F28833B
:107BD00039834A835B83C759D040C957DF4F288117
:107BE00039814A815B81C758D04029966FAD29976A
:107BF0002D967FAD2D9761968FAD619765969FAD60
:107C000065970F9464349B01AC0191E0EE969FAFB1
:107C1000EE97612F722D832D902F0F948B361816AF
:107C20000CF44CC0EE961FAEEE9748C024968CAD77
:107C30009DADAEADBFAD2497C956DF4F28813981C8
:107C40004A815B81C759D040821B930BA40BB50BB3
:107C5000B7FD34C03CAD3F3F19F04FEC57E002C0D8
:107C600041EE57E064EF77E026C020E030E040EAE4
:107C700051E429966FAD29972D967FAD2D9761968A
:107C80008FAD619765969FAD65970F9464349B01A6
:107C9000AC01612F722D832D902F0F94FB2F87FF46
:107CA0000DC04CAD4F3F19F048E957E002C04BEA18
:107CB00057E06FEB77E08CAD0E949C7524968CADFD
:107CC0009DADAEADBFAD2497880F991FAA1FBB1FF6
:107CD000C258DF4F288139814A815B81CE57D0401D
:107CE000821B930BA40BB50B84199509A609B70940
:107CF00081389F44A241B10568F0EAE7F7E084913A
:107D00008F010F5F1F4F882309F4F3CE0F943F2696
:107D1000F801F5CFAE964EAD5FADAE97EC968EAD59
:107D20009FADEC97841795070CF0B3C0EDE1F7E039
:107D300084918F010F5F1F4F882321F00F943F26FE
:107D4000F801F6CF9CAD97FD03C00AE113E002C035
:107D50000FE013E0B8018CE097E00E94A2FEB701AB
:107D6000A60188E097E00E9445FE8AE00F943F2636
:107D7000B80187EF96E00E94A2FE6C964CAD5DAD17
:107D80006EAD7FAD6C9783EF96E00E9445FE8AE072
:107D90000F943F26B80182EE96E00E94A2FEA096C4
:107DA0004CAD5DAD6EAD7FADA0978EED96E00E94BF
:107DB00045FE8AE00F943F26CA57DF4FA881C65878
:107DC000D040AA2309F4D5C5BCADB7FF31C0C092DD
:107DD0000615D0920715E0920815F09209152CEAC5
:107DE00035EC47E25EE36C966CAD7DAD8EAD9FAD3C
:107DF0006C970F9460306093021570930315809315
:107E00000415909305152CEA35EC47E25EE3A09645
:107E10006CAD7DAD8EAD9FADA0970F944135609355
:107E2000FE147093FF148093001590930115A1C563
:107E3000C0921215D0921315E0921415F0921515F8
:107E40002CEA35EC47E25EE36C966CAD7DAD8EAD11
:107E50009FAD6C970F94603060930E1570930F1563
:107E600080931015909311152CEA35EC47E25EE3F0
:107E7000A0966CAD7DAD8EAD9FADA0970F944135B2
:107E800060930A1570930B1580930C1590930D1544
:107E900070C50E9442BCF0CC80E50E949B6A88239A
:107EA00051F00E94646A60930615709307158093E1
:107EB00008159093091589E40E949B6A882381F034
:107EC0000E94646A2CEA35EC47E25EE30F9460306E
:107ED0006093021570930315809304159093051514
:107EE00084E40E949B6A882381F00E94646A2CEAE1
:107EF00035EC47E25EE30F9441356093FE147093D6
:107F0000FF148093001590930115ECEFF4E4849135
:107F10008F010F5F1F4F882321F00F943F26F80138
:107F2000F6CF409106155091071560910815709194
:107F300009158DEB98E00E9445FE2CEA35EC47E2EE
:107F40005EE3609102157091031580910415909184
:107F500005150F944135AB01BC0189EB98E00E94F7
:107F600045FE2CEA35EC47E25EE36091FE14709129
:107F7000FF1480910015909101150F946030AB01B2
:107F8000BC0185EB98E00E9445FE8AE00F943F26F5
:107F9000F0C483E50E949B6A811106C053E1E52E7F
:107FA00053E0F52E10E00EC010E00E94446A682FE6
:107FB000812F0E94F5EB1F5F1530B9F7EFCF1F5FE0
:107FC000143071F0F70181917F010E949B6A882330
:107FD000B1F30E94446A682F812F0E94F5EBEFCF26
:107FE00082E40E949B6A882331F00E94446A682FD1
:107FF00084E00E94F5EB0E945EEBBBC483E50E9427
:10800000E26A8823E1F10E94446A813041F08230C3
:10801000B1F533E1E32E33E0F32E10E021C043E16C
:10802000E42E43E0F42E10E0D7018D917D010E94F3
:10803000E26A882339F00E94446A4FEF682F812F4B
:108040000E94E0831F5F143079F782E40E94E26AA5
:108050008823A9F00E94446A12C01F5F1430A9F35C
:10806000F70181917F010E94E26A8823B1F30E94A7
:10807000446A482F6FEF812F0E94E083EECF0E9469
:108080005EEB77C4E7E6F7E484918F010F5F1F4F43
:10809000882321F00F943F26F801F6CFE1ECF8E0B9
:1080A00084918F010F5F1F4F882309F462C40F94DE
:1080B0003F26F801F5CF0E9427625BC480E00E9452
:1080C000F9640E94187C55C40E940A7E52C48AE555
:1080D0000E949B6A882329F18091AC039091AD03A3
:1080E000892B19F00E94646A08C060915D16709136
:1080F0005E1680915F16909160166093ED03709309
:10810000EE038093EF039093F00380E090E0A0E80B
:10811000BFE38093F1039093F203A093F303B09332
:10812000F40386E40E949B6A882381F10E94646ABA
:1081300020E030E040E85FE30F948B3618166CF4D3
:108140000E94646A20E030E040E85FE30F948B36E1
:10815000181684F00E94646A11C00E94646A20E0CC
:1081600030E0A9010F94FB2F87FFEACF60E070E0B9
:10817000CB0104C060E070E080E89FE36093F1030E
:108180007093F2038093F3039093F40383E50E94CA
:108190009B6A882351F00E94646A60930202709384
:1081A000030280930402909305028AE50E949B6A71
:1081B0008111DFC386E40E949B6A8111DAC383E5E3
:1081C0000E949B6A8111D5C336C70E9408F2D1C3B1
:1081D0000F94091DCEC383E50E949B6A882321F07A
:1081E0000E94556A91E089270F94B917C2C30E9473
:1081F0002B79BFC383E50E949B6A882309F4B9C326
:108200000E94556A8093270CB4C380E090E0A0E2FE
:10821000B1E489839A83AB83BC8380E090E0A4E3DC
:10822000B3E48D839E83AF83B88780E090E0A0EABB
:10823000B1E489879A87AB87BC8788E592E00E9482
:10824000DC6C811196C36091D2040E947ADF0E9497
:1082500043E2882319F081E00E94ABB385E40E94D9
:108260009B6A882381F00E94646A6B017C0120E094
:1082700030E0A9010F948B3687FF0AC0F7FAF0941B
:10828000F7F8F09405C0C12CD12CE12C20E4F22E9B
:10829000F7FAF094F7F8F094C8AED9AEEAAEFBAEB8
:1082A0008AE50E94E26A882379F08AE50E94E26A00
:1082B000882319F00E94646A03C060E070E0CB017B
:1082C00069877A878B879C8788E50E94E26A882382
:1082D00079F088E50E94E26A882319F00E94646AB6
:1082E00003C060E070E0CB0169837A838B839C8359
:1082F00089E50E94E26A882379F089E50E94E26AB2
:10830000882319F00E94646A03C060E070E0CB012A
:108310006D837E838F83988785E50E949B6A88237F
:1083200029F00E94646A6B017C010CC0E091581630
:1083300024E0E29FF0011124EA51FB4EC080D1807D
:10834000E280F38020E030E0A901C701B6010F947C
:108350008B3687FF04C0F7FAF094F7F8F094F7FA39
:10836000F094F7F8F094CCAADDAAEEAAFFAA18AA16
:1083700019AA1AAA1BAA8CE40E949B6A882329F0D6
:108380000E94646A6B017C010CC0E091581634E0D5
:10839000E39FF0011124E651FB4EC080D180E280C2
:1083A000F38020E030E0A901C701B6010F948B36BD
:1083B00087FF04C0F7FAF094F7F8F094CCA6DDA696
:1083C000EEA6FFA682E40E94E26A882321F00E94C2
:1083D000346A162F01C01AE00091FF0B8091540EF1
:1083E0008111E4C021E0AE014C5C5F4FBE016F5FC4
:1083F0007F4FCE01C8960F948A00882309F4D6C017
:108400006091581682E00E947ADFECEFF4E48491E8
:108410007F014FEFE41AF40A882321F00F943F26DE
:10842000F701F5CFE5E0FAE084917F015FEFE51A0F
:10843000F50A882321F00F943F26F701F5CF61E07C
:10844000812F0F942B0A0E948EA3DC01CB01805256
:108450009C46AB4FBF4F8093A5049093A604A09376
:10846000A704B093A8041092600E83E08093BB141D
:1084700081E08093AC15DD24D3948091AC158823E2
:1084800009F47AC060E0812F0F942B0A8091600E6E
:10849000882309F46DC06091581688E00E947ADF45
:1084A000ECEFF4E484917F019FEFE91AF90A882345
:1084B00021F00F943F26F701F5CFEEEDF9E084911E
:1084C0007F01AFEFEA1AFA0A882321F00F943F26C2
:1084D000F701F5CF8091AC15882321F081E00F944E
:1084E000BB1EF8CF1092A5041092A6041092A70408
:1084F0001092A8041092600E0E9478740F94DD2AE6
:108500006091581682E00E947ADFECEFF4E48491E7
:108510007F01BFEFEB1AFB0A882321F00F943F265F
:10852000F701F5CFE2EBF9E084917F012FEFE21A3A
:10853000F20A811119C00E948EA3DC01CB01805286
:108540009C46AB4FBF4F8093A5049093A604A09385
:10855000A704B093A8041092600ED092AC1561E00D
:10856000812F0F942B0A04C00F943F26F701DCCF14
:1085700081E00F94BB1E81CF81E08093BB1480E02B
:1085800090E0A0EAB1E488A399A3AAA3BBA3809139
:10859000540E882359F0212FAE01405E5F4FBE017B
:1085A000645D7F4FCE01C0960F94CC01013009F07D
:1085B000E0C10E94B693DDC18BE592E00E94DC6CC5
:1085C0008111D7C185E50E949B6A8823D9F100916A
:1085D000D20410E00E94646A6B017C0120E030E06C
:1085E000A9010F948B3687FF04C0F7FAF094F7F8CF
:1085F000F094000F111F000F111FF801EA51FB4EFC
:10860000C082D182E282F3820091D20434E0039FDF
:10861000800111240A511B4E20E030E048E453E46D
:10862000D8016D917D918D919C910F948B36181688
:108630004CF480E090E0A8E4B3E4F80180839183F7
:10864000A283B3838CE40E949B6A882309F491C1BE
:108650000091D20410E00E94646A6B017C0120E06A
:1086600030E0A9010F948B3687FF04C0F7FAF0942D
:10867000F7F8F094000F111F000F111FF801E651D9
:10868000FB4EC082D182E282F3820091D204F4E0F8
:108690000F9F8001112406511B4E20E030E048E47A
:1086A00053E4D8016D917D918D919C910F948B36FF
:1086B00018160CF05EC180E090E0A8E4B3E4F80185
:1086C00080839183A283B38354C18AE50E94E26AC6
:1086D000882309F438C00E94646A6B017C0120E0A1
:1086E00030E040E050EC0F948B3687FD13C020E063
:1086F00030E040EA50E4C701B6010F94FB2F181692
:108700004CF0C0923312D0923412E0923512F092B3
:1087100036122FC1E7E6F7E484918F010F5F1F4FF8
:1087200081110DC0E3E4FAE084918F010F5F1F4FC8
:10873000882309F41EC10F943F26F801F5CF0F944A
:108740003F26F801E9CFECEFF4E484918F010F5F4D
:108750001F4F882321F00F943F26F801F6CFE4E362
:10876000FAE084918F010F5F1F4F882321F00F944F
:108770003F26F801F6CF40913312509134126091A8
:1087800035127091361281E39AE00E9445FE8AE02C
:108790000F943F26EEC08BE40E94E26A8823B1F179
:1087A0008BE40E94E26A8823B1F00E94646A6B0144
:1087B0007C0120E030E0A9010F948B3687FD19C0C1
:1087C00020E030E040E251E4C701B6010F94FB2FF6
:1087D00018167CF003C0C12CD12C76010E942762B0
:1087E000C092FA14D092FB14E092FC14F092FD14A3
:1087F000C0C0EEE5FAE084918F010F5F1F4F882320
:1088000009F4B7C00F943F26F801F5CFECEFF4E47C
:1088100084918F010F5F1F4F882321F00F943F2613
:10882000F801F6CF4091FA145091FB146091FC14BA
:108830007091FD148DE79AE00E9445FE8AE00F9446
:108840003F2697C088E50E949B6A8823F1F00E942A
:10885000346A8B01072E000C220B330B0093EE14AD
:108860001093EF142093F0143093F114DB012FEFE9
:1088700030E00F945C3720ED37E040E050E00F949B
:108880002934B9018EE20E948FA28AE50E949B6A78
:10889000882329F00E94346A81E00E94358485E4AF
:1088A0000E949B6A882309F464C00E94346A82E0B3
:1088B0000E9435845EC081E080930A02109271129A
:1088C00083E50E94E26A882339F00E94556A81118B
:1088D00050C00F9489224DC083E50E949B6AF7CF58
:1088E0000F945A2B46C0F090A3140E942762FF20D9
:1088F00029F1ECEFF4E484918F010F5F1F4F88237F
:1089000021F00F943F26F801F6CF84E50F943F261F
:108910006F2D70E080E090E04AE00F94922680E2B4
:108920000F943F26EAE9FAE084918F010F5F1F4F11
:108930008823F9F00F943F26F801F6CF10925816CD
:10894000ECEFF4E484918F010F5F1F4F882321F037
:108950000F943F26F801F6CF6091581670E088E832
:108960009AE00E9489FE8AE00F943F2602C00F948D
:108970005A2B1092BB14C356DF4FF881CD59D0400B
:10898000FF2309F4DDC30F942322DAC30E942E6C67
:108990008CEB94E10F94CE2180915C1683FDA5C0F1
:1089A000C090C814D090C914E090CA14F090CB14B1
:1089B00020912F1230913012409131125091321289
:1089C000C701B6010F94FB2F882309F48EC0609174
:1089D0005416709155168091561690915716209105
:1089E0005916211129C00F94A93520916A0230919E
:1089F0006B026217730704F5C0922F12D0923012E7
:108A0000E0923112F0923212ECEFF4E484918F0193
:108A10000F5F1F4F882321F00F943F26F801F6CFF8
:108A2000E2EAF2E084918F010F5F1F4F882321F06B
:108A30000F943F26F801F6CF8090C8149090C91487
:108A4000A090CA14B090CB1420912F123091301204
:108A50004091311250913212C501B4010F94643427
:108A60006B017C0120E030E0A9010F948B3687FF79
:108A700004C0F7FAF094F7F8F094E091581624E067
:108A8000E29FF0011124EA5FFD4F20813181428194
:108A90005381C701B6010F94603020E030E048E414
:108AA00053E40F948B36181604F580922F1290928F
:108AB0003012A0923112B0923212ECEFF4E48491B1
:108AC0008F010F5F1F4F882321F00F943F26F8017D
:108AD000F6CFE3E8F2E084918F010F5F1F4F882308
:108AE00021F00F943F26F801F6CF609100027091BB
:108AF0000102072E000C880B990B0F940130209176
:108B000070023091710240917202509173020F9481
:108B100060302AE037ED43E25CE30F9460306CA7ED
:108B20007DA78EA79FA7E09058168091C4149091BE
:108B3000C514A091C614B091C7144091C0145091AF
:108B4000C1146091C2147091C3140091BC141091AF
:108B5000BD142091BE143091BF1409831A832B8356
:108B60003C8348A359A36AA37BA38CAB9DABAEAB5C
:108B7000BFAB18AE19AE1AAE1BAEAE014C5C5F4F68
:108B8000BE01605E7F4FCE0101960E94FD6FAE0177
:108B9000485C5F4F6A018E01045D1F4F28EC34E191
:108BA00044505109BE01605E7F4FCE0101960E9484
:108BB0007A500E9427BBDDCE0E94276288E50E9482
:108BC0009B6A882331F0179A8091130C8E7F8093D3
:108BD000130C89E50E949B6A882331F0169A8091D4
:108BE000130C8D7F8093130C8AE50E949B6A882367
:108BF00031F0159A8091130C8B7F8093130C85E4D0
:108C00000E949B6A882309F4B4CE149AB2CE0E94C3
:108C1000646A20E030E040E050EC0F94FB2F87FDC9
:108C200015C00E94646A20E030E040E050E40F94F8
:108C30008B3618162CF00E94646A6B017C010BC005
:108C4000C12CD12CE12CE0E4FE2E05C0C12CD12C8E
:108C5000E12C70ECF72E20914F1230915012409180
:108C60005112509152128091130C82FF10C000914A
:108C7000BE041091BF04C701B6010F9460300F9479
:108C8000A935600F711F7093BF046093BE0480E527
:108C90000E949B6A882329F00E94556A882309F460
:108CA00068CEA701960160913312709134128091C1
:108CB0003512909136120F9465346093331270938D
:108CC00034128093351290933612ECEFF4E48491D1
:108CD0008F010F5F1F4F882321F00F943F26F8016B
:108CE000F6CF409133125091341260913512709149
:108CF000361283E996E00E9445FE8AE00F943F26F3
:108D000038CEAE964EAD5FADAE97452B09F44AC155
:108D1000CE57DF4F488059806A807B80C258D04050
:108D2000480E591E6A1E7B1ECE57DF4F288139819F
:108D30004A815B81C258D040281B390B4A0B5B0B20
:108D4000CA01B90128962CAD3DAD4EAD5FAD289757
:108D50000F94F833A30192010F942934D501C40173
:108D6000820F931FA41FB51F84319105A105B10582
:108D70000CF14C015D018C3E9105A105B1052CF073
:108D8000FBEE8F2E912CA12CB12C40E8841691047F
:108D9000A104B104FCF08EEF90E0A0E0B0E08819EF
:108DA0009909AA09BB0928968CAF9DAFAEAFBFAF9A
:108DB000289716C0E4E18E2E912CA12CB12C24E131
:108DC00030E040E050E028962CAF3DAF4EAF5FAFB3
:108DD000289706C028968CAE9DAEAEAEBFAE289743
:108DE000B501A4018FE698E00E9462FE28964CAD82
:108DF0005DAD6EAD7FAD28978AE698E00E9462FE79
:108E0000E1964FADE197A1965FADA197A5966FADA5
:108E1000A597A9967FADA99783E698E00E9445FEA5
:108E2000E5964FADE597E6965FADE697E7966FADB1
:108E3000E797E8967FADE8978CE598E00E9445FEBD
:108E4000AE964EAD5FADAE97433051050CF4AAC05F
:108E500028966CAD7DAD8EAD9FAD28970F940130F7
:108E600020E030E040E850E40F9460306B017C017A
:108E7000E1962FADE197A1963FADA197A5964FAD95
:108E8000A597A9965FADA997E5966FADE597E6968C
:108E90007FADE697E7968FADE797E8969FADE897A9
:108EA0000F9464342BED3FE049E450E40F946030BC
:108EB00020E030E040E05FE30F9460309B01AC01C4
:108EC000C701B6010F9441356B017C01C301B201AA
:108ED0000F9401302FE632E143E85AE30F946030FB
:108EE0002B013C01B701A60186E598E00E9445FEF2
:108EF000B301A20180E598E00E9445FE2AE939E924
:108F000049E15FE3C701B6010F9460306B017C015A
:108F10009B01AC010F946534A30192010F9441357C
:108F20006C966CAF7DAF8EAF9FAF6C97A301920133
:108F3000C701B6010F94603020E030E040E05EE30E
:108F40000F946030A0966CAF7DAF8EAF9FAFA097AF
:108F5000E0E4F8E084913F015FEF651A750A882329
:108F600021F00F943F26F301F5CFB701A6018AE364
:108F700098E00E9445FE6C964CAD5DAD6EAD7FAD48
:108F80006C9784E398E00E9445FEA0964CAD5DADE1
:108F90006EAD7FADA0978EE298E00E9445FE8AE01C
:108FA0000F943F2628968CAD9DADAEADBFAD2897F2
:108FB000880D991DAA1DBB1DECADB595A79597957C
:108FC0008795E7FF03C08093D10407C0C556DF4FE4
:108FD000E881F981CB59D0408083AE962EAD3FAD6C
:108FE000AE972F5F3F4FAE963FAF2EAFAE9729960D
:108FF0003FAD2997E1963FAFE1972D964FAD2D9765
:10900000A1964FAFA19761965FAD6197A5965FAFAF
:10901000A59765968FAD6597A9968FAFA99724966A
:109020004CAC5DAC6EAC7FAC249791E0ED969FAFFD
:10903000ED970C94553D40915D1650915E166091F0
:109040005F167091601685E999E00E9445FE8AE0FE
:109050000F943F268AE00F943F2620E030E0A901DC
:109060006091ED037091EE038091EF039091F00316
:109070000F948B3618160CF056C020E030E0A90192
:109080006091F1037091F2038091F3039091F403E6
:109090000F948B3618160CF046C0E3E5F9E0849186
:1090A0008F010F5F1F4F882321F00F943F26F80197
:1090B000F6CF4091ED035091EE036091EF03709174
:1090C000F00389E399E00E9445FE8AE00F943F2671
:1090D00040910202509103026091040270910502D6
:1090E0008FE199E00E9445FE8AE00F943F2640916F
:1090F000F1035091F2036091F3037091F40385E062
:1091000099E00E9445FE8AE00F943F26E0EDF8E0EA
:1091100084918F010F5F1F4F882309F42ACC0F948D
:109120003F26F801F5CFE3E7F9E084918F010F5F67
:109130001F4F882309F4BDCF0F943F26F801F5CFC8
:10914000CF55DF4F0FB6F894DEBF0FBECDBFDF9116
:10915000CF911F910F91FF90EF90DF90CF90BF9034
:10916000AF909F908F907F906F905F904F903F90C7
:109170002F9008954F925F926F927F92BF92CF92FD
:10918000DF92EF92FF920F931F93CF93DF93CDB7B0
:10919000DEB72A970FB6F894DEBF0FBECDBF109290
:1091A000340E80912D0F882351F120911F1122231D
:1091B00021F18091C9119091CA11A091CB11B09168
:1091C000CC110097A105B105B9F0BC01CD016D59D5
:1091D0007F4F8F4F9F4F24E630E040E050E00F94E8
:1091E00007346091CD117091CE118091CF11909183
:1091F000D0110F94073401C020E02093E114809136
:109200003A0E10923A0E882339F00E94959180E030
:1092100091E00E941CD603C520910002309101020A
:109220004091650E5091660E6091670E7091680EC8
:10923000C901840F951F2436310524F48536910524
:109240003CF416C02436310531F08436910584F49F
:1092500084E690E00DC0473051056105710514F0BA
:10926000069706C04A3F5F4F6F4F7F4F6CF40696DC
:1092700090930102809300021092650E1092660E88
:109280001092670E1092680E809100029091010278
:109290008A3091053CF0883E43E094072CF087EE3D
:1092A00093E002C08AE090E0909301028093000274
:1092B0000E947FBFB82E0E9480BB80911012853122
:1092C00098F4BB2049F080910B0E90910C0E892BE5
:1092D00019F005E111E102C008EF1FE023E14FE0C2
:1092E00061E088E00E94B5D4809110128D3108F0C1
:1092F00008C18830A0F58091600EB11002C08111C4
:109300002EC060915A1670915B16072E000C880BC8
:10931000990B0F94013020E030E040E05FE30F94C0
:1093200065340F94A935CB010E9491E9FC0120819D
:10933000203229F42181203221F436E003C030E0CC
:1093400001C033E025E0231B2093131227E0209374
:1093500014120E94529285EF9FE00E9445928091E4
:1093600010128D31A0F580911212853180F120E02C
:1093700030E040E05FE360915416709155168091A3
:109380005616909157160F9465340F94A935CB015A
:109390000E9491E9FC018081803209F0B7C281818D
:1093A000803209F0ACC296E085E0891B80931312ED
:1093B0008CE180931412CF010E94529285EF9FE0BE
:1093C0000E94459280911012853108F49AC28091D2
:1093D00010128830A0F580915F0EB11002C081118B
:1093E0002EC06091D7047091D804072E000C880B12
:1093F000990B0F94013020E030E040E05FE30F94E0
:1094000065340F94A935CB010E9491E9FC012081BC
:10941000203229F42181203221F436E003C030E0EB
:1094200001C033E021E5231B2093131227E0209392
:1094300014120E94529285EF9FE00E944592809103
:1094400010128D31A0F580911212853180F120E04B
:1094500030E040E05FE36091D3047091D4048091E8
:10946000D5049091D6040F9465340F94A935CB019F
:109470000E9491E9FC018081803209F07DC28181E6
:10948000803209F072C296E081E5891B8093131245
:109490008CE180931412CF010E94529285EF9FE0DD
:1094A0000E94459280911012853108F460C280912B
:1094B00010128C3130F580911212843110F18091AC
:1094C0000B0E90910C0E019644E6489F9001499F27
:1094D000300D112437FF02C021503F4F832F932FAF
:1094E000990F990B009769F028E6209313122BE14E
:1094F000209314120E9491E90E94529285E20E94E8
:10950000B7D580911F11882349F0809110128433C0
:1095100028F4809112128A3208F05DC280911012F4
:10952000853328F480911212813308F07AC2609159
:10953000E114623048F080911012843328F4809155
:109540001212823308F072C280911012813308F037
:1095500060C080911212893208F45BC00E946D9342
:109560002B013C018CE3C82ED12CE12CF12CC30142
:10957000B201A70196010F940734CA01B901A701EE
:1095800096010F940734CA01F62EE72E69018E0169
:109590000F5F1F4F40E8441641E5540641E0640662
:1095A000710408F45EC2B90128E130E040E050E007
:1095B0000F94073429013A01EF92FF92C60168E146
:1095C00070E00F942D379F938F935F924F928EEBA5
:1095D0009AE09F938F931F930F930F94942F0FB63E
:1095E000F894DEBF0FBECDBF9AE049165104610466
:1095F000710408F060C298E0892F880F980F919548
:10960000955A9093131280E380931412C8010E941C
:109610005292E091D611F091D711848181112FC11E
:109620002091611630916216409163165091641634
:10963000609123127091241280912512909126122C
:109640000F9465346B017C0120E030E0A9010F9498
:10965000FB2F87FD05C020E030E040E05FE304C061
:1096600020E030E040E05FEBC701B6010F946534C5
:109670000F94A935CB010E94FEE8BC0183EE93E074
:109680000F94A937209165163091661640916716A0
:1096900050916816609127127091281280912912BA
:1096A00090912A120F9465346B017C0120E030E028
:1096B000A9010F94FB2F87FD05C020E030E040E0BA
:1096C0005FE304C020E030E040E05FEBC701B6019B
:1096D0000F9465340F94A935CB010E94FEE8BC01BC
:1096E0008EED93E00F94A9372091691630916A1698
:1096F00040916B1650916C1660912B1270912C1248
:1097000080912D1290912E120F9465346B017C0183
:1097100020E030E04AE754E40F9460302B013C0134
:1097200020E030E0A901C701B6010F94FB2F87FDAF
:1097300005C020E030E040EA50E404C020E030E022
:1097400040EA50ECC301B2010F94653420E030E0F0
:1097500040E251E40F9441350F94A9356B017C012F
:1097600097FD16C06031F7E27F0781059105D4F0BF
:1097700020E137E240E050E00F942934CA01B901FA
:109780002AE030E040E050E00F942934605D0BC0E7
:10979000F094E094D094C094C11CD11CE11CF11C45
:1097A0006DE201C060E26093A71428EEC21623E0C8
:1097B000D206E104F10494F0C701B60128EE33E0CB
:1097C00040E050E00F942934CA01B9012AE030E0AA
:1097D00040E050E00F942934605D01C060E2609386
:1097E000A814C701B60124E630E040E050E00F9431
:1097F00029349AE0492E512C612C712CCA01B901EF
:10980000A30192010F942934605D6093A914C701EC
:10981000B601A30192010F9429346B017C01672BDF
:10982000682B692B79F08EE28093AA14CA01B901E2
:10983000A30192010F942934605D6093AB1480E31F
:109840008C0D15C0CA01B901A30192010F942934EE
:10985000662339F08EE28093AA14605D6093AB14A6
:1098600005C080E28093AB148093AA1480E28093B9
:10987000AC1467EA74E187ED93E00F94A937809107
:1098800010128632A8F4809112128E3188F008E00E
:1098900020E84EE160E08CED91E10E94C29F809152
:1098A0001012863228F4809112128F3108F005C10F
:1098B00080911012823328F4809112128C3208F0B9
:1098C0008FC1809110128F3308F0A9C180911212BC
:1098D000883308F4A4C1109213128EE380931412FB
:1098E00089E69EE00E94C5BF182F0E94D8D5163188
:1098F00008F095C180E20E94B7D51F5FF8CF93E0D2
:1099000053CD80911212813118F461CD90E04CCD8D
:1099100060915A1670915B16072E000C880B990BFC
:109920000F940130209154163091551640915616DF
:10993000509157160F948B36181674F41092FC1130
:1099400002E022E041E16DE08CED91E10E94C29FD6
:1099500081E08093FC113BCD02E022E041E16DE02B
:109960008CED91E10E94C29F32CD93E08DCD80912C
:109970001212813118F49BCD90E086CD6091D7040E
:109980007091D804072E000C880B990B0F940130AE
:109990002091D3043091D4044091D5045091D60441
:1099A0000F948B36181674F41092FC1102E022E02A
:1099B00042E168E58CED91E10E94C29F81E08093D5
:1099C000FC1175CD02E022E042E168E58CED91E109
:1099D0000E94C29F6CCD07E028E04AE26AE28CED6B
:1099E00091E10E94C29F05E022E04CE262E38CED2F
:1099F00091E10E94C29F6AE08AE20E940BD56091C9
:109A0000DE117091DF1182E38093F8118BE2809375
:109A1000F91128EF31E142E38CED91E10E94009EC3
:109A20007DCD6AE486E30E940BD581CDF8E46F9F7B
:109A3000B0011124072E000C880B990B0F940130F4
:109A40002AE037ED43E25CE30F9460300F94AE35CB
:109A5000262F02E042E367E38CED91E10E94C29F72
:109A600073CDE4E6CE16D10498F4EF92FF923F93C3
:109A70002F9384EB9AE09F938F931F930F930F94F0
:109A8000942F0FB6F894DEBF0FBECDBF95E0B4CDD6
:109A9000EF92FF923F932F938CEA9AE09F938F93DC
:109AA0001F930F930F94942F0FB6F894DEBF0FBE41
:109AB000CDBF96E0A1CD99E09FCD1092FC1183E03F
:109AC0008093131215E21093141283EF9FE00E940B
:109AD00045928BE08093131210931412BB2029F04F
:109AE00083EE93E00E94529219C08091571280FD3C
:109AF0000DC003EE13E0F80181918F01882371F00E
:109B00008F3208F08FE30E943192F5CF8091130CD1
:109B100080FDE6CF8EEE9FE00E9445928BE280931F
:109B2000131215E2109314128CEE9FE00E944592DE
:109B300083E38093131210931412BB2029F08EED4F
:109B400093E00E94529219C08091571281FD0DC07E
:109B50000EED13E0F80181918F01882371F08F32AF
:109B600008F08FE30E943192F5CF8091130C81FDB4
:109B7000E6CF8EEE9FE00E94459283E5809313121C
:109B800015E2109314128AEE9FE00E9445928BE535
:109B90008093131210931412BB2029F087ED93E0E9
:109BA0000E94529219C08091571282FD0DC007ED9C
:109BB00013E0F80181918F01882371F08F3208F052
:109BC0008FE30E943192F5CF8091130C82FDE6CF96
:109BD00083EE9FE00E94459281E08093FC1168CE65
:109BE00084E00E94009283E08093131212E31093AA
:109BF000141286E00E9431920E9480BB8CE0809318
:109C000013121093141280910002909101020E948D
:109C100091E90E94529285E20E94B7D552CE2A96CF
:109C20000FB6F894DEBF0FBECDBFDF91CF911F916D
:109C30000F91FF90EF90DF90CF90BF907F906F904B
:109C40005F904F900895282F1092340E8091650EEA
:109C50009091660EA091670EB091680E8130904889
:109C6000A105B10540F01092650E1092660E10929B
:109C7000670E1092680E8091290E882331F0809132
:109C8000650E8093E4141092620E80911E0E1816D9
:109C9000FCF4082E000C990B821B91092091E4140E
:109CA000022E000C330B2817390794F097FF02C0DF
:109CB00080E090E08093E414092E000CAA0BBB0B0B
:109CC0008093650E9093660EA093670EB093680E16
:109CD0008091E4146623A9F090911F0E891714F463
:109CE00080931F0E20911F0E022E000C330B2C5F51
:109CF0003F4F482F082E000C550B241735071CF436
:109D0000845080931F0E08958091630E8630D8F49E
:109D100096E0899FF0011124ED54FC4F20915202EE
:109D200030915302318320834091650E5091660E2D
:109D30006091670E7091680E4283538364837583CC
:109D40008F5F8093630E08958AEB98E40C941CD681
:109D5000E091630EEE2369F0E150E093630E86E03C
:109D6000E89FF0011124ED54FC4F808191810C9407
:109D70001CD6EACFAF92BF92CF92DF92EF92FF92C2
:109D80000F931F93CF93DF935C016B010E94B7BFCA
:109D9000EC01C6010E94C5BF04E110E0081B1109D7
:109DA000DD270C171D071CF0FF24F39402C082E08E
:109DB000F82E8091DD1190E06F2D70E06F5F7F4F86
:109DC0000F944137E62EC6E0C60F80911012C817D7
:109DD00050F04091121250E02C2F30E02B503109FE
:109DE000421753079CF5D0E0C114D104C1F18AE3B6
:109DF0000E94B7D582E0F8120FC0CE0D80911012EC
:109E0000C81768F12091121230E08C2F90E00B9768
:109E1000281739071CF423C0DD2309F1902F990F6F
:109E2000090F000F00931312C093141280E20E94D6
:109E3000B7D5C601DF91CF911F910F91FF90EF90A1
:109E4000DF90CF90BF90AF900C945292109213126B
:109E5000C0931412C5010E94C2D5D1E0C5CFDF91D5
:109E6000CF911F910F91FF90EF90DF90CF90BF9017
:109E7000AF9008950F934CE0849F402D112421E072
:109E8000240F20935D128CE0840F80935E12E0918A
:109E90001012F0E090E002968E179F070CF1822FCF
:109EA00090E02091121230E082179307CCF46623E1
:109EB00071F081E08093FC114D5F0BE020E860E0E1
:109EC0008CED91E10E94C29F1092FC1103C081E0D1
:109ED0008093FC1180915E121092131280931412E1
:109EE0000F910895CF92DF92EF92FF920F93CF934D
:109EF000DF93982F862F6A017901692FBBDF90913C
:109F0000101280915E12891708F448C090911212C5
:109F100080915D12981708F441C0002321F0C70119
:109F20000E94B7BF03C0C7010E94C5BFD82FC4E1BC
:109F3000C81BF6018491882339F00E941A92C81B2D
:109F4000FFEFCF1ADF0AF5CF8AE30E94B7D5CC2303
:109F500029F080E20E94B7D5C150F9CF80915E12FE
:109F60009AEFD99FD02D1124D058D09313128093FB
:109F70001412C701002349F0DF91CF910F91FF9098
:109F8000EF90DF90CF900C944592DF91CF910F919D
:109F9000FF90EF90DF90CF900C945292DF91CF9191
:109FA0000F91FF90EF90DF90CF900895CF92DF92C6
:109FB000EF92FF920F93CF93DF93CDB7DEB7E9898E
:109FC000FA89C080D180E280F38020E030E0A901EE
:109FD000C701B6010F94FB2F87FD05C020E030E0DC
:109FE00040E05FE304C020E030E040E05FEBC70109
:109FF000B6010F9465340F94A935CB010E9491E905
:10A0000000E09C014D855E856C858B856BDFDF9163
:10A01000CF910F91FF90EF90DF90CF900895DF9256
:10A02000EF92FF920F931F93CF93DF931F92CDB7C1
:10A03000DEB77B01622F49831DDF90911012809162
:10A040005E124981891708F44CC0909112128091D8
:10A050005D12981708F445C0442359F10115110504
:10A0600041F5C7010E94B7BF26E130E0281B390B3C
:10A0700037FF02C02F5F3F4F3595279536E1D32E2E
:10A080002751822F8D0D87FD11C080E229830E9408
:10A09000B7D5DA942981F5CFF7018491882361F04F
:10A0A0000E941A92D81A8FEFE81AF80A1D14A4F326
:10A0B00003C086E1D82EFACF0115110559F01D1401
:10A0C0004CF4F80181918F01882321F00E941A92AB
:10A0D000D81AF5CF1D142CF480E20E94B7D5DA947B
:10A0E000F9CF0F90DF91CF911F910F91FF90EF90DB
:10A0F000DF9008952F923F924F925F926F927F92DE
:10A100008F929F92AF92BF92CF92DF92EF92FF9287
:10A110000F931F93CF93DF93CDB7DEB7CC57D10901
:10A120000FB6F894DEBF0FBECDBFE091FA03F091F9
:10A13000FB03EF2B11F00C94105A6C96DFAECEAEF1
:10A140006C972996EFAE299779016A015B01FC01B2
:10A150002081318142815381A6962CAF3DAF4EAF15
:10A160005FAFA69720914712309148124091491253
:10A1700050914A12A6966CAD7DAD8EAD9FADA6975F
:10A180000F9460300F949636E2966CAF7DAF8EAF31
:10A190009FAFE297D5018D919D910D90BC91A02D1F
:10A1A000AA968CAF9DAFAEAFBFAFAA9720914B12CE
:10A1B00030914C1240914D1250914E12BC01CD0184
:10A1C0000F9460300F949636E6966CAF7DAF8EAFED
:10A1D0009FAFE697D6012D913D914D915C91AE9642
:10A1E0002CAF3DAF4EAF5FAFAE9720914F12309185
:10A1F00050124091511250915212AE966CAD7DADFD
:10A200008EAD9FADAE970F9460300F949636EA9660
:10A210006CAF7DAF8EAF9FAFEA97D7012D913D9187
:10A220004D915C916A962CAF3DAF4EAF5FAF6A9790
:10A230002091531230915412409155125091561260
:10A240006A966CAD7DAD8EAD9FAD6A970F94603010
:10A250000F949636A0966CAF7DAF8EAF9FAFA09750
:10A2600080915C1683FF1CC0A0962CAD3DAD4EAD19
:10A270005FADA0972093D90E3093DA0E4093DB0E9A
:10A280005093DC0E6A968CAD9DADAEADBFAD6A97B6
:10A290008093C90E9093CA0EA093CB0EB093CC0EB0
:10A2A000D801BC91BBABF801F181F8AFD80112968F
:10A2B000BC91BCAFF801F3812D96FFAF2D97809133
:10A2C000830E9091840E891B8F708F3021F480E073
:10A2D0000F94BB1EF4CF0091830EEB960FAFEB975C
:10A2E0008091830E282E312C8091CD0E9091CE0E30
:10A2F000A091CF0EB091D00EE2968CAC9DACAEACDE
:10A30000BFACE297881A990AAA0ABB0A8091D10EBB
:10A310009091D20EA091D30EB091D40EE6964CAC93
:10A320005DAC6EAC7FACE697481A590A6A0A7B0AA4
:10A330008091D50E9091D60EA091D70EB091D80EE7
:10A34000EA962CAD3DAD4EAD5FADEA97281B390BBB
:10A350004A0B5B0B2BA33CA34DA35EA38091D90EAC
:10A360009091DA0EA091DB0EB091DC0EA0960CADB0
:10A370001DAD2EAD3FADA097081B190B2A0B3B0B53
:10A380000FA318A729A73AA7012B022B032B09F427
:10A39000BDC06091541670915516809156169091DB
:10A3A000571620915916211141C00F94A9352091BB
:10A3B0006A0230916B0262177307C4F5A0962CAD48
:10A3C0003DAD4EAD5FADA0972093D90E3093DA0E20
:10A3D0004093DB0E5093DC0E6A968CAD9DADAEAD16
:10A3E000BFAD6A978093C90E9093CA0EA093CB0E0F
:10A3F000B093CC0EECEFF4E484918F010F5F1F4F0C
:10A40000882321F00F943F26F801F6CFE1E5F2E131
:10A4100084918F010F5F1F4F882321F00F943F26F7
:10A42000F801F6CF1FA218A619A61AA66FA178A543
:10A4300089A59AA50F94013029960FAD2997A4E01C
:10A440000A9FF0011124EA5FFD4F20813181428192
:10A4500053810F9460306B017C0120E030E0A90152
:10A460000F948B3687FF04C0F7FAF094F7F8F09456
:10A47000609153127091541280915512909156121E
:10A480000F94A9359B01AC01A8ECB0E00F944534C2
:10A490000F9401309B01AC01C701B6010F948B36BC
:10A4A0001816C4F5A0962CAD3DAD4EAD5FADA0978E
:10A4B0002093D90E3093DA0E4093DB0E5093DC0ECE
:10A4C0006A968CAD9DADAEADBFAD6A978093C90E57
:10A4D0009093CA0EA093CB0EB093CC0EECEFF4E4A5
:10A4E00084918F010F5F1F4F882321F00F943F2627
:10A4F000F801F6CFE2E3F2E184918F010F5F1F4F85
:10A50000882321F00F943F26F801F6CF1FA218A64A
:10A5100019A61AA6D501C4018827B7FD83959927E6
:10A52000AA27BB27182F77FC12602BA13CA14DA1B5
:10A530005EA157FD14608FA198A5A9A5BAA5B7FD86
:10A5400018606FA178A589A59AA50F940130299666
:10A550000FAD2997A4E00A9FF0011124EA5FFD4F97
:10A5600020813181428153810F9460306B017C01E5
:10A5700020E030E0A9010F948B3687FF04C0C701AB
:10A58000B601905802C0C701B60120E030E040E0BB
:10A590005FE30F9465340F94AE356CAB7DAB8EAB3F
:10A5A0009FAB88E5829DF001839DF00D1124EB5F48
:10A5B000FA4F108216AB24968CAE9DAEAEAEBFAEF7
:10A5C0002497B7FE0DC022273327A901281939097E
:10A5D0004A095B0924962CAF3DAF4EAF5FAF24977D
:10A5E00088E5829DF001839DF00D1124EB5FFA4F09
:10A5F00024968CAD9DADAEADBFAD2497858B968B6B
:10A60000A78BB08F62964CAE5DAE6EAE7FAE62979A
:10A6100077FE0DC022273327A901241935094609E1
:10A62000570962962CAF3DAF4EAF5FAF629788E59A
:10A63000829DF001839DF00D1124EB5FFA4F62962D
:10A640008CAD9DADAEADBFAD6297818F928FA38F64
:10A65000B48F2BA13CA14DA15EA128962CAF3DAF9C
:10A660004EAF5FAF289757FF0DC05095409530957E
:10A6700021953F4F4F4F5F4F28962CAF3DAF4EAFC8
:10A680005FAF289788E5829DF001839DF00D11242E
:10A69000EB5FFA4F28968CAD9DADAEADBFAD289760
:10A6A000858F968FA78FB0A3C501B4010F94013099
:10A6B0002091F1043091F2044091F3045091F4049C
:10A6C0000F9460306BA77CA78DA79EA7698B7A8BB0
:10A6D0008B8B9C8BC301B2010F9401302091F50448
:10A6E0003091F6044091F7045091F8040F946030D3
:10A6F0006FA778AB89AB9AAB6D8B7E8B8F8B988F66
:10A700002091F9043091FA044091FB045091FC042B
:10A7100066962CAF3DAF4EAF5FAF66976BA17CA145
:10A720008DA19EA10F94013066962CAD3DAD4EAD2E
:10A730005FAD66970F9460304B015C01698F7A8F33
:10A740008B8F9C8F2091FD043091FE044091FF047B
:10A7500050910005C701B6010F9460306B017C0178
:10A760006D8F7E8F8F8F98A324968CAD9DADAEADEF
:10A77000BFAD24970697A105B1057CF562962CAD77
:10A780003DAD4EAD5FAD62972630310541055105B7
:10A7900024F528968CAD9DADAEADBFAD289706973C
:10A7A000A105B105D4F420E030E0A901C701B6014C
:10A7B0000F948B3687FF04C0F7FAF094F7F8F09403
:10A7C00088E5829DF001839DF00D1124EB5FFA4F27
:10A7D000C586D686E786F08AA1C16C96AEADBFADC0
:10A7E0006C97CD90DD90ED90FC9020E030E0A901D9
:10A7F000C701B6010F94FB2F882369F088E5829D7D
:10A80000F001839DF00D1124EB5FFA4FC586D686CB
:10A81000E786F08A34C02BA53CA54DA55EA5CA01EC
:10A82000B9010F9460306B017C012FA538A949A9AB
:10A830005AA9CA01B9010F9460309B01AC01C7014C
:10A84000B6010F9465346B017C01A5019401C5012B
:10A85000B4010F9460309B01AC01C701B6010F94A5
:10A8600065340F94D03628E5229DF001239DF00D2C
:10A870001124EB5FFA4F658776878787908B8091ED
:10A880002215882309F44AC1C090F103D090F20345
:10A89000E090F303F090F40320E030E0A901C70159
:10A8A000B6010F94FB2F882309F438C18090ED0383
:10A8B0009090EE03A090EF03B090F00320E030E022
:10A8C000A901C501B4010F94FB2F882309F426C107
:10A8D0002BA13CA14DA15EA12115310541055105DA
:10A8E00009F41CC157FD0BC080E090E0A0E8BFE375
:10A8F00024968CAF9DAFAEAFBFAF24970AC020E0C7
:10A9000030E040E85FEB24962CAF3DAF4EAF5FAF39
:10A91000249712FB112710F98091EC038117B1F1F4
:10A920001093EC036091E8037091E9038091EA03CE
:10A930009091EB030F9401302B013C01A501940190
:10A9400024966CAD7DAD8EAD9FAD24970F94603095
:10A95000A70196010F94603020914F123091501250
:10A9600040915112509152120F9460309B01AC01F2
:10A97000C301B2010F9465340F94A9356093E803C5
:10A980007093E9038093EA039093EB034090E8030C
:10A990005090E9036090EA037090EB038BA19CA1B7
:10A9A000ADA1BEA1181619061A061B0634F414141C
:10A9B0001504160417041CF0B1C077FEAFC0C30124
:10A9C000B2010F9401304B015C0188E5829DF001DA
:10A9D000839DF00D1124EB5FFA4F2091020230911C
:10A9E00003024091040250910502658576858785B2
:10A9F00090890F9441356B017C0120E030E040E804
:10AA00005FE30F948B36181634F4C12CD12C30E848
:10AA1000E32E3FE3F32EA7019601C501B4010F9485
:10AA200060300F94A9356B017C01DC01CB01F7FE8E
:10AA300007C088279927DC018C199D09AE09BF0939
:10AA400028960CAD1DAD2EAD3FAD2897080F191FF0
:10AA50002A1F3B1FC901B80128E5229D8001239DC3
:10AA6000100D11240B5F1A4FD8015D966D937D93E5
:10AA70008D939C9390974C185D086E087F084092C8
:10AA8000E8035092E9036092EA037092EB030F949B
:10AA9000FF2F9B01AC0124966CAD7DAD8EAD9FADBB
:10AAA00024970F94603066962CAD3DAD4EAD5FADF2
:10AAB00066970F9460306B017C01698F7A8F8B8F62
:10AAC0009C8F2BA53CA54DA55EA5CA01B9010F948D
:10AAD00060304B015C012FA538A949A95AA9CA01C8
:10AAE000B9010F9460309B01AC01C501B4010F9412
:10AAF00065344B015C01A7019601C701B6010F94B3
:10AB000060309B01AC01C501B4010F9465340F9412
:10AB1000D036F801658776878787908B88E5829D98
:10AB2000F001839DF00D1124EB5FFA4F0CA91DA9D4
:10AB30002EA93FA901A312A323A334A345895689B3
:10AB40006789708D058D168D278D30A1818D928D31
:10AB5000A38DB48D80179107A207B30710F4D90114
:10AB6000C80184179507A607B70710F4DB01CA01CF
:10AB70000CA91DA92EA93FA980179107A207B30709
:10AB800010F4D901C80128E5229DF001239DF00DA4
:10AB90001124EB5FFA4F85A396A3A7A3B0A706974E
:10ABA000A105B10508F435C4DF01AE5ABF4F80914D
:10ABB0000B0E90910C0E8D939C9329961FAD2997A7
:10ABC00011A7452B462B472B09F0179888E5829D46
:10ABD000F001839DF00D1124EB5FFA4F818D928D72
:10ABE000A38DB48D892B8A2B8B2B09F0169888E5C1
:10ABF000829DF001839DF00D1124EB5FFA4F858D4E
:10AC0000968DA78DB0A1892B8A2B8B2B09F01598D7
:10AC10002CA93DA94EA95FA9232B242B252B09F490
:10AC200001C48091F903882319F081508093F903BE
:10AC300029960FAD2997011104C0149880E28093E2
:10AC4000F903E0903715F0903815009139151091FF
:10AC50003A159701A8016BA978AD8CAD2D969FADE3
:10AC60002D970F94FB2F87FF06C0EBAAF8AE0CAF11
:10AC70002D961FAF2D9788E5829DF001839DF00DE5
:10AC80001124EB5FFA4F258536854785508960E0B2
:10AC900070E080E89FE30F94413524966CAF7DAF60
:10ACA0008EAF9FAF24979B01AC016BA978AD8CADA3
:10ACB0002D969FAD2D970F9460304B015C018091D4
:10ACC000830E9091810E891B8F7025968FAF2597EB
:10ACD000A501940160E074E284E799E40F944135A2
:10ACE0000F9496366B017C0125968FAD2597825087
:10ACF000863008F4A0C380916F0081FB222720F9E1
:10AD000081FF05C080916F008D7F80936F008091DF
:10AD1000010590910205A0910305B0910405C80EAC
:10AD2000D91EEA1EFB1EC0920105D0920205E092D8
:10AD30000305F0920405222329F080916F008260C0
:10AD400080936F0088E5829D8001839D100D112402
:10AD50000B5F1A4FD8011D962D913D914D915C913D
:10AD60005097C501B4010F9460309B01AC010F9462
:10AD7000603062966CAF7DAF8EAF9FAF6297F80187
:10AD8000618372838383948325A136A147A150A553
:10AD900028AF39AF4AAF5BAFCA01B9010F94FF2F9B
:10ADA0006CAF7DAF8EAF9FAFA50194010F94603063
:10ADB0000F942B350F94AE3566966CAF7DAF8EAF8A
:10ADC0009FAF6697F801EE5BFF4F608371838283CC
:10ADD00093838E010F5E1F4F2A961FAF0EAF2A97E7
:10ADE000005111092E961FAF0EAF2E970BE515E1FE
:10ADF000A2961FAF0EAFA2978E010F5D1F4F1AA331
:10AE000009A32E960EAD1FAD2E976C961FAF0EAFF9
:10AE10006C971BA21BA610E81FA70FE30BAB2A968B
:10AE2000AEADBFAD2A976D917D918D919D912A9682
:10AE3000BFAFAEAF2A97A50194010F9460306B01AC
:10AE40007C016C96EEADFFAD6C976193719381932D
:10AE500091936C96FFAFEEAF6C9720E030E0A901C4
:10AE60000F948B3687FF04C0F7FAF094F7F8F0944C
:10AE7000A296AEADBFADA2974D905D906D907D90C6
:10AE8000A296BFAFAEAFA297A3019201C701B601D0
:10AE90000F948B3618160CF40AC32A960EAD1FAD0C
:10AEA0002A9729A13AA10217130709F0B8CF20E089
:10AEB00030E040E85FE36BA17BA58FA59BA90F94D1
:10AEC000FB2F87FF57C07E0131E1E30EF11C2E9668
:10AED0000EAD1FAD2E972BA13BA54FA55BA9D801A9
:10AEE0006D917D918D919C910F946030F8016193EB
:10AEF0007193819391938F01EE15FF0561F728E51A
:10AF0000229DC001239D900D11248C010B5F1A4FCF
:10AF100078010E5B1F4F66966CAD7DAD8EAD9FAD1B
:10AF200066970F94FF2F2BA13BA54FA55BA90F940C
:10AF300060300F94AE35D8016D937D938D939C93C3
:10AF400013972BA13BA54FA55BA96BA17BA58FA553
:10AF50009BA90F9460309B01AC0162966CAD7DADF6
:10AF60008EAD9FAD62970F946030F701618372835D
:10AF70008383948324962CAD3DAD4EAD5FAD249775
:10AF80006CAD7DAD8EAD9FAD0F9460306BA37CA397
:10AF90008DA39EA388E5829D8001839D100D1124C1
:10AFA0000B5F1A4FD80155968D909D90AD90BC9037
:10AFB000589781149104A104B10409F090C25996E4
:10AFC0008D919D910D90BC91A02D892B8A2B8B2B5F
:10AFD00009F085C2F801858D968DA78DB0A1892BCA
:10AFE0008A2B8B2B09F07BC220914315309144159D
:10AFF00040914515509146156BA17CA18DA19EA154
:10B000000F9460300F942B350F94AE352B013C011B
:10B01000D801D7961C9288E5829D8001839D100DF2
:10B0200011240B5F1A4FF801E25BFF4F40825182FF
:10B0300062827382C301B2010F94FF2F6B017C0106
:10B040002BA13CA14DA15EA10F9441352C966CAF74
:10B050007DAF8EAF9FAF2C97D80151966D937D93A6
:10B060008D939C9354972DEB37E346E051E4C70151
:10B07000B6010F9460300F94AE35F80162AB73AB3C
:10B0800084AB95AB87A9882381F1FE96208131811D
:10B09000428153816091FA147091FB148091FC14E9
:10B0A0009091FD140F9460302C962CAD3DAD4EADBB
:10B0B0005FAD2C970F946030209153123091541251
:10B0C00040915512509156120F9460309B01AC0183
:10B0D00060E074E284EF99E40F9441350F94AE354B
:10B0E000D801D9967C936E93D89788E5829DF0011C
:10B0F000839DF00D1124EB5FFA4F018112812381B2
:10B10000348124960CAF1DAF2EAF3FAF2497C901F9
:10B11000B8010F94D036162F072F8BA39FA323E2DD
:10B1200035E160963FAF2EAF60973E0131E1630E8F
:10B13000711C43E255E15DAF4CAF2E964EAC5FAC57
:10B140002E976BA77FA78BAB9CAB18AED201CD908F
:10B15000DD90ED90FD902D0120E030E0A901C701C8
:10B16000B6010F948B3687FF04C0F7FAF094F7F816
:10B17000F094ECADFDAD81909190A190B190FDAFB8
:10B18000ECAFA5019401C701B6010F948B361816D8
:10B190000CF4B2C446145704C9F65BA56B965FAFB6
:10B1A0006B978FA5A1968FAFA1979BA9EC969FAFA8
:10B1B000EC97ACA9ED96AFAFED972596BFAD25976F
:10B1C000B111DAC46B968FAD6B97A1969FADA19725
:10B1D000EC96AFADEC97ED96BFADED978093F50390
:10B1E0009093F603A093F703B093F80388E5829D4C
:10B1F0008001839D100D11240B5F1A4F2BA53FA5D5
:10B200004BA95CA96BA57FA58BA99CA90F94603065
:10B21000D80119966D937D938D939C931C972C96D2
:10B220006CAD7DAD8EAD9FAD2C9790589B01AC0160
:10B230000F946534F80125853685478550890F942C
:10B2400060309B01AC016BE077ED83E29BE30F94F0
:10B2500064349B01AC018BE097EDA3E2BBE3F80102
:10B2600085839683A783B087108124966CAD7DADCE
:10B270008EAD9FAD24970F94FB2F18160CF0BCC514
:10B2800081E0182B88E5829DF001839DF00D11244B
:10B29000EB5FFA4F108380E1FE013196ADEABEE02C
:10B2A00001900D928A95E1F724960CAD1DAD2EAD5F
:10B2B0003FAD24970093A90E1093AA0E2093AB0ED6
:10B2C0003093AC0EE2962CAD3DAD4EAD5FADE29746
:10B2D0002093CD0E3093CE0E4093CF0E5093D00ED0
:10B2E000E6968CAD9DADAEADBFADE6978093D10E29
:10B2F0009093D20EA093D30EB093D40EEA960CADD9
:10B300001DAD2EAD3FADEA970093D50E1093D60E2E
:10B310002093D70E3093D80EA0962CAD3DAD4EADF8
:10B320005FADA0972093D90E3093DA0E4093DB0ED9
:10B330005093DC0EA6968CAD9DADAEADBFADA6977D
:10B340008093BD0E9093BE0EA093BF0EB093C00E1F
:10B35000AA960CAD1DAD2EAD3FADAA970093C10EC0
:10B360001093C20E2093C30E3093C40EAE962CAD34
:10B370003DAD4EAD5FADAE972093C50E3093C60E7A
:10B380004093C70E5093C80E6A968CAD9DADAEAD7E
:10B39000BFAD6A978093C90E9093CA0EA093CB0E4F
:10B3A000B093CC0E9091830E8091840E981303C0BD
:10B3B00084E68093800EEB968FADEB978F5F8F7056
:10B3C0008093830E8091830E9091820E81508F70B6
:10B3D000891314C50091840E0BA31091830E1FA333
:10B3E00098E50FA11BA1011392C5812C912CA12CD2
:10B3F000B12C1BA61FA61BAA1CAA212C312C00E0D5
:10B4000010E0FBA12FA1F2138FC52114310409F024
:10B4100040C680916F00826080936F0081E09EC77C
:10B4200080E09CC7E0903315F090341500913515FD
:10B43000109136150ECC80913B1590913C15A09142
:10B440003D15B0913E15C816D906EA06FB0608F070
:10B4500052CC8C199D09AE09BF09BC01CD01660F04
:10B46000771F881F991F25964FAD2597042F10E051
:10B4700020E030E0A90198010F940734CA01B90116
:10B480000F94FF2F0F949636C60ED71EE81EF91E96
:10B49000C701B6010F94FF2F9B01AC0160E074E27D
:10B4A00084E799E40F9441354B015C0124CCA7015A
:10B4B0009601C301B2010F9441357B018C019B01C0
:10B4C000AC016BA17BA58FA59BA90F948B36181699
:10B4D0000CF0E3CCEBA2FBA60FA71BABDECC0CA9B8
:10B4E0001DA92EA93FA9012B022B032B49F0609126
:10B4F0004715709148158091491590914A1508C0DB
:10B5000060913F15709140158091411590914215C1
:10B510002BA13CA14DA15EA10F9460300F942B355F
:10B520000F94AE352B013C012CA93DA94EA95FA972
:10B53000232B242B252BC9F020E030E0A9016091BA
:10B54000FA147091FB148091FC149091FD140F94E7
:10B55000FB2F882351F081E00FA118A529A53AA55A
:10B5600010161106120613060CF080E098E5929D65
:10B570008001939D100D11240B5F1A4FD801D796AF
:10B580008C93882309F4BAC02091BD0E3091BE0E71
:10B590004091BF0E5091C00EA6966CAD7DAD8EADA4
:10B5A0009FADA6970F9464346FA378A789A79AA735
:10B5B0002091C10E3091C20E4091C30E5091C40E25
:10B5C000AA966CAD7DAD8EAD9FADAA970F946434F5
:10B5D0006BA77CA78DA79EA72091C50E3091C60EA4
:10B5E0004091C70E5091C80EAE966CAD7DAD8EAD3C
:10B5F0009FADAE970F9464346B017C012FA138A5E9
:10B6000049A55AA5CA01B9010F9460306FA378A764
:10B6100089A79AA72BA53CA54DA55EA5CA01B9018E
:10B620000F9460309B01AC016FA178A589A59AA504
:10B630000F9465346FA378A789A79AA7A7019601ED
:10B64000C701B6010F9460309B01AC016FA178A5D2
:10B6500089A59AA50F9465340F94D0366B017C01AF
:10B660002091C90E3091CA0E4091CB0E5091CC0E54
:10B670006A966CAD7DAD8EAD9FAD6A970F946434C4
:10B68000A70196010F9441356B017C01F801FE96EC
:10B69000608371838283938320E030E040E450E450
:10B6A0000F948B3618161CF4F80117AA27C02091A6
:10B6B000FA143091FB144091FC145091FD14C70111
:10B6C000B6010F9460309B01AC0160912F15709111
:10B6D000301580913115909132150F9441352BA181
:10B6E0003CA14DA15EA10F9460300F94AE3564155E
:10B6F00075058605970510F42B013C018091DD044A
:10B700009091DE04A091DF04B091E00408AD19AD82
:10B710002AAD3BAD80179107A207B30708F4DCC040
:10B7200081149104A104B10441F12091E10430910C
:10B73000E2044091E3045091E404241535054605E4
:10B740005705D8F468AD79AD8AAD9BAD0F94F83349
:10B750006B017C01A3019201C501B4010F94F83380
:10B76000C616D706E806F90640F4C701B601A501DA
:10B7700094010F94073429013A0188E5829DF00174
:10B78000839DF00D1124EB5FFA4FC18CD28CE38CBA
:10B79000F48CC114D104E104F10441F12091E504D9
:10B7A0003091E6044091E7045091E80424153505F2
:10B7B00046055705D8F468AD79AD8AAD9BAD0F94B9
:10B7C000F8334B015C01A3019201C701B6010F944C
:10B7D000F83386169706A806B90640F4C501B401E9
:10B7E000A70196010F94073429013A0188E5829D4B
:10B7F000F001839DF00D1124EB5FFA4FC58CD68CC0
:10B80000E78CF0A0C114D104E104F10441F12091CE
:10B81000E9043091EA044091EB045091EC042415C2
:10B82000350546055705D8F468AD79AD8AAD9BADB1
:10B830000F94F8334B015C01A3019201C701B601DB
:10B840000F94F83386169706A806B90640F4C5018A
:10B85000B401A70196010F94073429013A0188E544
:10B86000829DF001839DF00D1124EB5FFA4FC1A082
:10B87000D2A0E3A0F4A0C114D104E104F10409F4BE
:10B88000CACB2091ED043091EE044091EF04509129
:10B89000F004241535054605570508F0BCCB68AD06
:10B8A00079AD8AAD9BAD0F94F8334B015C01A301D8
:10B8B0009201C701B6010F94F83386169706A806C1
:10B8C000B90608F0A8CBC501B401A70196010F94F1
:10B8D000073429013A019FCB81149104A104B104DA
:10B8E000A9F16091E1047091E2048091E3049091E8
:10B8F000E404641575058605970540F50F94FF2F40
:10B900002CAD3DAD4EAD5FAD0F9460306B017C0151
:10B91000C501B4010F94FF2F4B015C01C301B201BB
:10B920000F94FF2FA50194010F946030A701960199
:10B930000F948B36181654F4A5019401C701B60173
:10B940000F9441350F94AE352B013C0188E5829D63
:10B95000F001839DF00D1124EB5FFA4F818C928CE6
:10B96000A38CB48C81149104A104B104A9F1609159
:10B97000E5047091E6048091E7049091E804641571
:10B9800075058605970540F50F94FF2F2CAD3DAD4D
:10B990004EAD5FAD0F9460306B017C01C501B40109
:10B9A0000F94FF2F4B015C01C301B2010F94FF2FD5
:10B9B000A50194010F946030A70196010F948B3676
:10B9C000181654F4A5019401C701B6010F9441352E
:10B9D0000F94AE352B013C0188E5829DF001839DDB
:10B9E000F00D1124EB5FFA4F858C968CA78CB0A0DC
:10B9F00081149104A104B104A9F16091E90470914A
:10BA0000EA048091EB049091EC04641575058605B9
:10BA1000970540F50F94FF2F2CAD3DAD4EAD5FADBA
:10BA20000F9460306B017C01C501B4010F94FF2FAE
:10BA30004B015C01C301B2010F94FF2FA5019401DA
:10BA40000F946030A70196010F948B36181654F4AA
:10BA5000A5019401C701B6010F9441350F94AE358D
:10BA60002B013C0188E5829DF001839DF00D11249E
:10BA7000EB5FFA4FC1A0D2A0E3A0F4A0C114D1049F
:10BA8000E104F10409F4C7CA6091ED047091EE0479
:10BA90008091EF049091F004641575058605970573
:10BAA00008F0B9CA0F94FF2F2CAD3DAD4EAD5FAD80
:10BAB0000F9460304B015C01C701B6010F94FF2F5A
:10BAC0006B017C01C301B2010F94FF2FA701960106
:10BAD0000F946030A50194010F948B3618160CF06A
:10BAE0009ACAA7019601C501B4010F9441350F947C
:10BAF000AE352B013C018FCAF8ADFF2329F1A5011A
:10BB00009401612F702F8BA19FA10F9460304B0186
:10BB10005C012BA53FA54BA95CA9C701B6010F94F9
:10BB20006030A50194010F948B36181614F5A70107
:10BB30009601C501B4010F9441356BA77FA78BAB6C
:10BB40009CAB21E028AF26CBA7019601C501B4012B
:10BB50000F9441359B01AC016BA57FA58BA99CA9D6
:10BB60000F9460306BA77FA78BAB9CAB31E038AFF5
:10BB700011CB41E048AF0ECBC090A90ED090AA0ED9
:10BB8000E090AB0EF090AC0E2DEB37E346E855E3BA
:10BB9000C701B6010F94FB2F87FD14CBC701B60177
:10BBA0000F94D0366B017C019B01AC01612F702F8B
:10BBB0008BA19FA10F94FB2F87FD04C01C2D0D2D81
:10BBC000EBA2FFA29601A701612F702F8BA19FA16D
:10BBD0000F94413566966CAF7DAF8EAF9FAF669781
:10BBE000EDEAFEE02696FFAFEEAF269720E030E0CC
:10BBF00040E85FE328AF39AF4AAF5BAF1CAE269693
:10BC0000AEADBFAD26976D917D918D919D9126969C
:10BC1000BFAFAEAF269766962CAD3DAD4EAD5FADD6
:10BC200066970F9460306B017C012E96EEADFFADF0
:10BC30002E9781909190A190B1902E96FFAFEEAF8C
:10BC40002E97FCADFF2391F028AD39AD4AAD5BAD29
:10BC50000F9460306B017C0128AD39AD4AAD5BAD0E
:10BC6000C501B4010F9460304B015C01A501940142
:10BC7000C701B6010F948B3620E030E0A9011816F9
:10BC80002CF5C501B4010F948B3618164CF020E04A
:10BC900030E0A901C701B6010F94FB2F87FF05C053
:10BCA000A5019401C701B60124C02401350177FA2A
:10BCB000709477F87094A3019201C701B6010F94B4
:10BCC0008B3618165CF52601370128C0C501B40172
:10BCD0000F94FB2F87FD09C020E030E0A901C701C8
:10BCE000B6010F948B3618164CF4A7019601C501C6
:10BCF000B4010F9464342B013C0110C026013701BC
:10BD000077FA709477F87094A5019401C301B20199
:10BD10000F948B36181614F0240135016096AEADE1
:10BD2000BFAD6097CD90DD90ED90FD906096BFAF78
:10BD3000AEAF6097A7019601C301B2010F948B3695
:10BD40001816ACF4A3019201C701B6010F94413556
:10BD50009B01AC0168AD79AD8AAD9BAD0F946030AD
:10BD600068AF79AF8AAF9BAFBCADBF5FBCAF269663
:10BD7000EEADFFAD2697ED5BFE4009F040CF3CAD48
:10BD8000332371F028AD39AD4AAD5BAD612F702F13
:10BD90008BA19FA10F946030162F072F8BA39FA319
:10BDA00024EA30E74DE75FE3612F702F8BA19FA15D
:10BDB0000F9460306B017C019B01AC016091F50335
:10BDC0007091F6038091F7039091F8030F948B36EE
:10BDD00018165CF4A70196016BA57FA58BA99CA9F9
:10BDE0000F948B3618160CF4EDC91BA70FA70BA1E7
:10BDF0000BAB1FA11CABE6C983E043CAF090830ED6
:10BE00008FEF8F0D8F708BA3B090820E8091830E79
:10BE1000B81206C00091820E0BA3C12CD12C69C0B0
:10BE2000C12CD12C1BA11B15A9F31BA1812E912C78
:10BE300028E5289D8001299D100D11240B5F1A4FC4
:10BE4000D8018C9183FD27C00BAB1CAB01151105EC
:10BE500021F11996BC91BFA3F801F285FBA7D80187
:10BE60001B96BC91BFA7F801A484458056806780CB
:10BE700070842FA13BA54B2F5A2DC301B2010F9403
:10BE8000FB2F81117FC1C114D10439F0D6018C91EF
:10BE900080FD78C102C0CBAADCAA8BA181508F7033
:10BEA0008BA38091820EB81649F00BA10B1509F4F3
:10BEB000B1CF81E08B0D8F70B82EF3CFCBA8DCA86B
:10BEC000B1CF0BA1802E912C28E5289D8001299DC2
:10BED000100D11240B5F1A4FD8018C9183FD15C0F2
:10BEE0005801C114D10459F48BA18F5F8F708BA3BB
:10BEF00065018091830E1BA11813E3CF6BCAC601A5
:10BF00000E94CD848111F0CFB3C15601EDCF8FA136
:10BF100081508F70989FF0011124EB5FFA4F2081C0
:10BF200023FF63CA8FA35DCA28E53BA1239FC001FD
:10BF30001124AC014B5F5A4F1A01DA018C9183FD39
:10BF400019C015966D917D918D919C9118970F94C4
:10BF5000D036F62EE72ED82EC92E0115110509F47C
:10BF60008AC0F801808180FD0AC0D1018C9180FDDA
:10BF700006C081C0FBA4EFA4DBA8CCA881C0F80157
:10BF8000808181608083C8010E94CD8481116FC04F
:10BF9000F80161817281838194810F94D0362B01E5
:10BFA0003C019B01AC0160E070E080E89FE30F94EE
:10BFB00041354B015C019B01AC016F2D7E2D8D2D18
:10BFC0009C2D0F94603069837A838B839C83A501B9
:10BFD00094016BA57FA58BA99CA90F946030698BF8
:10BFE0007A8B8B8B9C8BAE014F5F5F4FBE016F5E78
:10BFF0007F4FC8010E94E870D801D7968C918823A2
:10C00000B1F12091FA143091FB144091FC1450913D
:10C01000FD14F801FE9660817181828193810F94F5
:10C02000603020915312309154124091551250912A
:10C0300056120F9460304B015C019B01AC01C301AF
:10C04000B2010F9460300F94AE35F80173AF62AF58
:10C05000A50194016F2D7E2D8D2D9C2D0F946030A8
:10C060000F94AE35D801DD967C936E93DC97F80182
:10C0700080818E7F80838F2C9E2CAD2CBC2C8101E7
:10C080008BA18F5F8F708BA3FBA6EFA6DBAACCAA38
:10C09000B8C9D1018C9181608C93C8010E94CD8474
:10C0A00081116BC0F10161817281838194810F9450
:10C0B000D0366B017C019B01AC0160E070E080E850
:10C0C0009FE30F9441352B013C012DEC3CEC4CE4FB
:10C0D0005DE30F94603069837A838B839C83A30133
:10C0E0009201B401C5010F946030698B7A8B8B8B00
:10C0F0009C8BAE014F5F5F4FBE016F5E7F4FC101F2
:10C100000E94E870D101D7968C918823B1F12091DB
:10C11000FA143091FB144091FC145091FD14F1017C
:10C12000FE9660817181828193810F9460302091AD
:10C1300053123091541240915512509156120F944F
:10C1400060304B015C019B01AC01C701B6010F944B
:10C1500060300F94AE35F10173AF62AF2DEC3CEC63
:10C160004CE45DE3C501B4010F9460300F94AE352B
:10C17000D101DD967C936E93DC97F10180818E7FF7
:10C18000808347C928E5289DF001299DF00D1124E1
:10C19000EB5FFA4F808181FD3FC0C114D10431F0C3
:10C1A000F601C580D680E780F08408C08BE0C82EF9
:10C1B00087EDD82E83E2E82E8BE3F82E28E5289D24
:10C1C000F001299DF00D1124EB5FFA4F81899289CE
:10C1D000A389B489BC01CD0190589B01AC010F9497
:10C1E0006534D8011D962D913D914D915C915097EC
:10C1F0000F9460309B01AC01C701B6010F94643409
:10C200001B016C019B01AC016FA17BA58FA59A2D31
:10C210000F94FB2F87FF04C02FA03BA4CFA4DA2CE0
:10C220009101A601C301B2010F94FB2F882309F4E9
:10C2300034CEB8E5B89DC001B99D900D1124FC0124
:10C24000EB5FFA4F4F01808181608083C8010E94BB
:10C25000CD84882329F0D4018C918E7F8C931DCEC0
:10C26000C101D601F40185839683A783B08715CEDB
:10C27000D6018C9181FD50C0D60115962D913D912E
:10C280004D915C9118972FA338A749A75AA715017C
:10C29000B5E02B0E311CF801458056806780708414
:10C2A000A30192016FA178A589A59AA50F94FB2FF0
:10C2B00087FF32C0F60181899289A389B489BC01C4
:10C2C000CD0190589B01AC010F946534D6011D96A9
:10C2D0002D913D914D915C9150970F9460309B0151
:10C2E000AC016FA178A589A59AA50F9464346B0160
:10C2F0007C01A30192010F94FB2F87FF0DC0D80191
:10C300008C9181608C93C5010E94CD848823E1F0DB
:10C31000F80180818E7F808318E5189DF001199DBA
:10C32000F00D1124EB5FFA4F21853285438554854A
:10C3300065817681878190850F94FB2F8111D4CD03
:10C340000BA10093820ED0CDD101CD92DD92ED9262
:10C35000FC9213970BA10093820EDECFC458DF4FDF
:10C360000FB6F894DEBF0FBECDBFDF91CF911F9106
:10C370000F91FF90EF90DF90CF90BF90AF909F9084
:10C380008F907F906F905F904F903F902F90089587
:10C390008091830E9091840E891B8F708F3021F4D1
:10C3A00080E00F94BB1EF4CF8091830E8F5F8F705F
:10C3B000E091830E98E59E9FF0011124EB5FFA4F08
:10C3C000DF011D929A95E9F798E090834091CD0E98
:10C3D0005091CE0E6091CF0E7091D00E458B568B42
:10C3E000678B708F4091D10E5091D20E6091D30E19
:10C3F0007091D40E418F528F638F748F4091D50E00
:10C400005091D60E6091D70E7091D80E458F568FF1
:10C41000678F70A34091D90E5091DA0E6091DB0EB8
:10C420007091DC0E41A352A363A374A32091830EE9
:10C430009091840E291303C094E69093800E80930C
:10C44000830E80916F00826080936F0008959091B9
:10C45000830E8091840E981721F080E00F94BB1E0C
:10C46000F6CF8091FA039091FB03892BB1F70895E1
:10C470009091830E8091840E981721F080E00F94A4
:10C48000BB1EF6CF8091FA039091FB03892BB1F785
:10C490000D947D21CF93DF9390916F0091FB222724
:10C4A00020F991FF05C090916F009D7F90936F00E0
:10C4B00094E0899FE0011124FE01E452F54F608170
:10C4C000718182819381222329F020916F00226063
:10C4D00020936F000F940130CF50DB4F28813981BA
:10C4E0004A815B810F946030DF91CF9108952F9244
:10C4F0003F924F925F926F927F928F929F92AF92F4
:10C50000BF92CF92DF92EF92FF920F931F93CF9340
:10C51000DF93CDB7DEB7E8970FB6F894DEBF0FBE56
:10C52000CDBF20912215222309F4E6C01C01009101
:10C53000890E10918A0E20918B0E30918C0E4090B6
:10C540008D0E50908E0E60908F0E7090900E4DA6B6
:10C550005EA66FA678AA8090910E9090920EA09001
:10C56000930EB090940E4091950E5091960E60915E
:10C57000970E7091980E8091990E90919A0EA091BD
:10C580009B0EB0919C0E89AB9AABABABBCABC09091
:10C590009D0ED0909E0EE0909F0EF090A00E809188
:10C5A000A10E9091A20EA091A30EB091A40E409066
:10C5B000A50E5090A60E6090A70E7090A80E4DAAE2
:10C5C0005EAA6FAA78AE4090850E5090860E60905D
:10C5D000870E7090880E49825A826B827C828D828F
:10C5E0009E82AF82B886C986DA86EB86FC860D8786
:10C5F0001E872F87388B498B5A8B6B8B7C8B8D8B4F
:10C600009E8BAF8BB88F8DA59EA5AFA5B8A9898F3E
:10C610009A8FAB8FBC8F49A85AA86BA87CA84D8E67
:10C620005E8E6F8E78A28DA99EA9AFA9B8AD89A3A1
:10C630009AA3ABA3BCA320E030E040E450E4D101D6
:10C640006D917D918D919C910F94653469A77AA726
:10C650008BA79CA720E030E04EE353E4F101648116
:10C660007581868197810F9464346DA37EA38FA317
:10C6700098A7C10108969F938F93CE0185969F93AB
:10C680008F9304969F938F938DB79EB784970FB621
:10C69000F8949EBF0FBE8DBFADB7BEB7119684E2B2
:10C6A000FE01319601900D928A95E1F70E94CAFE33
:10C6B00020E030E040E450E469A57AA58BA59CA574
:10C6C0000F946434D1016D937D938D939C93139754
:10C6D00020E030E04EE353E46DA17EA18FA198A548
:10C6E0000F946534F10164837583868397830FB655
:10C6F000F894DEBF0FBECDBFE8960FB6F894DEBF4C
:10C700000FBECDBFDF91CF911F910F91FF90EF90A2
:10C71000DF90CF90BF90AF909F908F907F906F9061
:10C720005F904F903F902F9008959091260CE92FA5
:10C73000F0E0EF5DF34F80839F5F953018F49093A6
:10C74000260C02C01092260C80910A0E8F5F8093F7
:10C750000A0E0895CF92DF92EF920F931F93CF931B
:10C76000DF93CDB7DEB760970FB6F894DEBF0FBE8C
:10C77000CDBFE0905816E3E2F2E180859185A28575
:10C78000B385448155816681778100811181228141
:10C79000338109831A832B833C834D835E836F83AC
:10C7A000788789879A87AB87BC871D861E861F86F8
:10C7B000188AAE01475F5F4FBE016B5F7F4FCE01AE
:10C7C00001960E94FD6FCE010D966C0100E712E00C
:10C7D0002FE232E1AE01475F5F4FBE016B5F7F4FDB
:10C7E0000C970E947A5060960FB6F894DEBF0FBE89
:10C7F000CDBFDF91CF911F910F91EF90DF90CF9040
:10C8000008954F925F926F927F928F929F92AF9214
:10C81000BF92CF92DF92EF92FF920F931F93CF932D
:10C82000DF93CDB7DEB72C970FB6F894DEBF0FBEFF
:10C83000CDBF6D837E838F83988729873A874B8707
:10C840005C87470158013601809170029091710216
:10C85000A0917202B091730289839A83AB83BC83E7
:10C86000D601CD90DD90ED90FC9020E030E0A90164
:10C87000C701B6010F94FB2F811106C0E1E5FAE470
:10C88000C590D590E590F490A501940160912B128C
:10C8900070912C1280912D1290912E120F94FB2FDB
:10C8A00087FF11C0C0927002D0927102E0927202B2
:10C8B000F092730280922B1290922C12A0922D1261
:10C8C000B0922E1247DFF301408051806280738066
:10C8D00020E030E0A901C301B2010F94FB2F8111C8
:10C8E00008C040906C0250906D0260906E02709093
:10C8F0006F024092700250927102609272027092C6
:10C9000073028D819E81AF81B885809323129093AD
:10C910002412A0932512B093261289859A85AB859F
:10C92000BC858093271290932812A0932912B0936C
:10C930002A1210DFA501940160912B1270912C1224
:10C9400080912D1290912E120F948B3618168CF424
:10C95000C0927002D0927102E0927202F092730261
:10C9600080922B1290922C12A0922D12B0922E1225
:10C97000F1DE6DDD89819A81AB81BC81809370028B
:10C9800090937102A0937202B09373022C960FB62B
:10C99000F894DEBF0FBECDBFDF91CF911F910F91F5
:10C9A000FF90EF90DF90CF90BF90AF909F908F90CF
:10C9B0007F906F905F904F900895CF93FC0180819E
:10C9C0008B33A1F080910A0E853080F4C62FBF0111
:10C9D0008091260C20E6829FC0011124875D934F31
:10C9E0000F94A9378C2FA1DE81E001C080E0CF91A8
:10C9F0000895BF92CF92DF92EF92FF920F931F9311
:10CA0000CF93DF9300D01F92CDB7DEB79091140C77
:10CA1000981731F1B82E81110E9441E360912312E1
:10CA20007091241280912512909126122091271244
:10CA3000309128124091291250912A1219821A829B
:10CA40001B821C82E0902B12F0902C1200912D1270
:10CA500010912E12FE0131966F01D3DEB092140CAC
:10CA600080E00F900F900F900F90DF91CF911F916A
:10CA70000F91FF90EF90DF90CF90BF90089580913D
:10CA8000650490916604A0916704B0916804809356
:10CA9000700290937102A0937202B093730280911E
:10CAA00063049091640490930102809300020895BE
:10CAB0008091700290917102A0917202B091730204
:10CAC0008093650490936604A0936704B093680410
:10CAD000809100029091010290936404809363041A
:10CAE00084E690E090930102809300020895CF9233
:10CAF000DF92EF92FF920F931F936A01E0902B1247
:10CB0000F0902C1200912D1210912E12FB01208119
:10CB1000318142815381FC016081718182819381E5
:10CB200070DE1F910F91FF90EF90DF90CF900895EE
:10CB3000CF92DF92EF92FF920F931F936B01FC0154
:10CB4000E080F18002811381E3E2F2E1248135810A
:10CB500046815781608171818281938152DE1F916C
:10CB60000F91FF90EF90DF90CF9008950F931F9358
:10CB7000CF93DF9394E0899FE00111248E010F5938
:10CB8000194EFE01EB5EF34FDE01A155BB4E2D9118
:10CB90003D914D915C9160817181828193810F946F
:10CBA0006534F8016083718382839383FE01EE52C2
:10CBB000FC4E85919591A591B491FE01EE5EFD4FDD
:10CBC00080839183A283B383FE01E252FC4E859160
:10CBD0009591A591B491C95ADD4F88839983AA8311
:10CBE000BB83DF91CF911F910F910895CF93DF9376
:10CBF000EC0160E0CE01E1DE811104C080E00F9421
:10CC0000BB1EF7CFCE010F94DC048823B9F3DF916C
:10CC1000CF910895DF92EF92FF920F931F93CF93DE
:10CC2000DF93CDB7DEB76E970FB6F894DEBF0FBEB9
:10CC3000CDBF60915812709159126115710501F1C3
:10CC40004DE150E0CE0101967C010F946B2F1E8EBA
:10CC5000F7018F010E191F09D190DD2019F09AE01C
:10CC6000D912F7CFF701E00FF11F108260E0C70182
:10CC7000A4DE882329F0C7010F94DC04811109C0C8
:10CC800081E02091581230915912232BA1F480E0B9
:10CC900012C0DD2049F00F5F1F4F80915812909114
:10CCA0005912080F191F02C000E010E0109359122A
:10CCB00000935812E5CF6E960FB6F894DEBF0FBE04
:10CCC000CDBFDF91CF911F910F91FF90EF90DF903B
:10CCD00008954F925F926F927F929F92AF92BF9210
:10CCE000CF92DF92EF92FF920F931F93CF93DF9338
:10CCF0001F92CDB7DEB78EDF81114CC280910A0E34
:10CD0000853028F40F946A27AC0197FF39C18091D0
:10CD10002D0F882309F43EC280910A0E811102C0B2
:10CD200010926204EE24E3944091CD115091CE1103
:10CD30006091CF117091D0118091C9119091CA1159
:10CD4000A091CB11B091CC11481759076A077B0706
:10CD500008F4E12C00E010E0BB24B39480E6A82E98
:10CD600098E9C92E93E1D92E2DE8922E80910A0ED2
:10CD7000853008F00FC2E1100DC28091620481116C
:10CD800009C28091241190912511A0912611B09192
:10CD900027118093CD119093CE11A093CF11B09312
:10CDA000D01141E050E0BE016F5F7F4F8CE191E117
:10CDB0000E9455CD019719F4898190E002C08FEF50
:10CDC0009FEFF82EEE24E3944090CD115090CE11B9
:10CDD0006090CF117090D0114091C9115091CA113B
:10CDE0006091CB117091CC114416550666067706FA
:10CDF000C8F4E12C8F3FFFEF9F0709F46BC02AE0D6
:10CE0000821709F48CC08DE0F81609F488C093E20B
:10CE1000F91619F0EAE3FE1299C0809161048111BC
:10CE200095C072C014DB8CE191E10E947ED18091AB
:10CE30003711882359F1815080933711989EC00192
:10CE4000112441E061E0845C9E4E0E940CDCE09184
:10CE5000371124E0E29FF0011124E85CFE4E40818E
:10CE60005181628173814093CD115093CE116093B3
:10CE7000CF117093D0118CE191E10E943FCB809152
:10CE80002E0F8823B1F0B0922D0F13C010922D0FEA
:10CE9000EFDA0E9413940E946D936D337105810542
:10CEA000910528F0D0925912C0925812B3DE109218
:10CEB000E11480912D0F81112BC0EBEAF3E18491F5
:10CEC0003F019FEF691A790A8823F1F00F943F26FA
:10CED000F301F5CFE7E6F7E484913F012FEF621A03
:10CEE000720A882321F00F943F26F301F5CFECE975
:10CEF000F3E184913F019FEF691A790A882321F0B9
:10CF00000F943F26F301F5CFE3E2FE1208C005C0FF
:10CF100023E2F2123CC100E010E0B09262041092F1
:10CF200061040115110519F40E94A5770CC08091C8
:10CF3000260CA89E000D111D1124F801E75DF34F8A
:10CF4000108280E0F2DB00E010E010CF0F35110519
:10CF500008F00CCFFBE3FF1202C0B0926104809195
:10CF60006104811103CF8091260CF801A89EE00D89
:10CF7000F11D1124E75DF34FF0820F5F1F4FF6CED6
:10CF8000982F20917D1430917E148A3019F09D30B5
:10CF900009F0CBC0109260042115310519F40E94EC
:10CFA000A577ACCEF901E050FC4F108210927E14B0
:10CFB00010927D1420E034E08901F90180812F5F17
:10CFC0003F4F8032C9F378018E3409F07CC00115DF
:10CFD000110509F478C063E973E1C8010F947A2F51
:10CFE000DD24D394892B11F4D12C09C06EE470E0B8
:10CFF000C80104960F949E37009709F08C014AE00F
:10D0000050E060E070E0C80101960F94DB2C609363
:10D01000FC037093FD038093FE039093FF03009144
:10D020007F141091801420918114309182140F5F2D
:10D030001F4F2F4F3F4F601771078207930729F04B
:10D04000D11003C080E693E12AC06AE270E0C70114
:10D050000F94CD379C01009701F1982F9E1910E095
:10D06000992339F09150F701E90FF11D80811827BC
:10D07000F7CF4AE050E060E070E0C90101960F94FC
:10D08000DB2C012F10E020E030E0601771078207F1
:10D09000930741F081E493E102C087E193E10E94AC
:10D0A000BBDD35CE8091FC039091FD03A091FE0382
:10D0B000B091FF0380937F1490938014A093811408
:10D0C000B093821407C080912B0F882319F08CE64F
:10D0D00092E1E5CF80910A02811122C067E470E0FD
:10D0E000C7010F949E370097D9F04AE050E060E006
:10D0F00070E001960F94DB2C6430710588F4E0EA4F
:10D10000F2E184918F010F5F1F4F882321F00F946C
:10D110003F26F801F6CF60E086E992E10E94E1BB8C
:10D1200061E080E094E049DCE9CD2F3531050CF079
:10D13000E5CD9C35C1F40F946A2797FDDFCD209192
:10D1400060042111DBCD20917D1430917E14A90162
:10D150004F5F5F4F50937E1440937D14F901E05070
:10D16000FC4F8083CBCD9B3319F481E08093600426
:10D17000809160048111C2CDC901019690937E1403
:10D1800080937D14F901E050FC4F4083B7CD10929D
:10D190006104CACE0F90DF91CF911F910F91FF9044
:10D1A000EF90DF90CF90BF90AF909F907F906F9067
:10D1B0005F904F9008950F931F93CF93DF93CDB758
:10D1C000DEB72C970FB6F894DEBF0FBECDBFE3E2FB
:10D1D000F2E180859185A285B38544815581668180
:10D1E0007781008111812281338109831A832B8306
:10D1F0003C834D835E836F83788789879A87AB876B
:10D20000BC87AE01475F5F4FBE016B5F7F4FCE01B2
:10D210000196F3D62FE232E1AE01475F5F4FBE01C8
:10D220006B5F7F4FCE0101960E940C8E2C960FB63D
:10D23000F894DEBF0FBECDBFDF91CF911F910F914C
:10D2400008952F923F924F925F926F927F929F929A
:10D25000AF92BF92CF92DF92EF92FF920F931F9304
:10D26000CF93DF93CDB7DEB764970FB6F894DEBFE8
:10D270000FBECDBF2A013B01902EA12E6901082FC0
:10D2800010E0F801EA56F54BE491BB24B3941E1666
:10D290000CF4B12CFF24F39420E030E0A901C30189
:10D2A000B2010F948B3618160CF0F12C000F111FE1
:10D2B000000F111FC8018D5D9D4E1C01FC011082E5
:10D2C00011821282138277DFF101408251826282E1
:10D2D0007382E090581620E030E0A901692D7A2D84
:10D2E000C6010F94FB2F811108C0F801E75BF54BD5
:10D2F00085919591A591B49103C0892D9A2DD60160
:10D30000898B9A8BAB8BBC8B80912B1290912C12BA
:10D31000A0912D12B0912E124091271250912812F7
:10D320006091291270912A120091231210912412F7
:10D33000209125123091261209831A832B833C8376
:10D340004D835E836F83788789879A87AB87BC8795
:10D350001D861E861F86188AAE01475F5F4FBE017D
:10D360006B5F7F4FCE01019648D6CE010D966C01C2
:10D370008E010F5E1F4F2FE232E1AE01475F5F4F1C
:10D38000BE016B5F7F4F0C970E947A5060D8BF1030
:10D390000E94629364960FB6F894DEBF0FBECDBFB5
:10D3A000DF91CF911F910F91FF90EF90DF90CF9081
:10D3B000BF90AF909F907F906F905F904F903F9005
:10D3C0002F90089590912215891781F0809322154E
:10D3D000811108C00F94912186E192E188D80F94C1
:10D3E000740303C083E292E182D8E5CE089580E021
:10D3F000E9DFE5E8FEE080E090E0A0E8BFE38083BD
:10D400009183A283B38314821582168217821086B9
:10D410001186128613861486158616861786808BCB
:10D42000918BA28BB38B148A158A168A178A108E59
:10D43000118E128E138E148E158E168E178E80A35B
:10D4400091A3A2A3B3A308958091AC039091AD03DF
:10D45000009731F04AE050E060E070E00D94032E58
:10D4600060E070E0CB0108958091AC039091AD0332
:10D47000009731F04AE050E060E070E00D94DB2C62
:10D4800060E070E0CB010895EFDF97FD0AC0ECDFAC
:10D490006F3F71058105910509F02CF4E5DF862FBA
:10D4A000089580E008958FEF08958091AC039091E6
:10D4B000AD03892B31F0E8DF91E0811103C090E0EA
:10D4C00001C091E0892F08950F931F93CF9380910E
:10D4D000AC039091AD03009711F1FC018F01C19154
:10D4E0002C2F2F7DA9F0C53411F0C536B9F7F801FE
:10D4F000108260E070E08091AC039091AD030F94D6
:10D50000742BF801C083562F472F382F292F0BC0BB
:10D5100060E070E0CF911F910F910D94742B50E05B
:10D5200040E030E020E0652F742F832F922FCF91C1
:10D530001F910F91089581548A3108F041C0A82F9E
:10D54000B0E040919D1450919E1460919F14709191
:10D55000A01404C076956795579547958A95D2F79C
:10D5600040FF2EC0E0915216F0915316AD57BB4EBE
:10D570008C918823E9F0E80FF11D808190ED980FE0
:10D580009A3098F08E3211F481810CC08D3211F0F6
:10D590008B3271F4818190ED980F9A3030F08E3299
:10D5A00039F4828180538A3018F49E2F8F2F02C065
:10D5B00090E080E09093AC038093AD0381E0089508
:10D5C00080E00895B8DF882341F081E02091AC032A
:10D5D0003091AD03232B09F480E008954F925F92C0
:10D5E0006F927F92AF92BF92CF92DF92EF92FF92B3
:10D5F0000F931F93CF93DF93CDB7DEB7A0970FB6EE
:10D60000F894DEBF0FBECDBF0E9443E2811111C16D
:10D6100080E5D8DF882319F027DF162F01C010E03E
:10D6200083E5D0DF882319F01FDF5B0103C04CE0E6
:10D63000A42EB12C84E5C6DF811116DF82E5C2DF9E
:10D64000882321F041DF2B013C0106C0412C512CE5
:10D6500030ED632E30E4732E113009F4EAC012303D
:10D6600009F088C080E090E0A4E3B2E489839A8363
:10D67000AB83BC8380E090E0ACE2B3E48D839E8317
:10D68000AF83B88780E090E0A0E0BFEB89879A87FE
:10D69000AB87BC87AA2009F4CCC01D861E861F86D6
:10D6A000188ACE010D966C01E12CF12C00E01FEBE5
:10D6B00020E030E04CE253E460E070E084E392E488
:10D6C000A0D8B12C00E010E01D861E861F86188AA7
:10D6D000B801012E000C880B990B0F9401302CE738
:10D6E00039ED40E25FE30F9460306B017C010F94F1
:10D6F0003E35A30192010F94603020E030E04CE20F
:10D7000053E40F946534698F7A8F8B8F9C8FC70198
:10D71000B6010F94C636A30192010F94603020E049
:10D7200030E044E352E40F9465346D8F7E8F8F8F29
:10D7300098A3AE01435F5F4FBE01675E7F4FCE018E
:10D740004D96D5D90F5F1F4F0A30110509F0BCCF98
:10D75000B394BA1408F4B6CF1D861E861F86188AA5
:10D76000AE01435F5F4FBE016B5F7F4FCE010196FD
:10D77000BED95FC080E090E0A6EEB2E489839A83D0
:10D78000AB83BC8340E050E06CE273E44D835E8386
:10D790006F83788780E090E0A0E0BFEB89879A876D
:10D7A000AB87BC8700E010E024E332E40D871E87DE
:10D7B0002F87388B498B5A8B6B8B7C8B8D8B9E8BF9
:10D7C000AF8BB88F198E1A8E1B8E1C8ECE01499688
:10D7D0006C01E12CF12C00E01FEB9A01AB0160E041
:10D7E00070E084E392E40DD8BB24B594A79410E0D4
:10D7F000812F90E08A159B05E4F4198E1A8E1B8EFA
:10D800001C8EAE01475E5F4FBE016B5F7F4FCE0146
:10D8100001966DD9198E1A8E1B8E1C8EAE01475E35
:10D820005F4FBE016F5E7F4FCE010D9660D91F5FC7
:10D83000DFCFA0960FB6F894DEBF0FBECDBFDF914D
:10D84000CF911F910F91FF90EF90DF90CF90BF90FD
:10D85000AF907F906F905F904F900895AF92BF927E
:10D86000CF92DF92EF92FF920F931F93CF93DF93AC
:10D8700083E1A82E83E0B82E9CEBE92E94E1F92EEB
:10D8800003E212E121E6C22E26E1D22EC0E0D0E072
:10D89000F50181915F014FDE882319F115DEFE014C
:10D8A000E255FC4F2081211104C02091B2032223B4
:10D8B00041F0F80120813181428153810F94653418
:10D8C0000AC0C330D10539F0F6012081318142818F
:10D8D00053810F946434F70160837183828393834F
:10D8E0000AC0F80180819181A281B381F701808310
:10D8F0009183A283B3832196F4E0EF0EF11C0C5FB9
:10D900001F4F84E0C80ED11CC430D10509F0C0CF30
:10D9100086E458DE8823B9F0D7DD20E030E0A901A5
:10D920000F948B3618167CF4CFDD20E030E040E712
:10D9300052E40F94413560937002709371028093AA
:10D9400072029093730280915C1683FD2AC06091ED
:10D95000C8147091C9148091CA149091CB1420916D
:10D960002F12309130124091311250913212E091C9
:10D97000000CEE23B1F00F9464349B01AC01609174
:10D980000D0C70910E0C80910F0C9091100C0F9457
:10D99000653460930D0C70930E0C80930F0C909374
:10D9A000100CDF91CF911F910F91FF90EF90DF90BE
:10D9B000CF90BF90AF900895EF92FF920F931F9377
:10D9C000CF93DF937C0184E5FDDDD82F882341F1DF
:10D9D0005BDDC82F181604F5ECEFF4E484918F0199
:10D9E0000F5F1F4F882321F00F943F26F801F6CFD9
:10D9F0008DE40F943F26B70180E090E04AE00F9459
:10DA000092266C2FCC0F770B8FEB93E10E9489FE4F
:10DA10008AE00F943F2608C08093D204D0E004C06F
:10DA2000809158168093D2048D2FDF91CF911F9152
:10DA30000F91FF90EF900895FC01238121110C9428
:10DA40007ED1089580E1E3E2F2E1ACEBB4E1019034
:10DA50000D928A95E1F708954F925F926F927F92AF
:10DA60008F929F92AF92BF92CF92DF92EF92FF92EE
:10DA7000CF93DF93CDB7DEB72C970FB6F894DEBF08
:10DA80000FBECDBF8091D3049091D404A091D50452
:10DA9000B091D60489839A83AB83BC836091D70409
:10DAA0007091D804072E000C880B990B0F9401304D
:10DAB00029813A814B815C810F9464346B017C0134
:10DAC00060939704709398048093990490939A04B8
:10DAD00020910615309107154091081550910915B0
:10DAE0000F9460306D837E838F8398876093930457
:10DAF00070939404809395049093960420918F04DE
:10DB0000309190044091910450919204C701B60164
:10DB10000F9465344B015C0160938F047093900403
:10DB200080939104909392042091021530910315F3
:10DB300040910415509105150F94603069877A87DC
:10DB40008B879C8760938B0470938C0480938D04E7
:10DB500090938E0420ED3CEC4CE45DE36091FE1468
:10DB60007091FF1480910015909101150F94603011
:10DB70002B013C0120918704309188044091890455
:10DB800050918A0469817A818B819C810F946434DD
:10DB90009B01AC01C301B2010F9460302B013C0129
:10DBA00023E333E343E75FE36091830470918404EC
:10DBB00080918504909186040F9460309B01AC01A4
:10DBC000C301B2010F9465342B013C0160938304BF
:10DBD00070938404809385049093860489819A814C
:10DBE000AB81BC818093870490938804A0938904BF
:10DBF000B0938A0429853A854B855C856D817E8149
:10DC00008F8198850F946534A30192010F94643439
:10DC10002B013C0120E030E04FE753E40F948B36BA
:10DC200020E030E0A9011816ACF4C701B6010F944A
:10DC30008B3618166CF5A7019601C501B4010F9437
:10DC4000643460938F047093900480939104909354
:10DC500092041EC0C301B2010F94FB2F87FF22C0A4
:10DC600020E030E0A901C701B6010F94FB2F87FF28
:10DC700016C0A7019601C501B4010F9464346093E6
:10DC80008F0470939004809391049093920407C042
:10DC9000412C512C8FE7682E83E4782E03C0412C51
:10DCA000512C3201C301B2012C960FB6F894DEBF9D
:10DCB0000FBECDBFDF91CF91FF90EF90DF90CF905F
:10DCC000BF90AF909F908F907F906F905F904F909C
:10DCD00008952F923F924F925F926F927F928F9210
:10DCE0009F92AF92BF92CF92DF92EF92FF92CF932B
:10DCF000DF9300D01F92CDB7DEB760905A167090B8
:10DD00005B168090541690905516A0905616B090C1
:10DD10005716B301072C000C880B990B0F94013098
:10DD2000A50194010F9464346B017C0160937F041E
:10DD300070938004809381049093820420ED3CECE6
:10DD40004CE45DE360910A1570910B1580910C1500
:10DD500090910D150F9460301B012C0120917B04D4
:10DD600030917C0440917D0450917E04C501B40142
:10DD70000F9464349B01AC01C201B1010F94603077
:10DD80001B012C0123E333E343E75FE36091770456
:10DD9000709178048091790490917A040F946030A6
:10DDA0009B01AC01C201B1010F94653469837A8390
:10DDB0008B839C83609377047093780480937904B9
:10DDC00090937A0480927B0490927C04A0927D04CC
:10DDD000B0927E048091600E882321F081E08093D0
:10DDE0007604B9C020E030E040E251E4C701B6015A
:10DDF0000F948B36181624F481E080937604A4C027
:10DE000020E030E040E251ECC701B6010F94FB2F57
:10DE100087FDE4CF672811F380917604882351F0C1
:10DE2000109272041092730410927404109275048C
:10DE3000109276042091121530911315409114150B
:10DE400050911515C701B6010F9460302B013C01AC
:10DE500060936E0470936F048093700490937104C8
:10DE600020917204309173044091740450917504B0
:10DE7000C701B6010F9465344B015C0160937204D5
:10DE800070937304809374049093750420910E151D
:10DE900030910F1540911015509111150F9460306D
:10DEA0009B01AC0160936A0470936B0480936C04D3
:10DEB00090936D04C301B2010F94653429813A81B6
:10DEC0004B815C810F9464342B013C0120E030E0F5
:10DED0004FE753E40F948B3620E030E0A901181689
:10DEE000ACF4C701B6010F948B3618166CF5A70178
:10DEF0009601C501B4010F94643460937204709369
:10DF0000730480937404909375041EC0C301B2011E
:10DF10000F94FB2F87FF22C020E030E0A901C7014A
:10DF2000B6010F94FB2F87FF16C0A7019601C5010C
:10DF3000B4010F94643460937204709373048093FB
:10DF400074049093750407C0412C512C8FE7682E00
:10DF500083E4782E03C0412C512C3201C301B2015D
:10DF60000F900F900F900F90DF91CF91FF90EF9057
:10DF7000DF90CF90BF90AF909F908F907F906F90E9
:10DF80005F904F903F902F900895EF92FF920F93E4
:10DF90001F93CF93DF931F92CDB7DEB78C017B0128
:10DFA00080E249830F943F2649814F3F11F084E579
:10DFB00001C082E40F943F268AE30F943F26F801C4
:10DFC000608171818281938142E00F94F826F7018C
:10DFD000408151816281738183E396E10E9445FE15
:10DFE00062E070E080E090E00F90DF91CF911F91B0
:10DFF0000F91FF90EF900C9456A3CF92DF92EF9287
:10E00000FF920F931F93CF93DF93CDB7DEB728977F
:10E010000FB6F894DEBF0FBECDBF2091221522238C
:10E0200009F462C0C52ED42E8B017C0120E030E0C3
:10E0300040E450E4FC0160817181828193810F94FE
:10E0400065346D837E838F83988720E030E04EE3D4
:10E0500053E4F80160817181828193810F9464346B
:10E0600069837A838B839C83CF92DF92CE01019662
:10E070009F938F9304969F938F938DB79EB78497AA
:10E080000FB6F8949EBF0FBE8DBFADB7BEB7119649
:10E0900084E2E5E8FEE001900D928A95E1F70E94A6
:10E0A000CAFE20E030E040E450E46D817E818F8143
:10E0B00098850F946434F70160837183828393831E
:10E0C00020E030E04EE353E469817A818B819C81CA
:10E0D0000F946534F80160837183828393830FB654
:10E0E000F894DEBF0FBECDBF28960FB6F894DEBF02
:10E0F0000FBECDBFDF91CF911F910F91FF90EF9099
:10E10000DF90CF900895CF92DF92EF92FF928091AF
:10E110006F15882371F1C0906B15D0906C15E0904D
:10E120006D15F0906E1520E030E0A901C701B60131
:10E130000F94FB2F8823E9F020E030E040E05FE31C
:10E14000C701B6010F9460309B01AC010F946030A1
:10E150002BED3FE049E450E40F9460309B01AC01AB
:10E1600060E070E080E89FE30F9441356B017C0133
:10E1700006C0C12CD12C80E8E82E8FE3F82EC09287
:10E18000D904D092DA04E092DB04F092DC046091CE
:10E19000100270911102072E000C880B990B0F943E
:10E1A00001302AE037ED43E25CE30F946030A701D1
:10E1B00096010F946030609306027093070280937B
:10E1C000080290930902FF90EF90DF90CF9008959E
:10E1D0004F925F926F927F928F929F92AF92BF9277
:10E1E000CF92DF92EF92FF920F931F93CF93DF9323
:10E1F000CDB7DEB768970FB6F894DEBF0FBECDBFC0
:10E200008C015B014A01FC01EE5BFF4F6081718173
:10E21000828193810F94FF2F6B017C01D5012D9199
:10E220003D914D915C910F9460300F942B350F947C
:10E23000AE3569877A878B879C87F401208131818D
:10E2400042815381C701B6010F9460300F942B3582
:10E250000F94AE356D877E878F87988B29853A8599
:10E260004B855C85283731054105510540F488E729
:10E2700090E0A0E0B0E089879A87AB87BC872D85C6
:10E280003E854F855889283731054105510540F4B1
:10E2900088E790E0A0E0B0E08D879E87AF87B88BDD
:10E2A0009801225B3F4FD9018D919D910D90BC91BA
:10E2B000A02D89839A83AB83BC83BC01CD010F94CD
:10E2C00001302B013C0169857A858B859C850F94F3
:10E2D000FF2F698B7A8B8B8B9C8B20E030E0A90120
:10E2E000C301B2010F94FB2F882329F1A7019601E6
:10E2F000C701B6010F9460304B015C0129893A894E
:10E300004B895C89CA01B9010F9460309B01AC0153
:10E31000C501B4010F9464344B015C01A301920167
:10E32000C301B2010F9465349B01AC01C501B40176
:10E330000F94413503C060E070E0CB010F942B35A2
:10E340000F94AE356D837E838F83988769817A8140
:10E350008B819C8190958095709561957F4F8F4FB3
:10E360009F4F0F9401304B015C016D857E858F8539
:10E3700098890F94FF2F69837A838B839C8320E095
:10E3800030E0A901C501B4010F94FB2F882349F1A6
:10E3900029813A814B815C81CA01B9010F946030B7
:10E3A0006D8B7E8B8F8B988FA7019601C701B6016D
:10E3B0000F9460309B01AC016D897E898F89988DA7
:10E3C0000F9464346B017C01A5019401C501B40173
:10E3D0000F9465349B01AC01C701B6010F94413520
:10E3E00003C060E070E0CB010F94DA35F80185A03E
:10E3F00096A0A7A0B0A4750164012D813E814F8134
:10E400005885C21AD30AE40AF50A0F94AE35C61A23
:10E41000D70AE80AF90AF7FE73C020E030E0A90144
:10E42000C301B2010F94FB2F882309F443C0A30159
:10E430009201C301B2010F9465346B017C01C501E7
:10E44000B4010F94FF2F9B01AC01C701B6010F94DB
:10E4500060306B017C0129893A894B895C89CA014A
:10E46000B9010F9460309B01AC01C701B6010F9454
:10E4700064346B017C0129813A814B815C81CA0142
:10E48000B9010F9460309B01AC01C701B6010F9434
:10E4900065346B017C0120E030E040E850E4C301CA
:10E4A000B2010F9460309B01AC01C701B6010F941B
:10E4B000413503C060E070E0CB010F942B357B0148
:10E4C0006C0120E030E0A9010F948B36181624F07F
:10E4D000E12CF12CC12CD12CB701C6010F94AE3523
:10E4E0006D837E838F83988786169706A806B90664
:10E4F00020F48D829E82AF82B886C12CD12C760109
:10E500008D819E81AF81B885F80182A793A7A4A7CA
:10E51000B5A7C80ED91EEA1EFB1EC6A6D7A6E0AA3E
:10E52000F1AAEA5BFF4F29853A854B855C852083FC
:10E5300031834283538334968D859E85AF85B88918
:10E5400080839183A283B38368960FB6F894DEBF6D
:10E550000FBECDBFDF91CF911F910F91FF90EF9034
:10E56000DF90CF90BF90AF909F908F907F906F90F3
:10E570005F904F90089580916F0081FB992790F9EB
:10E5800081FF05C080916F008D7F80936F00109296
:10E5900001051092020510920305109204059923BB
:10E5A00029F080916F00826080936F0008954F92F0
:10E5B0005F926F927F928F929F92AF92BF92CF9213
:10E5C000DF92EF92FF920F931F93CF93DF933C0163
:10E5D000B0E2A0E06A2F70E0AB014B0F511D5595E2
:10E5E00047954A1711F04B130BC0E8E6F4E165912B
:10E5F0007491072E000C880B990B0F94013062C0A8
:10E60000CA010197880F991F880F991FFC01E651D5
:10E61000FC4E059114919A01220F331F220F331FD4
:10E62000F901E651FC4EC591D4916016710614F4BF
:10E63000B42FD2CFA42FC615D7050CF4CBCF84515D
:10E640009C4EFC01E590F490F901E451FC4EC5901C
:10E65000D490B7010F2C000C880B990B0F9401304C
:10E660004B015C01B301601B710B072E000C880B82
:10E67000990B0F9401302B013C01B6016E197F09F3
:10E68000072E000C880B990B0F9401309B01AC01F5
:10E69000C301B2010F9460306B017C01C01BD10B30
:10E6A000BE01DD0F880B990B0F9401309B01AC016B
:10E6B000C701B6010F9441359B01AC01C501B401FE
:10E6C0000F946534DF91CF911F910F91FF90EF90E0
:10E6D000DF90CF90BF90AF909F908F907F906F9082
:10E6E0005F904F9008950F931F93CF93DF93CDB713
:10E6F000DEB728970FB6F894DEBF0FBECDBF60918E
:10E700005A1670915B16072E000C880B990B0F940C
:10E7100001306D837E838F8398878091541690910A
:10E720005516A0915616B091571689839A83AB83DC
:10E73000BC834DEFBE016B5F7F4FCE01019625DCA0
:10E740006091D7047091D804072E000C880B990BA8
:10E750000F9401306D837E838F8398878091D304DB
:10E760009091D404A091D504B091D60489839A8362
:10E77000AB83BC834FEFBE016B5F7F4FCE01019631
:10E7800004DCEBE3F6E184918F010F5F1F4F8823D8
:10E7900021F00F943F26F801F6CFE091D204F0E08B
:10E7A000E053FB4F608170E080E090E00E940AD36C
:10E7B000E6E3F6E184918F010F5F1F4F882321F07C
:10E7C0000F943F26F801F6CF6091D10470E080E00D
:10E7D00090E00E940AD328960FB6F894DEBF0FBED1
:10E7E000CDBFDF91CF911F910F9108950F930FB778
:10E7F0000F9300916E000B7F00936E0078940F933F
:10E800000BB70F930CB70F921F922F933F934F9319
:10E810005F936F937F938F939F93AF93BF93EF9388
:10E82000FF93112409D2FF91EF91BF91AF919F9176
:10E830008F917F916F915F914F913F912F911F9099
:10E840000F900CBF0F910BBF0F910460F8940093D1
:10E850006E000F910FBF0F911895CF92DF92EF923C
:10E86000FF92C090D304D090D404E090D504F090EF
:10E87000D6048091D7049091D8040897BC01990FD1
:10E88000880B990B0F9401309B01AC01C701B601B5
:10E890000F94FB2F87FF1FC020E030E040E050E4E2
:10E8A000C701B6010F9465340F94AE357093B4046C
:10E8B0006093B3040E948EA3DC01CB01805A954182
:10E8C000AF4FBF4F8093AF049093B004A093B104B7
:10E8D000B093B20408C01092AF041092B00410922A
:10E8E000B1041092B204FF90EF90DF90CF900895A2
:10E8F000CF92DF92EF92FF92C0905416D0905516AF
:10E90000E0905616F090571680915A1690915B162B
:10E910000D97BC01990F880B990B0F9401309B0147
:10E92000AC01C701B6010F94FB2F87FF1FC020E089
:10E9300030E040E050E4C701B6010F9465340F9415
:10E94000AE357093AE046093AD040E948EA3DC01DB
:10E95000CB01805E914BAF4FBF4F8093A904909342
:10E96000AA04A093AB04B093AC0408C01092A9040D
:10E970001092AA041092AB041092AC04FF90EF9096
:10E98000DF90CF90089510925B1610925A1680E097
:10E99000AFDF1092D8041092D7045FDF0E94139467
:10E9A00010925B1610925A1680E0A2DF1092D004EB
:10E9B00075981092D8041092D7041092D104A5989B
:10E9C00008954F925F926F927F928F929F92AF9233
:10E9D000BF92CF92DF92EF92FF920F931F93CF934C
:10E9E000DF933C01BAE3A0E06A2F70E0AB014B0F6C
:10E9F000511D559547954A1711F04B130BC0EFEB7E
:10EA0000F5E165917491072E000C880B990B0F941A
:10EA1000013062C0CA010197880F991F880F991FA2
:10EA2000FC01E752FB4E059114919A01220F331F0E
:10EA3000220F331FF901E752FB4EC591D4916016A6
:10EA4000710614F4B42FD2CFA42FC615D7050CF439
:10EA5000CBCF85529B4EFC01E590F490F901E55235
:10EA6000FB4EC590D490B7010F2C000C880B990B6E
:10EA70000F9401304B015C01B301601B710B072E39
:10EA8000000C880B990B0F9401302B013C01B6014F
:10EA90006E197F09072E000C880B990B0F9401301B
:10EAA0009B01AC01C301B2010F9460306B017C018A
:10EAB000C01BD10BBE01DD0F880B990B0F940130E9
:10EAC0009B01AC01C701B6010F9441359B01AC011C
:10EAD000C501B4010F946534DF91CF911F910F915F
:10EAE000FF90EF90DF90CF90BF90AF909F908F906E
:10EAF0007F906F905F904F90089560E08091B70491
:10EB00009091B80454DD6093541670935516809319
:10EB10005616909357168091B5049091B60451DF24
:10EB20006093D3047093D4048093D5049093D60457
:10EB3000A8951092B9040895CF92DF92FF920F9397
:10EB40001F93CF93DF931F921F92CDB7DEB7F82E9E
:10EB50008A0180910A02882309F444C0E7E6F7E4B9
:10EB600084916F019FEFC91AD90A882341F0698304
:10EB70007A830F943F26F60169817A81F1CFFB01F8
:10EB800084916F019FEFC91AD90A882321F00F944D
:10EB90003F26F601F5CFEFE6F4E184916F019FEF98
:10EBA000C91AD90A882321F00F943F26F601F5CF20
:10EBB000F7FC0BC06F2DFF0C770B880B990B0E9495
:10EBC0000AD38AE00F943F260DC0EAE6F4E184916F
:10EBD0006F019FEFC91AD90A882321F00F943F26AD
:10EBE000F601F5CF80916904811108C010920A02E4
:10EBF00081E080936904C8010F94DA050F900F90AB
:10EC0000DF91CF911F910F91FF90DF90CF90BBCEFE
:10EC10008F3F19F044EF55E102C044E056E165E151
:10EC200076E18ACF8F3F19F041EC55E102C041ED0A
:10EC300055E162EE75E180CF0F931F93CF93DF9381
:10EC400080910F028F3790F08F579091D00490935E
:10EC5000CF04992311F0759A01C075989091D10451
:10EC60009093CE04992359F0A59A0AC09091CF04AD
:10EC7000891708F075989091CE04891708F0A59827
:10EC80008F5F80930F029091CD0481E0892780935C
:10EC9000CD0481110E9488BB80910E02853018F44A
:10ECA000C1E0C80F01C0C0E0823009F4ACC048F434
:10ECB0008823F9F0813009F0DAC010927B0080E4FB
:10ECC000B8C0843009F4BDC008F4B0C0853009F084
:10ECD000CEC09091CC04911102C08093CC0480915D
:10ECE000CC0481508093CC04882309F4C0C0C5E0D3
:10ECF000BEC080910D028F5F80311CF480930D02A5
:10ED0000B6C010920D028091B904811113C0809198
:10ED1000C2049091C3049093B8048093B704809187
:10ED2000C0049091C1049093B6048093B50481E02F
:10ED30008093B9048AE0E2ECF4E0DF011D928A9549
:10ED4000E9F71092C1041092C0040091B704109129
:10ED5000B804119501951109D1E08091D004811179
:10ED600001C0D0E08091EF0B9091F00B91958195CF
:10ED700091098017910744F4DD2331F041EC55E10E
:10ED800062EE75E180E0D8DE80913B0290913C021A
:10ED90009195819591090817190744F4DD2331F005
:10EDA00044EF55E165E176E180E0C6DE11E0809157
:10EDB000D104811101C010E02091B5043091B60456
:10EDC0008091ED0B9091EE0B8217930744F0112385
:10EDD00031F041ED55E162EE75E18FEFADDE20914E
:10EDE000390230913A028091B5049091B6048217AD
:10EDF0009307ECF11123D9F144E056E165E176E1A6
:10EE00008FEF9ADE34C080917A0086FD2DC080910C
:10EE10007800909179002091C2043091C304820F50
:10EE2000931F9093C3048093C20421C010927B006F
:10EE300082E480937C0080917A00806480937A00E1
:10EE400016C080917A0086FD11C080917800909163
:10EE500079002091C0043091C104820F931F9093D8
:10EE6000C1048093C00403C0C2E001C0C4E0C093E9
:10EE70000E0220E030E0A1E0B4E0C901880F991F44
:10EE8000FC01E654FB4F608171816115710509F445
:10EE900036C0F894223001F550910901547015984C
:10EEA00040910B01161617060CF4409544704093E0
:10EEB0000901000000004A2F4A950000E9F7429A34
:10EEC0004B2F4A950000E9F7429840910B015111F0
:10EED00040954470409309017894FC01E654FB4F3F
:10EEE000161617063CF44081518141505109518357
:10EEF000408305C0808191810196918380832F5F3B
:10EF00003F4F2330310509F0B8CF0E94B69280916F
:10EF1000FA039091FB03009799F001979093FB03FC
:10EF20008093FA03892B61F487E296E1909359125A
:10EF300080935812DF91CF911F910F910C940A6624
:10EF4000DF91CF911F910F9108958F929F92AF9271
:10EF5000BF92CF92DF92EF92FF920F93CF93DF9306
:10EF600000D01F92CDB7DEB78091AB1581111CC1C7
:10EF70008091B904811110C00F900F900F900F90E5
:10EF8000DF91CF910F91FF90EF90DF90CF90BF90E6
:10EF9000AF909F908F900895B0DD0E948EA34B019B
:10EFA0005C0180910B0290910C02181619060CF06E
:10EFB0001CC1019790930C0280930B028091600E0C
:10EFC000811117C08091A5049091A604A091A70477
:10EFD000B091A8040097A105B10559F0A5019401CD
:10EFE000281B390B4A0B5B0B57FD03C081E0809354
:10EFF000600E60915A1670915B16072E000C880BFC
:10F00000990B0F94013069837A838B839C833EE153
:10F01000E32EF12C00E09E012F5F3F4F44E556E1C7
:10F0200061EA74E080EA94E00E943FD6C0905416F2
:10F03000D0905516E0905616F09057168091F10B2F
:10F040009091F20BBC01990F880B990B0F94013032
:10F050009B01AC01C701B6010F948B3618160CF456
:10F06000A7C060E06093D0048091A9049091AA04A5
:10F07000A091AB04B091AC040097A105B10521F1BA
:10F08000A5019401281B390B4A0B5B0B57FD1CC0D3
:10F090006091AD047091AE0480E090E00F94FF2F7A
:10F0A0009B01AC01609154167091551680915616D3
:10F0B000909157160F94FB2F87FFBFC04FEA54E182
:10F0C00061EC74E180E038DD8091AF049091B00490
:10F0D000A091B104B091B2040097A105B10511F15E
:10F0E000881A990AAA0ABB0AB7FC1CC06091B3042B
:10F0F0007091B40480E090E00F94FF2F9B01AC016D
:10F100006091D3047091D4048091D5049091D60479
:10F110000F94FB2F87FF88C04DE854E160EA74E14B
:10F120008FEF0ADD6091D7047091D804072E000C90
:10F13000880B990B0F94013069837A838B839C83AE
:10F140009AE0E92EF12C0FEF9E012F5F3F4F43ED28
:10F1500054E06BE974E08FE994E00E943FD680911F
:10F160005F0E81113FC0C090D304D090D404E090D2
:10F17000D504F090D60420E030E040EA50E4C70126
:10F18000B6010F948B3687FD0BC020E030E046E1DE
:10F1900053E4C701B6010F94FB2F18160CF046C0BC
:10F1A00060E06093D104E8CE80ED94E10F94DA053D
:10F1B00060913D0270913E02072E000C880B990B66
:10F1C0000F9401309B01AC01C701B6010F94FB2FD6
:10F1D00087FF47CF80E00E94696E0F94A93575952F
:10F1E000679540CF1092D104C7CEC0905416D090EE
:10F1F0005516E0905616F090571620E030E848E992
:10F2000053E4C701B6010F948B361816CCF020E0FA
:10F2100030E040EA50E4C701B6010F94FB2F87FFAE
:10F22000CDCE80E0F5DCCACE18DB7CCF0E942C6D01
:10F230000F94A93575956795B4CF80E059DB44CF1D
:10F2400080E0F0DCC0905416D0905516E090561631
:10F25000F0905716DCCFCF93DF9381E08093E514D5
:10F260000E944AEC1092E5148823B1F0ECEFF4E42C
:10F270008491EF012196882321F00F943F26FE010F
:10F28000F7CFEDEEF7E18491EF012196882321F08D
:10F290000F943F26FE01F7CFDF91CF910895CF93D2
:10F2A00080916F0081FBCC27C0F981FF05C0809160
:10F2B0006F008D7F80936F008091840E8093830E0A
:10F2C0008093820E8093810E84E68093800E53D9C2
:10F2D00088EE93E09093FB038093FA03CC2329F00C
:10F2E00080916F00826080936F0081E08093DB0AE1
:10F2F0000E9427620F94912186E192E10E94776239
:10F300000F947403CF910C94DB68CF93DF93ECEFF1
:10F31000F4E48491EF012196882321F00F943F2695
:10F32000FE01F7CF83E50E949B6A882321F00E94AB
:10F33000556A80936302E7E5F7E18491EF01219636
:10F34000882321F00F943F26FE01F7CF80916302BE
:10F35000811103C0E3E5F7E102C0EFE4F7E1849136
:10F36000EF012196882321F00F943F26FE01F7CF6D
:10F37000E7E4F7E18491EF012196882321F00F94CF
:10F380003F26FE01F7CF2091611630916216409121
:10F39000631650916416609112027091130280916D
:10F3A0001402909115020F946534AB01BC0185E401
:10F3B00097E10E9445FE20916516309166164091B6
:10F3C000671650916816609116027091170280912D
:10F3D0001802909119020F946534AB01BC0182E4CC
:10F3E00097E10E9445FE2091691630916A1640917E
:10F3F0006B1650916C1660911A0270911B028091ED
:10F400001C0290911D020F946534AB01BC018FE387
:10F4100097E10E9445FEE7E3F7E18491EF01219631
:10F42000882321F00F943F26FE01F7CF209161162B
:10F4300030916216409163165091641660915702A4
:10F44000709158028091590290915A020F9465343C
:10F45000AB01BC0185E397E10E9445FE2091651652
:10F4600030916616409167165091681660915B0264
:10F4700070915C0280915D0290915E020F94653400
:10F48000AB01BC0182E397E10E9445FE2091691621
:10F4900030916A1640916B1650916C1660915F0224
:10F4A0007091600280916102909162020F946534C4
:10F4B000AB01BC018FE297E10E9445FE8AE0DF913B
:10F4C000CF910D943F2682E40E949B6A882351F0DD
:10F4D0000E94246A60933B1570933C1580933D1500
:10F4E00090933E1583E50E949B6A882351F00E9409
:10F4F000646A60933715709338158093391590932B
:10F500003A1584E50E949B6A882351F00E94646A40
:10F510006093331570933415809335159093361599
:10F5200088E50E949B6A882351F00E94646A609378
:10F53000231570932415809325159093261589E53E
:10F540000E949B6A882351F00E94646A6093271589
:10F55000709328158093291590932A158AE50E94A7
:10F560009B6A882351F00E94646A60932B15709304
:10F570002C1580932D1590932E1585E40E949B6A7F
:10F58000882351F00E94646A60932F1570933015A0
:10F5900080933115909332150895CF9383E50E949F
:10F5A000E26A8823A1F00E94646A60934715709311
:10F5B00048158093491590934A1560933F157093B1
:10F5C00040158093411590934215C0E001C0C1E001
:10F5D00080E50E94E26A882359F00E94646A609381
:10F5E0004715709348158093491590934A15C0E0CC
:10F5F00082E50E94E26A882359F00E94646A60935F
:10F600004315709344158093451590934615C0E0BB
:10F6100084E50E94E26A882359F00E94646A60933C
:10F620003F157093401580934115909342152AC061
:10F63000CC2341F1409147155091481560914915EF
:10F6400070914A158FE197E10E9445FE4091431564
:10F650005091441560914515709146158CE197E1E4
:10F660000E9445FE40913F15509140156091411513
:10F670007091421589E197E10E9445FE8AE0CF91A1
:10F680000D943F26CF910895FF920F931F93CF9330
:10F69000DF930BE515E1C3E1D3E0FC2E84E0F80E27
:10F6A00089910E949B6A882339F00E94646AF8015C
:10F6B00060837183828393830C5F1F4FFC12F0CFB2
:10F6C000DF91CF911F910F91FF900895FF920F93BB
:10F6D0001F93CF93DF930BE415E1C3E1D3E0FC2E3E
:10F6E00084E0F80E89910E949B6A882349F00E9469
:10F6F000646A0F94AE35F8016083718382839383CB
:10F700000C5F1F4FFC12EECFDF91CF911F910F9135
:10F71000FF900C94A28DCF9388EC90E00E94DC6C5B
:10F72000811140C084E40E949B6A8823C1F10E9439
:10F73000646AC1E020E030E0A9010F94FB2F811141
:10F7400001C0C0E0C0936F15CC2349F10E94646AE8
:10F75000E091D20424E0E29FF0011124E559FA4E31
:10F76000608371838283938320E030E0A9016091FC
:10F770006B1570916C1580916D1590916E150F94AD
:10F78000FB2F81110CC080E090E0A0E4B0E48093F6
:10F790006B1590936C15A0936D15B0936E15CF916A
:10F7A0000C948370CF910895EF92FF920F931F9363
:10F7B000CF93DF931F92CDB7DEB7082F162FE4E16A
:10F7C000F7E184917F012FEFE21AF20A882331F0EA
:10F7D00099830F943F26F7019981F3CFE02FF92FFA
:10F7E00084917F019FEFE91AF90A882321F00F9491
:10F7F0003F26F701F5CFE2E1F7E184917F012FEF9A
:10F80000E21AF20A882321F00F943F26F701F5CF80
:10F81000612F70E080E090E00E940AD38AE00F90B0
:10F82000DF91CF911F910F91FF90EF900D943F26A4
:10F830004F925F926F927F928F929F92AF92BF9200
:10F84000CF92DF92EF92FF92CF93DF93EFE0F7E159
:10F850008491EF012196882321F00F943F26FE0129
:10F86000F7CF209161163091621640916316509146
:10F870006416609123127091241280912512909148
:10F8800026120F94653442E00F94F826EBE0F7E17E
:10F890008491EF012196882321F00F943F26FE01E9
:10F8A000F7CF2091651630916616409167165091FA
:10F8B00068166091271270912812809129129091F8
:10F8C0002A120F94653442E00F94F826E7E0F7E13E
:10F8D0008491EF012196882321F00F943F26FE01A9
:10F8E000F7CF2091691630916A1640916B165091AE
:10F8F0006C1660912B1270912C1280912D129091A8
:10F900002E120F94653442E00F94F826E3E0F7E1FD
:10F910008491EF012196882321F00F943F26FE0168
:10F92000F7CF60912F127091301280913112909127
:10F93000321242E00F94F82680916F0081FB9927E4
:10F9400090F981FF05C080916F008D7F80936F00DB
:10F9500040903712509038126090391270903A12DD
:10F9600080903B1290903C12A0903D12B0903E12BD
:10F97000C0903F12D0904012E0904112F09042129D
:10F98000992329F080916F00826080936F00E9EFE6
:10F99000F6E18491EF012196882321F00F943F2610
:10F9A000FE01F7CFC301B2010E940AD3E5EFF6E1F1
:10F9B0008491EF012196882321F00F943F26FE01C8
:10F9C000F7CFC501B4010E940AD3E1EFF6E18491BB
:10F9D000EF012196882321F00F943F26FE01F7CFF7
:10F9E000C701B6010E940AD38AE0DF91CF91FF9050
:10F9F000EF90DF90CF90BF90AF909F908F907F90CF
:10FA00006F905F904F900D943F262F923F924F92B0
:10FA10005F926F927F928F929F92AF92BF92CF929E
:10FA2000DF92EF92FF920F931F93CF93DF93CDB7A7
:10FA3000DEB763970FB6F894DEBF0FBECDBF0E944E
:10FA400043E28111CEC09DE3892E9AE4992E83E290
:10FA500092E19A8B898BFE0131965F0106E91AE4E7
:10FA60001F01F3E0F00FFB8BF40165917591859117
:10FA70009491E989FA89C190D190E190F190FA8B43
:10FA8000E98BA70196010F9464342B013C0120E01F
:10FA900030E040EA51EC0F948B3687FD10C020E037
:10FAA00030E040EA51E4C301B2010F94FB2F181675
:10FAB00034F0F10140825182628273820DC0F801FC
:10FAC00084911816B4F7F7FAF094F7F8F094F1016E
:10FAD000C082D182E282F382F101C190D190E190A3
:10FAE000F1901F0120E030E040EA51ECC701B6017F
:10FAF0000F948B3687FF03C0E7E6F7E40BC020E0E6
:10FB000030E040EA51E4C701B6010F94FB2F18160C
:10FB10003CF5F2CF84918F010F5F1F4F882321F0B6
:10FB20000F943F26F801F6CFEFECF7E184918F01B7
:10FB30000F5F1F4F882321F00F943F26F801F6CF67
:10FB400061E081EC97E10E94E1BB0E94A44E88E253
:10FB500090E0988B8F8788EC90E09E878D873AC0E5
:10FB6000F4E08F0E911C0F5F1F4F8B8980137CCFA9
:10FB700085E1E82E8CE0F82E10E0F501819191915D
:10FB8000A191B1915F01F70181939193A193B193F9
:10FB90007F01812F0E94B6651F5F133071F748DE29
:10FBA00060E081EB97E10E94E1BB83E992E0988BF2
:10FBB0008F8704E610E01E870D87BE01615F7F4FCF
:10FBC000CE010D960E942DDF8AEB92E0988B8F87F5
:10FBD0001E870D87BE01615F7F4FCE010D960E948B
:10FBE0002DDF63960FB6F894DEBF0FBECDBFDF9159
:10FBF000CF911F910F91FF90EF90DF90CF90BF902A
:10FC0000AF909F908F907F906F905F904F903F90BC
:10FC10002F9008950F931F93CF93DF93CDB7DEB747
:10FC20002C970FB6F894DEBF0FBECDBF83E50E94C0
:10FC30009B6A882349F00E94556A182F811106C0DB
:10FC400080E00E94E26902C0109122158091231287
:10FC500090912412A0912512B091261289839A8343
:10FC6000AB83BC838091271290912812A091291216
:10FC7000B0912A128D839E83AF83B88780912B1217
:10FC800090912C12A0912D12B0912E1289879A87F3
:10FC9000AB87BC8786E50E949B6A882321F084E9B4
:10FCA00097E10F946F2A812F0E94E269111103C01E
:10FCB000ECEFF4E41CC0809122158111F9CFE7E646
:10FCC000F7E484918F010F5F1F4F882321F00F9479
:10FCD0003F26F801F6CFE5E7F7E184918F010F5F4A
:10FCE0001F4F882329F30F943F26F801F6CF849104
:10FCF0008F010F5F1F4F882321F00F943F26F801DB
:10FD0000F6CF80912215811103C06BE173E002C030
:10FD100067E173E087E697E10E94A2FE8AE00F9414
:10FD20003F264CE050E063E272E1CE0101960F9471
:10FD30006A37892B59F02C960FB6F894DEBF0FBEA8
:10FD4000CDBFDF91CF911F910F9172CD2C960FB641
:10FD5000F894DEBF0FBECDBFDF91CF911F910F9101
:10FD60000895EF92FF920F931F93CF9383E1E82EB4
:10FD700083E0F82E05E11CE0C0E0F70181917F01EE
:10FD80000E949B6A882351F00E94646AF801608394
:10FD90007183828393838C2F0E94B665CF5F0C5F43
:10FDA0001F4FC33051F7CF911F910F91FF90EF90EC
:10FDB0003FCDCF93DF9383E50E94E26A882321F051
:10FDC0000E94346AEB0102C0C0E0D0E0DD27C230FF
:10FDD000D105BCF0E7E6F7E48491EF012196882392
:10FDE00021F00F943F26FE01F7CFEFECF6E184916E
:10FDF000EF012196882309F450C00F943F26FE019D
:10FE0000F6CF88E40E94E26A8823A9F00E94346A4F
:10FE1000683771053CF0633281E078072CF062E2CC
:10FE200071E002C068E770E0FE01EE0FFF1FE25EC6
:10FE3000FA4E7183608386E40E94E26A8823A9F007
:10FE40000E94346AFE01EE0FFF1FEA5EFA4E7183D4
:10FE500060836F3F710519F014F06FEF70E077FF6A
:10FE600002C060E070E07183608382E40E94E26A15
:10FE7000882399F00E94346A6530710534F068383F
:10FE800071052CF067E870E002C065E070E0CC0F0F
:10FE9000DD1FC65EDA4E79836883DF91CF910895C6
:10FEA000CF93DF9383E50E94E26A882351F00E949A
:10FEB000446A8D3308F08CE380936402DF91CF9124
:10FEC0000895ECEFF4E48491EF012196882321F06A
:10FED0000F943F26FE01F7CF4091640250E060E0AE
:10FEE00070E088EC96E10E9428FE8AE0DF91CF91D5
:10FEF0000D943F26DF92EF92FF920F931F93CF93C3
:10FF0000DF9383E50E949B6A882359F083E50E9472
:10FF1000E26A882319F00E94446A01C080E080935D
:10FF20005C16ECEFF4E48491EF012196882321F034
:10FF30000F943F26FE01F7CFE1ECF6E18491EF014B
:10FF40002196882321F00F943F26FE01F7CF809160
:10FF50005C16882389F183EBE82E86E1F82E00E019
:10FF600010E020E080915C1690E0002E02C0959594
:10FF700087950A94E2F780FF16C0DD24D394D20E51
:10FF8000222319F08CE20F943F26F701259134913A
:10FF9000F9018491E9012196882321F00F943F26ED
:10FFA0009E01F6CF2D2D0F5F1F4FF2E0EF0EF11CDB
:10FFB00005301105B9F60BC0EDEBF6E18491EF01C8
:10FFC0002196882321F00F943F26FE01F7CF8AE087
:10FFD000DF91CF911F910F91FF90EF90DF900D94E3
:10FFE0003F262F923F924F925F926F927F928F9215
:10FFF0009F92AF92BF92CF92DF92EF92FF920F93B8
:020000021000EC
:100000001F93CF93DF93CDB7DEB762970FB6F89407
:10001000DEBF0FBECDBF80915C1683FD88C183E536
:100020000E94E26A8C87811106C082E50E94E26A22
:10003000882309F47CC10E94646A0F94A93566394B
:1000400071050CF071C17093D8046093D7040E94BD
:100050002D746091D7047091D804072E000C880B82
:10006000990B0F9401302091D3043091D404409126
:10007000D5045091D6040F948B3618161CF085E9E0
:1000800096E102C084EA96E160E00E94E1BB81E073
:1000900080936902809158168093D2041A821B8241
:1000A0001C821D82188619861A861B8619821D8657
:1000B0002CE32E873CE13F8746E4488BE12CF12C72
:1000C00000E81FEB812C912C54016091D7047091B2
:1000D000D804072E000C880B990B0F940130698B04
:1000E0007A8B782E692E9B01482F592FB701C801B2
:1000F0000F94FB2F8823B1F12091D3043091D404C5
:100100004091D5045091D60469897A89872D962D1E
:100110000F94FB2F881F8827881F89835C855523B0
:1001200029F1882319F180916902882309F4FFC01D
:1001300062960FB6F894DEBF0FBECDBFDF91CF91B0
:100140001F910F91FF90EF90DF90CF90BF90AF90F5
:100150009F908F907F906F905F904F903F902F90E7
:100160000D94AE23E98AFA8A702E612E0E948EA326
:100170006B017C01DC01CB01288539854A855B85D3
:10018000821B930BA40BB50BB7FD3AC0D701C60178
:1001900088519C4FAF4FBF4F88879987AA87BB87ED
:1001A0000E947373E1E9F6E184918F010F5F1F4FA5
:1001B000882321F00F943F26F801F6CF8114910493
:1001C000A104B104B9F0D501C40188519C4FAF4FCF
:1001D000BF4FBC01CD016C197D098E099F0928EE26
:1001E00033E040E050E00F940734CA01B9010E94A7
:1001F0000AD303C08FE30F943F268AE00F943F2673
:1002000080E00F94BB1E0E948EA3609382157093B2
:10021000831580938415909385159091D3049E83C4
:10022000A091D404AF830091D5041091D604292F56
:100230003A2FA80169897A89872D962D0F94643405
:100240001B012C0120E030E0A9010F948B3687FFC1
:1002500004C057FA509457F8509420E030E040EA38
:1002600050E4C201B10181149104A104B10429F444
:100270000F94FB2F87FF07C004C00F948B3618160E
:1002800014F446015701B981BB2391F12A813B81C6
:100290004C815D81211531054105510541F0D701A2
:1002A000C601821B930BA40BB50BB7FD21C02E8199
:1002B0003F81A8016D857E858F8598890F94643470
:1002C00020E030E040EC5FE30F94FB2F87FD2BCF65
:1002D000D701C601805A9541AF4FBF4F8A839B8398
:1002E000AC83BD839E819D87AF81AE870F87188BBE
:1002F00080916902882309F416CF81149104A10426
:10030000B10429F4E988FA88072D162DDECEB8EE5F
:10031000CB1AB3E0DB0AE108F108C818D908EA08EB
:10032000FB08F7FE00CFEECF66E970E08CCE629658
:100330000FB6F894DEBF0FBECDBFDF91CF911F91F6
:100340000F91FF90EF90DF90CF90BF90AF909F9074
:100350008F907F906F905F904F903F902F90089577
:1003600080915C1683FD14C083E50E94E26A8823B5
:1003700079F00E94646A0F94A9356639710514F00A
:1003800066E970E07093D8046093D7040C942D74E0
:1003900008952F923F924F925F926F927F928F9229
:1003A0009F92AF92BF92CF92DF92EF92FF920F9304
:1003B0001F93CF93DF93CDB7DEB762970FB6F89454
:1003C000DEBF0FBECDBF8DE690E00E94DC6C8111D8
:1003D00086C180915C1683FD82C183E50E94E26A3A
:1003E0008E83811106C082E50E94E26A882309F4A7
:1003F00076C10E94646A0F94A93570935B1660936E
:100400005A1680E00E94787460915A1670915B16BB
:10041000072E000C880B990B0F9401302091541675
:100420003091551640915616509157160F948B36B1
:10043000181634F02E81211108C089E696E102C019
:100440008DE796E160E00E94E1BB81E08093690264
:100450001A821B821C821D8219861A861B861C86A4
:1004600019821D863CE33E874CE14F8756E4588B4A
:10047000E12CF12C00E81FEB812C912C54016091B0
:100480005A1670915B16072E000C880B990B0F946F
:100490000130698B7A8B782E692E9B01482F592F5A
:1004A000B701C8010F94FB2F8823B9F1209154168E
:1004B00030915516409156165091571669897A8990
:1004C000872D962D0F94FB2F881F8827881F8983DF
:1004D0008E81882331F19981992319F180916902E4
:1004E000882309F4FCC062960FB6F894DEBF0FBEF5
:1004F000CDBFDF91CF911F910F91FF90EF90DF90D3
:10050000CF90BF90AF909F908F907F906F905F90B3
:100510004F903F902F900D94AE23E98AFA8A702E67
:10052000612E0E948EA36B017C01DC01CB01298529
:100530003A854B855C85821B930BA40BB50BB7FDED
:100540003AC0D701C60188519C4FAF4FBF4F898732
:100550009A87AB87BC870E947373E5E6F6E18491C6
:100560008F010F5F1F4F882321F00F943F26F80162
:10057000F6CF81149104A104B104B9F0D501C401EE
:1005800088519C4FAF4FBF4FBC01CD016C197D0905
:100590008E099F0928EE33E040E050E00F940734C5
:1005A000CA01B9010E940AD303C08FE30F943F260A
:1005B0008AE00F943F2680E00F94BB1E0E948EA31A
:1005C000609382157093831580938415909385159D
:1005D000909154169F83A0915516A88700915616A6
:1005E00010915716292F3A2FA80169897A89872DEA
:1005F000962D0F9464341B012C0120E030E0A901FA
:100600000F948B3687FF04C057FA509457F85094D4
:1006100020E030E040E251E4C201B10181149104D4
:10062000A104B10429F40F94FB2F87FF07C004C075
:100630000F948B36181614F446015701B981BB2369
:1006400091F12A813B814C815D8121153105410564
:10065000510541F0D701C601821B930BA40BB50BCA
:10066000B7FD21C02F813885A8016D857E858F85D6
:1006700098890F94643420E030E040EC5FE30F94FD
:10068000FB2F87FD2BCFD701C601805A9541AF4F75
:10069000BF4F8A839B83AC83BD839F819D87A88541
:1006A000AE870F87188B80916902882309F416CFD3
:1006B00081149104A104B10429F4E988FA88072D72
:1006C000162DDDCEB8EECB1AB3E0DB0AE108F10857
:1006D000C818D908EA08FB08F7FE00CFEECF6296EB
:1006E0000FB6F894DEBF0FBECDBFDF91CF911F9143
:1006F0000F91FF90EF90DF90CF90BF90AF909F90C1
:100700008F907F906F905F904F903F902F900895C3
:10071000CF93DF938091830E9091840E891B8F700D
:1007200009F445C09091800E992351F0833030F444
:100730008FEF890F19F08093800E3BC01092800ECE
:10074000E091840E88E5E89FF0011124EB5FFA4FF9
:10075000808180FD2EC08091010590910205A091BD
:100760000305B0910405EF01CC5ADF4F4881598150
:100770006A817B81841B950BA60BB70B80930105C7
:1007800090930205A0930305B09304058091840E15
:100790008F5F8F708093810E9091840E8091820E76
:1007A00098130AC08091810E8093820E05C00E942A
:1007B000BB7280E090E001C0CF01DF91CF9108953E
:1007C00067FD2CC0813061F028F0823099F08330D1
:1007D000D9F024C0662311F0A19A2AC0A19828C09C
:1007E000809108016111809580788093060147FF10
:1007F00027C00895809108016111809580748093CD
:10080000060147FF23C0089580910801611180957A
:1008100088708093060147FF1FC0089547FD24C0DC
:10082000813071F038F0823089F08330A9F008957A
:1008300047FD1AC0442311F0A09A0895A098089586
:10084000442311F0A29A0895A29808958091080176
:1008500041118095807205C08091080141118095F9
:1008600080718093060108950895DB01833070F450
:1008700094E0899FF0011124E251FB4EAB01770F08
:10088000660B770B4083518362837383813089F0D9
:1008900018F08230D9F008952FEF30E00F945C37D4
:1008A00020ED37E040E050E00F942934B9018EE2AA
:1008B00019C02FEF30E00F945C3720ED37E040E0B7
:1008C00050E00F942934B9018DE20CC02FEF30E0D5
:1008D0000F945C3720ED37E040E050E00F9429346E
:1008E000B9018CE20C948FA2CF93DF93CEEED4E1CA
:1008F0006881798180E0B9DF6C817D8181E0B5DF3D
:100900006885798582E0DF91CF91AFCF90916F00BC
:1009100091FB222720F991FF05C090916F009D7FE8
:1009200090936F0034E0839FC0011124FC01E95CC7
:10093000FD4E4081518162817381FC01E452F54F8B
:10094000408351836283738381E08093DB0A222397
:1009500029F080916F00826080936F0008959091DC
:100960006F0091FB222720F991FF05C090916F0045
:100970009D7F90936F0094E0899FF0011124E95CC2
:10098000FD4E6081718182819381222329F0209123
:100990006F00226020936F000895BC012091D90A56
:1009A0003091DA0A4091D90A5091DA0A24173507B2
:1009B00011F09A01F7CF81E06217730709F080E028
:1009C00008950F930FB70F9300916E000F930B7F55
:1009D00000936E0000916F000D7F00936F000F93E6
:1009E0000BB70F930CB70F921F922F933F934F9318
:1009F0005F936F937F938F939F93AF93BF93EF9387
:100A0000FF9311245DD0FF91EF91BF91AF919F9122
:100A10008F917F916F915F914F913F912F911F9097
:100A20000F900CBF0F910BBF0F910260F8940093D1
:100A30006F000F9100936E000F910FBF0F911895EB
:100A400080918B0A80FF07C080910B018270809398
:100A500009018FEF07C080910B0180958270809310
:100A6000090181E08093850A80918B0A81FF08C08B
:100A700080910B0180958170809309018FEF06C0F2
:100A800080910B0181708093090181E08093860A37
:100A900080918B0A82FF07C080910B018470809344
:100AA00009018FEF07C080910B01809584708093BE
:100AB000090181E08093870A00000000000008958A
:100AC0002F923F924F925F926F927F928F929F925E
:100AD000AF92BF92CF92DF92EF92FF920F931F934C
:100AE000CF93DF9300D000D0CDB7DEB7F8948FEF6F
:100AF0009FEF90938900809388002AE02D83212C1A
:100B0000312C78948091D50A9091D60AA091D70A79
:100B1000B091D80A892B8A2B8B2B09F0CDC18091FB
:100B2000DB0A8823D1F01092DB0A8091D90A9091D8
:100B3000DA0A892B91F01092CC0A1092DA0A1092FC
:100B4000D90A9091830E8091840E981731F080918C
:100B5000840E8F5F8F708093840E8091D90A90915C
:100B6000DA0A892B09F4A8C14091D10A5091D20A1E
:100B70006091D30A7091D40A9091BF0A0091CD0A76
:100B80001091CE0A2091CF0A3091D00A041B150B88
:100B9000260B370B892F90E0A0E0B0E0081719076B
:100BA0002A073B0710F4D901C801E82F840F951FCD
:100BB000A61FB71F8093D10A9093D20AA093D30A9D
:100BC000B093D40A2091840030918500225E3F4F7B
:100BD0004091A50A5091A60A6091A70A7091A80AAF
:100BE0008091950A9091960AA091970AB091980ADF
:100BF000840F951FA61FB71F8093A50A9093A60A7E
:100C0000A093A70AB093A80AB7FD1CC0409A4091D0
:100C10003712509138126091391270913A128091C6
:100C2000850A082E000C990BAA0BBB0B840F951F8D
:100C3000A61FB71F8093371290933812A0933912D2
:100C4000B0933A124091A90A5091AA0A6091AB0A56
:100C50007091AC0A8091990A90919A0AA0919B0A8E
:100C6000B0919C0A840F951FA61FB71F8093A90AF5
:100C70009093AA0AA093AB0AB093AC0AB7FD1CC02C
:100C8000419A40913B1250913C1260913D127091FB
:100C90003E128091860A082E000C990BAA0BBB0B02
:100CA000840F951FA61FB71F80933B1290933C1291
:100CB000A0933D12B0933E124091AD0A5091AE0AFE
:100CC0006091AF0A7091B00A80919D0A90919E0A3E
:100CD000A0919F0AB091A00A840F951FA61FB71F6D
:100CE0008093AD0A9093AE0AA093AF0AB093B00A76
:100CF000B7FD1CC0429A40913F1250914012609142
:100D00004112709142128091870A082E000C990BB3
:100D1000AA0BBB0B840F951FA61FB71F80933F1212
:100D200090934012A0934112B09342124091B10AA5
:100D30005091B20A6091B30A7091B40A8091A10AED
:100D40009091A20AA091A30AB091A40A840F951FC2
:100D5000A61FB71F8093B10A9093B20AA093B30A5B
:100D6000B093B40AB7FD3AC0C0904312D090441279
:100D7000E0904512F09046124091880A042E000C33
:100D8000550B660B770B4C0D5D1D6E1D7F1D409343
:100D9000431250934412609345127093461240914F
:100DA000910A5091920A6091930A7091940A841B5F
:100DB000950BA60BB70B8093B10A9093B20AA09340
:100DC000B30AB093B40A90918B0A8091BD0A93FF45
:100DD00002C0815001C08F5F8093BD0A8091840062
:100DE0009091850082179307C8F38091A50A90918E
:100DF000A60AA091A70AB091A80AB7FD15C0409114
:100E0000910A5091920A6091930A7091940A841BFE
:100E1000950BA60BB70B8093A50A9093A60AA093F7
:100E2000A70AB093A80A40988091A90A9091AA0AAB
:100E3000A091AB0AB091AC0AB7FD15C04091910AE0
:100E40005091920A6091930A7091940A841B950BB9
:100E5000A60BB70B8093A90A9093AA0AA093AB0A9A
:100E6000B093AC0A41988091AD0A9091AE0AA091DE
:100E7000AF0AB091B00AB7FD15C04091910A5091E8
:100E8000920A6091930A7091940A841B950BA60BA9
:100E9000B70B8093AD0A9093AE0AA093AF0AB093BC
:100EA000B00A4298E15041F0809184009091850011
:100EB00082179307C8F38ACE809127029091280267
:100EC000A0912902B0912A02892B8A2B8B2B09F041
:100ED0009AC08091BE0A882309F455C0C090D10AF7
:100EE000D090D20AE090D30AF090D40A4091B90A87
:100EF0005091BA0A6091BB0A7091BC0A8091BD0AF8
:100F00004C155D056E057F0588F42091890A3091A6
:100F10008A0AE0918E0AF0918F0AE217F30730F403
:100F200081508093BD0A2150310915C0C416D506E1
:100F3000E606F706E8F42091890A30918A0A409182
:100F40008C0A50918D0A2417350790F48F5F809397
:100F5000BD0A2F5F3F4F30938A0A2093890A409140
:100F600023025091240260912502709126020EC046
:100F70008FEF9FEFDC018093230290932402A093D4
:100F80002502B09326024FEF5FEFBA018091BD0AB0
:100F900087FD03C080910B0103C080910B018095F8
:100FA0008074809309012091840030918500225E35
:100FB0003F4F8091BD0A8823F1F0439A80918400CD
:100FC0009091850082179307C8F38091BD0A87FF2F
:100FD00002C08F5F01C081508093BD0A4398809109
:100FE000BD0A882331F38091840090918500821797
:100FF0009307C8F3DCCF40932702509328026093F5
:10100000290270932A028091D50A9091D60AA09164
:10101000D70AB091D80A892B8A2B8B2B09F06AC387
:10102000A091D90AB091DA0A109739F1C090D10A8B
:10103000D090D20AE090D30AF090D40A4091CD0A21
:101040005091CE0A6091CF0A7091D00AC416D5068D
:10105000E606F706C8F01092CC0A1092DA0A10924F
:10106000D90A9091830E8091840E981731F0809167
:10107000840E8F5F8F708093840EA0ED8A2EA7E080
:101080009A2EA12CB12C81C14091C80A5091C90A55
:101090006091CA0A7091CB0A4C155D056E057F05FB
:1010A00008F46EC04091C40A5091C50A6091C60A06
:1010B0007091C70AD2960D911D912D913C91D597B3
:1010C000EE27419FF12D529FC001629F900D619FBD
:1010D000800D911D429FF00D811D9E1F519FF00DAF
:1010E000811D9E1F609FF00D811D9E1F509FF10D61
:1010F0008E1F9E1FF6958E1F9E1F349F800D911D83
:10110000359F900D1124FD01EA5BFF4F0081118195
:1011100022813381080F191F211D311D0093C00A40
:101120001093C10A2093C20A3093C30A3497808077
:101130009180A280B38080169106A206B30640F487
:101140008092C00A9092C10AA092C20AB092C30AC9
:101150008090C00A9090C10AA090C20AB090C30AC1
:1011600088EF9FE177247394FC01059115912591F7
:101170003491081519052A053B0508F432C33CC310
:101180002091B90A3091BA0A4091BB0A5091BC0A29
:1011900029833A834B835C832C153D054E055F05FF
:1011A00008F068C04091B50A5091B60A6091B70A3C
:1011B0007091B80AD2960D911D912D913C91D597C1
:1011C000EE27419FF12D529FC001629F900D619FBC
:1011D000800D911D429FF00D811D9E1F519FF00DAE
:1011E000811D9E1F609FF00D811D9E1F509FF10D60
:1011F0008E1F9E1FF6958E1F9E1F349F800D911D82
:10120000359F900D11248C0120E030E04090C00A01
:101210005090C10A6090C20A7090C30AFD01E65B5B
:10122000FF4F041515052605370580F48080918051
:10123000A280B380401A510A620A730A4814590402
:101240006A047B0438F42401350104C040805180D5
:101250006280738088EF9FE131E03E83FC0105915D
:10126000159125913491041515052605370508F4C7
:1012700040C34CC38091BD0A8823D9F0D8964D91C4
:101280005C91D99760E070E00091230210912402F4
:1012900020912502309126020417150726073707EB
:1012A00041F0109227021092280210922902109207
:1012B0002A0240911F0250912002609121027091F8
:1012C000220277FF5AC0AE5BBF4F8D919D910D906A
:1012D000BC91A02D28EF3FE141E0F901C590D590E8
:1012E000E590F490C816D906EA06FB0658F4B695C0
:1012F000A79597958795440F2C5F3F4F50E2243177
:10130000350759F74093BF0A80329105A105B10511
:1013100008F4EBC38097A109B1098115E8E09E07A5
:10132000A105B10508F4BCC324E0929FF00111248B
:101330009F012850344EF901329645915491EE2781
:10134000859FB001849F610D7E1F06946E1F7E1FD6
:101350001124AB0160E070E0F90185919491A0E067
:10136000B0E0841B950BA60BB70B80931F029093E4
:101370002002A0932102B093220280901F0290903D
:101380002002A0902102B09022028091D90A90916F
:10139000DA0A892B09F0A6C1BBD99093DA0A8093A7
:1013A000D90A892B09F49EC16090D90A7090DA0A93
:1013B000D3018C9183FF3FC0F30185899689A7896A
:1013C000B08D8093371290933812A0933912B09356
:1013D0003A12818D928DA38DB48D80933B129093A0
:1013E0003C12A0933D12B0933E12858D968DA78D31
:1013F000B0A180933F1290934012A0934112B093FA
:10140000421281A192A1A3A1B4A18093431290930F
:101410004412A0934512B09346129091830E80918E
:10142000840E981709F4B8CF8091840E8F5F8F7067
:101430008093840EB1CF5596CD90DD90ED90FC90C9
:10144000589781E0C114D104E104F10409F480E06B
:10145000F301018D128D238D348D011511052105A8
:10146000310509F08260D3015D964D915D916D91DA
:101470007C919097411551056105710509F08460D3
:101480008093CC0A1092B50A1092B60A1092B70A4D
:101490001092B80A1092C40A1092C50A1092C60A95
:1014A0001092C70AF30185A196A1A7A1B0A58093C8
:1014B000CD0A9093CE0AA093CF0AB093D00A882485
:1014C00099245401881A990AAA0ABB0A8092B10A7F
:1014D0009092B20AA092B30AB092B40A8092AD0A76
:1014E0009092AE0AA092AF0AB092B00A8092A90A76
:1014F0009092AA0AA092AB0AB092AC0A8092A50A76
:101500009092A60AA092A70AB092A80ACC0CDD1C61
:10151000EE1CFF1CC092950AD092960AE092970AA0
:10152000F092980A000F111F221F331F0093990A8F
:1015300010939A0A20939B0A30939C0A440F551FDC
:10154000661F771F40939D0A50939E0A60939F0ADF
:101550007093A00A41A152A163A174A1440F551F29
:10156000661F771F4093A10A5093A20A6093A30AB3
:101570007093A40A880F991FAA1FBB1F8093910A1A
:101580009093920AA093930AB093940A1092D10A6E
:101590001092D20A1092D30A1092D40A82A593A56F
:1015A000A4A5B5A58093C80A9093C90AA093CA0AB6
:1015B000B093CB0A86A597A5A0A9B1A98093B90A33
:1015C0009093BA0AA093BB0AB093BC0A81A58093FA
:1015D000900A97A99093BE0A992361F024AD35AD86
:1015E00030938F0A20938E0A22AD33AD30938D0A4B
:1015F00020938C0AD301D6969C9120918B0A92134A
:101600000AC020911E0230E0482F082E000C550B16
:101610004217530729F090938B0A80931E0210DA29
:10162000A5D72FEF3FEFA90120931F02309320028F
:101630004093210250932202F301EA5BFF4F808125
:101640009181A281B3818093C00A9093C10AA09333
:10165000C20AB093C30A28EF3FE141E0F901C59007
:10166000D590E590F490C816D906EA06FB0658F422
:10167000B695A79597958795440F2C5F3F4FE0E26D
:1016800024313E0759F74093BF0A80329105A105E6
:10169000B10508F452C28097A109B109811538E05B
:1016A0009307A105B10508F425C244E0949F900179
:1016B00011242850344EF901329645915491EE2769
:1016C000859FB001849F610D7E1F06946E1F7E1F53
:1016D0001124F90185909490A12CB12C861A970AB7
:1016E000A108B1088092D50A9092D60AA092D70A92
:1016F000B092D80A0091D50A1091D60A2091D70A43
:101700003091D80A40912702509128026091290215
:1017100070912A027801F22FE32F401751076207D8
:10172000730718F47A01F62FE72FC701AF2FBE2FEA
:101730000097E1E0AE07B10520F08FEF9FEFA0E04A
:10174000B0E0081B190B2A0B3B0B0093D50A109332
:10175000D60A2093D70A3093D80A4F3FFFEF5F078E
:101760006F077F0761F0481B590B6A0B7B0B409397
:101770002702509328026093290270932A02F8945A
:101780002091840030918500205F3F4F4D81415072
:101790004D83442339F0280E391E2216330608F4EF
:1017A000B0C901C019013092890020928800789454
:1017B00026960FB6F894DEBF0FBECDBFDF91CF9156
:1017C0001F910F91FF90EF90DF90CF90BF90AF905F
:1017D0009F908F907F906F905F904F903F902F9051
:1017E0000895B694A79497948794770C0496E0E2B2
:1017F00084319E0709F0B8CC7092BF0A80E2881647
:101800009104A104B10408F41CC190E2891A910862
:10181000A108B1088114E8E09E06A104B104F8F023
:10182000F4E09F9EC00111248850944EFC01329632
:1018300025913491F82DEE27F39F8001F29F010D41
:101840001E1F06940E1F1E1F1124FC0185909490EC
:10185000A12CB12C801A910AA108B10823C09501CE
:1018600084013695279517950795F801EC7F9F0120
:101870002850384EF90185919491F90132960591DD
:101880001491E82DE770E09F9001E19F300D112445
:10189000F3E036952795FA95E1F74C01821A930A01
:1018A000A12CB12C480D591D6A1D7B1D4093C40A03
:1018B0005093C50A6093C60A7093C70A8091BE0A06
:1018C000882359F0472D50E060E070E0C416D5063B
:1018D000E606F70609F06CC084C02FEF3FEFA901C0
:1018E0002093230230932402409325025093260232
:1018F0009AC076946794579447942E81220F2E8332
:10190000049630E28431930709F0A8CC2E8120930D
:10191000BF0A30E2431651046104710408F4BAC0EE
:1019200080E2481A510861087108411498E059068C
:101930006104710408F48BC0E4E05E9EC0011124D0
:101940008850944EFC01329605911491F42DEE27A7
:10195000F19F9001F09F210D3E1F06942E1F3E1F08
:101960001124FC0185909490A12CB12C821A930A29
:10197000A108B108480D591D6A1D7B1D4093B50A89
:101980005093B60A6093B70A7093B80A8091BE0A62
:101990008823F1F149815A816B817C812E81420F2C
:1019A000511D611D711D4C155D056E057F05C8F447
:1019B0008091BD0A882309F4E8CCD8964D915C91BA
:1019C000D99760E070E000912302109124022091E9
:1019D000250230912602041715072607370709F458
:1019E000D4CC109227021092280210922902109251
:1019F0002A02D8968D919C91D997A0E0B0E080936F
:101A0000230290932402A0932502B0932602BDCC1A
:101A10008FEF9FEFDC018093230290932402A09329
:101A20002502B09326028091BD0A882309F4ADCC2B
:101A300010922702109228021092290210922A0274
:101A4000A4CC00E2802E912CA12CB12CDECE9301EF
:101A500082013695279517950795F801EC7FCF0100
:101A60008850984EFC0185909490FC013296259107
:101A70003491E42DE770E29FC001E39F900D1124A3
:101A800023E0969587952A95E1F7881A990AA12C63
:101A9000B12C70CFF0E24F2E512C612C712C40CF25
:101AA000AC01BD017695679557954795FA01EC7F96
:101AB000AF014850584EFA0125913491FA013296FF
:101AC000459154918770849FB001859F700D1124BA
:101AD000CB01F3E096958795FA95E1F7A901481BAC
:101AE000590BCA01A0E0B0E040CC80E290E0A0E059
:101AF000B0E010CCAC01BD01769567955795479540
:101B0000FA01EC7F9F012850384EF901859094909E
:101B1000F9013296259134918770829FA001839FAD
:101B2000500D1124CA0123E0969587952A95E1F777
:101B3000881A990AA12CB12CD5CD80E290E0A0E0C2
:101B4000B0E0A9CD8F929F92AF92BF92CF92DF92D9
:101B5000EF92FF920F931F93CF93DF9300D01F92CA
:101B6000CDB7DEB78BE4882E85E1982E97E4A92EB9
:101B700092E1B92E01EE14E0C12CD12C7601C39470
:101B8000F40161917191819191914F01F501219140
:101B90003191419151915F0129833A834B835C8359
:101BA0000F94FF2F29813A814B815C810F94603023
:101BB0000F94AE35F80161937193819391938F01E6
:101BC000C616D706E806F90610F46B017C01FBE5A2
:101BD0008F16F5E19F06A1F66FEF7FEFCB01A7010E
:101BE00096010F9407342093DD043093DE04409374
:101BF000DF045093E0040F900F900F900F90DF914F
:101C0000CF911F910F91FF90EF90DF90CF90BF90F9
